:020000040000FA
:100000000882012001210000CD5C00006121000078
:1000100061210000612100006121000061210000D8
:10002000000000000000000000000000151F00009C
:10003000612100000000000000000000B15C000031
:10004000D9200000D9200000D9200000D9200000CC
:10005000D9200000D9200000D9200000D9200000BC
:10006000D9200000D9200000D9200000D9200000AC
:10007000D9200000D9200000D9200000D92000009C
:10008000D9200000D9200000D9200000D92000008C
:10009000D9200000D9200000D9200000D92000007C
:1000A000D9200000D9200000D9200000D92000006C
:1000B000D9200000D9200000D9200000D92000005C
:1000C000D9200000D9200000D9200000D92000004C
:1000D000D9200000D9200000D9200000D92000003C
:1000E000D9200000D9200000D9200000D92000002C
:1000F000D9200000D9200000D9200000D92000001C
:10010000D9200000D9200000D9200000D92000000B
:10011000D9200000D9200000D9200000D9200000FB
:10012000D9200000D9200000D9200000D9200000EB
:10013000D9200000D9200000D9200000D9200000DB
:10014000D920000053B94AB9002908BF00281CBFB4
:100150004FF0FF314FF0FF3000F080B9ADF1080CE7
:100160006DE904CE00F006F8DDF804E0DDE90223D5
:1001700004B070472DE9F04F099D04468846002BD6
:1001800040F084808A42174643D9B2FA82F242B1E3
:10019000C2F120009140974024FA00F0944040EAD8
:1001A00001084FEA174C230C1FFA87FEB8FBFCF638
:1001B0000CFB168106FB0EF043EA0143984207D977
:1001C000FB1806F1FF3102D2984200F231810E464F
:1001D000191AA3B2B1FBFCF00CFB101100FB0EFED0
:1001E00043EA0144A64507D93C1900F1FF3302D286
:1001F000A64500F21A81184640EA0640A4EB0E0418
:1002000000261DB1D4400023C5E900433146BDE8B6
:10021000F08F02B9FFDEB2FA82F2002A52D1CB1B74
:100220004FEA174E1FFA87F80126210CB3FBFEFC9C
:100230000EFB1C3008FB0CF941EA004189450BD943
:1002400079180CF1FF332CBF01200020894502D919
:10025000002800F0F0809C46A1EB0901A3B2B1FB9D
:10026000FEF00EFB101108FB00F843EA0144A04524
:1002700007D93C1900F1FF3302D2A04500F2D28029
:100280001846A4EB080440EA0C40BAE78B4209D9AF
:10029000002D00F0BE800026C5E900013046314641
:1002A000BDE8F08FB3FA83F6002E4DD18B42C0F03B
:1002B000B380824240F2B0803046002DA6D0C5E91E
:1002C0000048A3E79740C2F1200301FA02F04FEA89
:1002D000174ED94024FA03F31FFA87F894400343DA
:1002E000B1FBFEF01E0C0EFB101100FB08FC46EAF1
:1002F00001418C450ED9791800F1FF362CBF4FF023
:1003000001094FF000098C4503D9B9F1000F00F045
:1003100096803046A1EB0C019BB2B1FBFEF60EFBC2
:10032000161106FB08FC43EA01418C4507D97918F0
:1003300006F1FF3302D28C4500F288801E46A1EB05
:100340000C0346EA004670E7C6F1200703FA06F4FC
:1003500002FA06FC01FA06FEFA4020FA07F8F94014
:1003600000FA06F3224348EA0E044FEA12484FEA25
:10037000144E1FFA82F9B1FBF8FA08FB1A110AFBB6
:1003800009F04EEA014E70450ED912EB0E0E0AF13D
:10039000FF312CBF4FF0010B4FF0000B704502D91D
:1003A000BBF1000F4ED08A46AEEB000EA4B2BEFBEE
:1003B000F8F008FB10EE00FB09F944EA0E4EF14597
:1003C00007D912EB0E0E00F1FF3101D2F14540D8F2
:1003D000084640EA0A40AEEB090EA0FB0C89CE4568
:1003E00041464C4602D306D1434504D20138B8EB0E
:1003F0000C0169EB02047DB35A1A6EEB040EF24055
:100400000EFA07F72EFA06F300261743C5E9007324
:10041000FCE62E462846F9E6841A61EB030101202A
:1004200088464AE702383C442BE702383C44E3E67E
:10043000023E3B44CCE6ACF1020C39440CE70238F6
:10044000394467E7AAF1020A9644ADE7023E39440F
:1004500075E702389644BCE72E46D7E6704700BFE2
:100460007FB5314B314A3248C3F800264921C3F8E1
:100470000426C3F80826C3F80C26C3F81026C3F8D0
:100480001426C3F81826C3F81C2605F0BEFA04F09B
:1004900076FE284800F05EF828B94521254A26480E
:1004A00005F0B3FAFEE701A800F066FC234B1B68D9
:1004B000834204D04521224805F0A7FAFEE74921EE
:1004C000039A204805F0A1FA49211F4805F09DFA3A
:1004D0004FF48031002002F011FE20B145211B486D
:1004E00005F093FAFEE769469DF8080000F03EF833
:1004F000009B039C1C44019B1D8966194FF0200240
:10050000EFF3118382F31188BFF36F8F05F0D1FBF6
:1005100000F016FF635983F30888736898474521F4
:100520000B4805F072FAFEE7008001503546526E26
:1005300010690000296900003C690000BC460120E8
:100540005B6900007E690000AD690000D2690000AF
:10055000056A000010B5044C236813B903F07CF958
:100560002060206810BD00BFB846012008B540B12A
:10057000024600230448452105F047FA6FF01500B4
:1005800008BD0860FCE700BF286A00002DE9F04FB5
:10059000DFF81C92DDB01546DDE968481E46DDF83F
:1005A00098B1D9F8007000F099FE01227E4B3CA86A
:1005B000C3F8002503F014FDCDF814903CB1B8F158
:1005C000000F04DD424621463CA805F028F94FF013
:1005D00000096B89B5F808809844EB689844C845D1
:1005E0004ED80FA93CA803F06DFD00226E4BC3F856
:1005F0000025C3F800256A9B23B1202218460FA9C5
:1006000005F0A2FB00233246009329464FF6FF7304
:1006100009A804F0B5FD0446002844D14FF0FF3589
:10062000DFF890A1DFF8808103900DF11E0307AA87
:1006300008A909A804F0F0FD041E34DB40F0A480F2
:10064000BDF81E90B9F1100F38D1BDF81C90B9F16A
:10065000200F40F0A3804B46304608993CAA05F095
:1006600002FA0446F8B94A463CA90FA804F04BFE2A
:1006700004464E4B1B68834215D101230393D4E7F4
:10068000679AA8EB09039A4228BF1A4649461346BF
:10069000924630465A4605F0E6F9044638B1002243
:1006A000414BC3F8002520465DB0BDE8F08F5246AF
:1006B00059463CA805F0B3F8D14490E7B9F1010FD1
:1006C0003FD1BDF81C30202B68D8304608993CAA91
:1006D00005F0C9F904460028E5D19DF81C50202DED
:1006E0000AD8DAF80030DFF8D0B00493049B9C42BB
:1006F00005DB0023C8F800354FF0FF341DE000F0A3
:10070000EDFDC8F800951FA803F06AFCDBF8042093
:100710001FA812685BF8081B05F081F817A91FA82D
:1007200003F0D0FC00223CA9C8F8002517A82A46EF
:1007300005F0FAFA18B9C8F80005254675E701343E
:10074000D4E7B9F1220F7FF470AF002D19DBDAF88E
:100750000030AB4215DDBDF81C30802B1ED8304672
:1007600008993CAA05F07FF9044600289BD1EDB218
:100770002021BDF81C3000953CAA0FA800F01EF8FF
:1007800007464FF0FF3550E7039B53B1074B1B68FB
:10079000BB4201D0059B1F683C4684E74FF0FF3405
:1007A00081E701247FE700BF00008450BC460120A0
:1007B00000450120C8650000CC6500002DE9F0412E
:1007C00096B017461D469DF87020354B0E4653F8DF
:1007D000321003EBC2035B68804618680191302336
:1007E000014402AA01A804F0A7FF10B14FF0FF30A6
:1007F00053E0DDE901431C44214606AB03AA01A8EE
:1008000004F0C2FF0028F1D1049A072AEED125494D
:10081000059805F089FA0028E8D1079A082AE5D159
:100820002149089805F080FA0028DFD1214602AA64
:1008300001A804F095FF0028D8D1DDE90132134466
:100840009C42D3D1412AD1D13D443023294603AA29
:1008500002A8029704F070FF0028C7D1DDE9023238
:1008600013449D42C2D32A4602A906A804F01FFDE4
:100870000028BBD12A4602A90EA804F018FD0028C2
:10088000B4D1202EB2D101990B78042BAED13346CE
:10089000404606AA013100F039FD16B0BDE8F081EE
:1008A000CC6500004E6A0000566A00002DE9F04158
:1008B000032386B00D466F460026DFF86C80ADF846
:1008C000003017F8010B01A901F0F2F80446D8B97D
:1008D00001981023816802AA103905F0C4F8044673
:1008E00028B1019805F0BEF80EE00126E9E71022D4
:1008F000414602A805F018FA50B1019805F0B2F887
:10090000002EF2D04FF0FF34204606B0BDE8F08153
:10091000019805F07CFB0423A0F108012A46019808
:1009200005F0A1F80446DCE7646700002DE9F0411A
:10093000384B88B0064600200D461C6804F016FCB3
:1009400006A9C0B201F0B4F8002857D1294604F036
:100950000DFC2C2407A9C0B204FB056401F0A8F823
:10096000002836D04FF02C0808FB05F806EB0807E6
:10097000396911F0100137D14FF480730193264B80
:10098000224600930846CDE90311069B0291FFF72A
:10099000FDFD0446214B56F8082006989A420CD1DA
:1009A0003A89FB68D1438B4207D81344826893424B
:1009B00003D21B4B1B68A3421DD045B382680021A4
:1009C00005F0A0F8174A4521174805F01EF8012444
:1009D00011E0079805F0CFF80746079805F042F8B0
:1009E000631EE21C93420DD1002DF0D030460699D3
:1009F00004F083FD2C46069805F034F8204608B034
:100A0000BDE8F08113F8011FB942EBD0AAE7074A0D
:100A1000D9E700BF00450120F05401203DB8F3960E
:100A2000BC4601205F6A0000716A0000696A00002C
:100A300073B50D46002104462846CDE9001104F0A7
:100A40001BFD30B3164E2268B24203D1204601AAE4
:100A500004F089FCE36AB34204D16A4601212046CE
:100A600004F081FCDDE90032934288BF0193019BD1
:100A7000AB60019A2946204600F020FB094B1A681A
:100A8000002A03DD5721084804F0BFFF002002B010
:100A900070BD05F10801FFF709FFAB680193E8E7B6
:100AA0003DB8F396204F0120996A00002DE9F84FD8
:100AB0008A46904699460026DFF870B0194C1A4DC8
:100AC0000B9B9E4201D300200FE00B9B50469F1BC7
:100AD000B7F5806F28BF4FF48067144A3B4606EB9A
:100AE000090104F0C0FF10B10120BDE8F88F0A9998
:100AF0003B465A464046711804F0D2FF0028F3D115
:100B0000C4F800563E44C4F80456C4F80856C4F865
:100B10000C56C4F81056C4F81456C4F81856C4F845
:100B20001C56CDE7008001503546526EF050012032
:100B30002DE9F043884B0446602285B00F46002122
:100B40001E6805F02CF90021844B08466362844B33
:100B5000236504F00BFB04F12001C0B200F0A8FFF4
:100B60000121002004F002FB04F14C01C0B200F0AE
:100B70009FFF0546204604F057FC024630B1802214
:100B80005721784804F041FF01238DE001462046BB
:100B900004F031FC804618B1002257217248F1E779
:100BA000204600F0A3F90028EED0684604F05BFC74
:100BB0006946204604F0F6FC18B1424657216B48BE
:100BC000E0E7684604F058FC80F001006A46C1B2D4
:100BD000204604F010FC02460028DDD1684604F0EF
:100BE0004BFC804660BB69462046FFF721FF9DF81D
:100BF000073084F85830033B012B06D8404604F0F8
:100C00001FFD10B1FF2384F858309DF80730023BD8
:100C1000022B0BD8002004F001FD38B1FF2384F82B
:100C200058304521524804F0F0FEFEE794F8583061
:100C3000FF2BF6D06A460021204604F0DCFBA3E738
:100C40009DF80790B9F1010F23D1104602F0DCFAAC
:100C5000831E022B80460DD849462046FFF766FECC
:100C6000444B1B68984205D001280CBF4FF0010887
:100C70004FF0050884F8588094F85830042B8DF80C
:100C8000073014D8012B18D82FD0FF2384F8583000
:100C90002BE001212046FFF749FE364B1B689842A6
:100CA00014BF05239DF8073084F85830E4E7052B7E
:100CB000EBD1002004F0C4FC12E069462046FFF7A7
:100CC000B7FE94F858300546DA1E012A0BD80020EA
:100CD00004F0B6FC05460028D7D1002004F09EFCA5
:100CE000054610B1D1E7022BF7D094F85830FF2B0E
:100CF00004D145211E4804F088FEFEE7012B06D0F2
:100D00006A460021204604F076FB0546B8B900216A
:100D10002046FFF70BFE0646DFF85880D8F8003073
:100D200098420CD110220021684605F038F8236A59
:100D3000D8F800605A783A715B683C60BB60E06C40
:100D400004F090FE206A04F08DFE002D14BF2846AA
:100D5000304605B0BDE8F083004501202047012062
:100D6000204B0120C86A00000A6B0000366B0000AF
:100D7000606B0000BC46012008B501460148FFF742
:100D8000D7FE08BDC046012073B516461C4633B3D6
:100D9000436A5D686379012B15D101BB1F4B226843
:100DA0001B689A4298BF0025002004F0DFF901A9D2
:100DB000C0B200F07DFEF0B10125019804F052FEB2
:100DC000284602B070BD022B09D12368012B08D937
:100DD000124A1268934202D8B1FA81F149090025FA
:100DE000E2E7FCD10029DFD00129F8D121790239CD
:100DF00018BF0121F3E7294620233246019804F069
:100E000032FE05460028D7D1002CD6D035680448DC
:100E10002D1A18BF4FF0FF35CFE700BF0445012062
:100E20003DB8F3962DE9F04F07460C4685B00146D4
:100E30000020164604F06EFA051E51DB3846E46DBC
:100E400004F072FA5FFA84F94FF0000A4FF0010BD8
:100E50004FF0FF3405F1FF3809FB08089DB9BAF1DE
:100E6000010F03DD4521204804F0CFFD631C06D0AF
:100E70007F2C2ADC40F2011301343460B380284611
:100E800005B0BDE8F08F6B1E009341460123384644
:100E90000DF10F0204F0E7FD031E019322DB012296
:100EA00038460DF10F0105F0C3F8019B40B15B45D9
:100EB00001D00AF1010A9B46009DA8EB0908CDE785
:100EC000B4F1FF3F08BF2C46F5E70223803C737165
:100ED000631004F001040133013433603471CEE750
:100EE0000725CCE70125CAE76C6B0000816A426DDB
:100EF00038B5914208D0531C8B4205D05721134876
:100F000004F083FD002038BD80291CD957211048EA
:100F1000F6E7446A056D04EBC30405EBC30564689A
:100F20006D68AC4202D057210A48E9E701339A4282
:100F3000EFD1914205D9436A03EBC2025368A34241
:100F4000F1D10120DFE700231C46F0E78F6B0000A2
:100F5000C76B0000F66B000000B589B0032004A940
:100F600005F0C9F89DF81020012A41D0254B2649EB
:100F7000032A18BF0B469DF81320492102929DF8C1
:100F80001220224801929DF811200092204A04F07C
:100F90003CFD072006A905F0AEF89DF81820012AAF
:100FA00028D0184B1849032A18BF0B469DF81B2060
:100FB000492102929DF81A20144801929DF81920A7
:100FC0000092144A04F021FD9DF81030012B13D13A
:100FD0009DF81230032B0FD19DF81830012B0BD048
:100FE0000D48492104F011FD022009B05DF804FB11
:100FF0000A4BC0E7094BD9E70948492104F005FD30
:101000000020F2E7276C00002D6C00003F6C000010
:10101000316C0000806C0000906C0000226C0000BD
:10102000AF6C000070B5064618464B6814461D4A62
:1010300003F0FF2393420D4686B02ED10B68012B9F
:101040002BD104A905F057F89DF81020012A26D0CD
:10105000154B1649032A18BF0B469DF8132049214A
:1010600002929DF81220124801929DF811200092E0
:10107000104A04F0CAFC9DF81030032B0DD1214614
:10108000304604F03AFA204605F02CF82046A968CC
:1010900004F05AF9204602F059F806B070BD064B2C
:1010A000DBE700BF00010004276C00002D6C00008E
:1010B0003F6C0000806C0000226C00002DE9F04FB6
:1010C000436A2DED028B0C465E6805460121002324
:1010D0008BB033449A42084601F10101F9D8784FA8
:1010E0003860204604F0C8F9BB46C8B1E86D04F08A
:1010F0000CF90022AB6A013B3244824201D2013B2F
:10110000FAE7DBF800209A420AD357216D4804F031
:101110007CFC0123E3710BB0BDEC028BBDE8F08FCA
:1011200008A9032000F0C4FC09A9072000F0C0FCB6
:10113000072321462846099AFFF774FF6379012B9C
:1011400008D1DBF80070DFF880A1DBF80030A7B928
:101150000123236002230127DFF86C81637105936B
:10116000DBF80030DDF820909F424DD9484604F06E
:1011700079FC099804F076FCCDE7226801339B1ACC
:101180009F423FD86B6A012A196853F8370003EB76
:10119000C70353F8083CDDF82080A3EB010308EEF9
:1011A000103AA0EB010912D1E268099B022A0AD089
:1011B00041462846039304F0A0F9224641462846BA
:1011C00004F0D1F9039B1946284604F096F93246FB
:1011D0004946404604F08FF918EE103A424641461F
:1011E0002846CDE90096FFF761FC2146284604F029
:1011F00050F923680133236020B1DAF8003001335D
:10120000CAF80030013FA0E723689F4256D3696ABD
:10121000286D51F83730FA0004930B68083A50F8FB
:1012200002C0039303682079DDF824A00128ACEB09
:10123000030341D189580793039B3246C91A484694
:10124000069104F058F90699079B4A4600912846F2
:10125000514601960693FFF729FC2146284604F0E3
:1012600018F9059B2371069B20B1D8F800200132A4
:10127000C8F80020194632465046069304F03BF960
:10128000069B494600932846DDE9032301969B1AF5
:101290005246FFF70BFC2146284604F0FAF8236873
:1012A000013323604FF00103237138B1D8F80030C7
:1012B0000133C8F8003001E00228DBD001374FE7E6
:1012C00004450120C66C0000204F0120024B0A4655
:1012D0001B680021184700BF0845012070B5094D63
:1012E0002B7853B90126084CC4F8006502F01AFFA8
:1012F00028B92E70C4F8000570BD0020FCE74FF03F
:10130000FF30F9E7F05501200000845070B5AEB011
:101310001D460446CDE90221FFF7E0FFDDE9022189
:101320000123064E05A8C6F800352346009504F0B3
:1013300090FF0023C6F800352EB070BD0000845029
:101340000122124B12491A604FF0FF33C1F84833A3
:10135000C1F8083301F580514A60043100210D4A7B
:10136000C2F84833C2F80833A2F55042C2F800155B
:10137000C2F8083302F58052C2F80015C2F80833EB
:101380004FF05022C2F80833704700BF04400150AC
:1013900000400150005001500B6801330B60014BBD
:1013A0001B6818470C450120014B1860704700BFAF
:1013B0000C45012007B50B46002102460191034868
:1013C00001A900F0E9F803B05DF804FB99130000EF
:1013D0002DE9F74FB0F81890044619F00808934625
:1013E0000ED001290CBF49F0100949F02009A0F8DE
:1013F00018908BF31188BFF36F8F03B0BDE8F08FA7
:10140000DFF890A109F00709022907D1204604F06E
:101410004DFA0028EDD00128238B4BD16769218B31
:10142000002F15DA256821F00701C4E9008841F092
:10143000010121830026218B01F007024A4502D0D9
:10144000A368002B57D10DB9002E6FD0002353E0B5
:1014500001F007035A1F012A1DD821F00701062BAE
:10146000256889B2C4E900880AD13DB12A46638B58
:10147000126801339BB2002AFAD1638341F0020162
:101480002046218304F012FA0028D3D0238B43F0A6
:1014900020032383CEE7042B0AD121F0070189B270
:1014A0002046218304F002FA10B141F0200121838B
:1014B0000025BFE7032809D1226923F00703166836
:1014C00043F00603002523832F46B4E7042806D102
:1014D000226923F00703566843F00403F2E7052866
:1014E00006D1226923F00703966843F00503E9E774
:1014F00000252E46E8E7012341F0080121838BF304
:101500001188BFF36F8F03BB002D31D116B1514647
:101510002046B0474FF02003EFF3118B83F311887F
:10152000BFF36F8F238B23F008032383238BDA060B
:1015300027D5012123F010032383B4F8189009F074
:10154000070900297FF460AF53E7A1680029DBD0C9
:10155000D1F800903B462046D1F804B00192D8471C
:10156000019AB9F1000FCFD04946D9F80090F1E7C0
:1015700029463B46204601922D6804F0B3F9019AB2
:10158000C2E713F020011EBF23F0200302212383B2
:10159000D3E700BF115900002DE9F04F8B464FF003
:1015A000000A8FB01F46531E00900193019B58788C
:1015B0005C1C252822D100204FF0FF36014634461E
:1015C0004FF00A0E03F1020C02909CF80020CDF8B7
:1015D00004C0392A0CF1010C58D81F2A18D8002A47
:1015E00000F005825946009B25209847019B5946EB
:1015F0001878009B98470AF1020AD7E7002800F004
:10160000F6815946009B98470AF1010A0194CDE7FB
:10161000A2F12003192BE5D801A555F823F000BF4E
:1016200089160000E5150000E51500008916000088
:10163000E515000009170000E5150000E51500009C
:10164000E5150000E51500004B17000089160000A5
:10165000E51500005F17000017170000E5150000F2
:10166000231700003F1700003F1700003F1700003E
:101670003F1700003F1700003F1700003F17000012
:101680003F1700003F17000010469EE7582A00F061
:101690004581A2F16303DDB2172DA3D8172BA1D882
:1016A00001A555F823F000BF791900008517000047
:1016B000E5150000E5150000E515000065170000C0
:1016C00085170000E5150000E5150000651700000E
:1016D000E5150000E5150000E5150000C318000041
:1016E000E5150000E51500005B190000E515000098
:1016F00085170000E5150000E5150000C31800007F
:10170000E51500006517000059462520009B984705
:101710000AF1010A4AE7029B002603F0FE03029346
:1017200053E7002C0BDA002E0BDA029B002B00F0A3
:101730005A8124EAE4740EFB0424303C45E7002E71
:10174000F7DB0EFB0626303E3FE7002E57F8043B42
:1017500001DB1E4639E71C1EBFF637AF6442022389
:10176000029332E7682A03D1682906D148212CE781
:101770006C2A02D16C2900F0388100297FF432AF45
:10178000114622E77A2908D13D4655F8043B984690
:101790004FEAE379752A19D111E06C29F4D04C296C
:1017A00005D1FD1D25F00705F5E80289F2E73B6844
:1017B000752A984607F1040506D14FF00009202844
:1017C00078D18D4F013C0CE04FEAE379B8F1000F7E
:1017D00079F10003F3DAD8F10008884F69EB490981
:1017E000013C0DAB079300230393039B40460693F4
:1017F000013B494603930A220023FEF7A3FC079B03
:10180000303203F8012940460A2249460793002353
:10181000CDE90489FEF796FCDDE90423002B08BF1F
:101820000A2A80468946E0D2069B0EAAC3F1010926
:1018300003EB0208002EA8F1040804DA029B13F05F
:10184000010F18BF2646A6EB0903002B0393029B4A
:10185000D4BFA4EB0904A41B9A0740F1AE80AAEB05
:10186000070606EB070A17F8010B002840F0A780CF
:10187000039E013E40F1A780039B4E465A1E013253
:10188000ACBF1F460027013E40F1A28009F1FF32A4
:101890000132ACBF4B460023264603EB0709013E4D
:1018A00040F19C80631E0133B8BF0024A1442F4641
:1018B000CA447BE62B280ABF514F524F04F1FF3434
:1018C0008FE7702A2AD13D4655F8041B00295DD0C8
:1018D00088464FF000094C4F023C02F06002A2F132
:1018E000390E00220DF1340C08F00F03092B88BFCC
:1018F00073443033B9F1000F0CF8013908BFB8F167
:10190000100F4FEA181302F1FF3043EA09734FEA50
:1019100019111ED2C2F101090EAB89E76C2906D15B
:101920003D4655F8043B4FF00009984606E04C2927
:10193000F6D1FD1D25F00705F5E80289232806D11B
:10194000314B12F0200F314F18BF1F46C4E72D4F07
:10195000C3E7024698468946C6E73D4655F8048BDC
:10196000404604F0CEF9002E814602DBB042A8BF0B
:10197000B1460026234F66E73D4655F8043B4FF03D
:1019800001098DF820300DF12008F2E74FF005092C
:10199000DFF87C80EDE759462020009B9847013E08
:1019A000F9D5621E531CACBF21460021C4F10004CE
:1019B000B8BF00248A44144451E72646EFE759464D
:1019C000009B98474DE75946009B3020984750E7C9
:1019D000594618F8010B009B984754E75946009B5D
:1019E000202098475BE70123BAE64C21EDE55046FD
:1019F0000FB0BDE8F08F00BF52710000506D0000C5
:101A0000526D000068740000546D0000576D0000B6
:101A10005A6D000007B501904FF02002EFF31183DB
:101A200082F31188BFF36F8F04F043F9019800F03F
:101A300065FD034803F02DFF00F0D6FAFCE700BF78
:101A4000606D00004FF02002EFF3118382F31188E4
:101A5000BFF36F8F0121044AC2F8401583F3118848
:101A6000BFF36F8F002070470090035020B1034BED
:101A7000800143F001031847704700BFC0650000B4
:101A8000094B30B51D68094B1C6800239D4202DCE0
:101A90000021084630BD1A01A25C04EB031182420A
:101AA000F7D00133F2E700BFB06600001045012017
:101AB000084B10B51B680C462BB1FFF7E1FF28B1AE
:101AC0002060002010BD6FF00C00FBE76FF00100FC
:101AD000F8E700BF1045012030B589B00C46154627
:101AE0000190FFF7CDFFB8B1436822680293836885
:101AF000C068CDE903350023CDE90623059303F043
:101B000091FF60B1074901AA04F0CDF9079808B91F
:101B1000059B236009B030BD6FF01500FAE76FF048
:101B20001200F7E7295A000008B50448FFF73CFC0B
:101B3000024800F079FE002008BD00BF411B0000F4
:101B4000F7B5044603250F4E8DF80700EFF3118714
:101B50004FF0200181F3118801220DF107010020CF
:101B600001F026FE87F3118820B10123337020464F
:101B700003B0F0BD3378002BF9D0013DE6D13570CC
:101B8000F5E700BFF155012070B504460C250D485E
:101B90000E46231A9A100C4B40215343DBB25D438F
:101BA00005F14003184403F0F8FF011E04DB074B66
:101BB0002B445B689847002120463346BDE87040BF
:101BC000184700BF384F0120B76DDBB6EC65000049
:101BD0002DE9F0410F4C104D031B9B105D43EBB200
:101BE0000C255D43074605F140000E462044402188
:101BF00003F0ECFF011E08DB084B2C44C4E90E3651
:101C0000074B5B59BDE8F041184738463346BDE8FD
:101C1000F0411847384F0120B76DDBB6355C000046
:101C2000EC65000070B5002201210446052000F09B
:101C30009FF9052000F07EF90F4801F00DFC0F4BD5
:101C4000984215D104F07DFA26690D49304603F01B
:101C50007DFE00280BDB012535642469084904F169
:101C60001C0003F073FE002801DB0020E56470BD5A
:101C70006FF00400FBE700BFC11C00000000AD0BCB
:101C80000466000073B50C23014600264B430A4846
:101C9000C4184033D4E90E521844A663019203F0ED
:101CA000B3FF35B12B46019A044802B0BDE870403D
:101CB000184702B070BD00BF384F0120A445012075
:101CC00010B1012804D07047034B1B6C5B0701D196
:101CD000FFF7D8BF704700BF384F012008B54FF05D
:101CE0002003EFF3118183F31188BFF36F8F124A42
:101CF000136843F0020013F0010310600CD04FF0A2
:101D00005022D2F80C34D2F80C2413F0010303D083
:101D10000A4803F079FF012381F31188BFF36F8F25
:101D200023B1BDE808400020FFF7ACBF0120BDE8AB
:101D3000084001F0A1BB00BF884F0120784F01206F
:101D4000074BD3E8EF2F22F00201C3E8E01F002881
:101D5000F7D1D30702D4012001F0C0BB704700BF08
:101D6000884F01202DE9F843012206463649D1E883
:101D7000EF3FC1E8E02F0028F9D133B933493448A7
:101D80004B60CB608A6003F0F4FD731E012B32D8E8
:101D9000012E07D14FF05023D3F81C3403F0030376
:101DA000022B28D004F04AFA044618B9294B1B78B4
:101DB000002B41D14FF02003EFF3118583F31188FD
:101DC000BFF36F8F0124244FDFF89080DFF89090ED
:101DD0004FF05022D2F81834D2F81824D2030CD580
:101DE00003F00303022B01D0012E06D1F4B185F3D9
:101DF0001188BFF36F8FBDE8F883284600F002F921
:101E00004FF05022D2F81835DBB2012BE0D13968FF
:101E10000029DDD00021396039680221C2F8181587
:101E20002022C8F88021C9F80030D1E74FF05023B4
:101E30000222C3F80423DEE74FF0502302220546B6
:101E4000C3F80823BFE700BF8C4F0120284F0120B3
:101E5000544F0120045A01200451005000E100E0D9
:101E600008500050F8B5002427460F4E0F4B104A7B
:101E700018461D6804B1F8BDD2F80413C903FAD599
:101E800031680029F7D0346031684FF48031C2F8EE
:101E900048130124D2F8401525B100205A681F606C
:101EA000A847E3E70560E6E740510150944F012061
:101EB0000050015038B500244FF480334FF4001225
:101EC0000D4D0121C5F80845C5F804330B4B15200D
:101ED000C3F88021224600F04BF8152000F02AF8C4
:101EE0000123074A02201360064A2B601360FFF7A4
:101EF00039FF204638BD00BF0050015000E100E02E
:101F0000085001509C4F0120014801F0D7BD00BF8F
:101F1000B46600001EF0040F0CBFEFF30880EFF36F
:101F20000980816911F8021C0229FFD001B503F074
:101F3000C9FE01BD43B2002B08DB012200F01F00E7
:101F400002FA00F0024A5B0942F82300704700BF22
:101F500000E100E0054B420953F82220012300F084
:101F60001F0003FA00F01040704700BF00E100E0DE
:101F700043B2002B01F10101ACBF03F16043064BFA
:101F80004FEA4111C9B2ABBF03F5614300F00F0046
:101F900083F800131954704714ED00E00446084616
:101FA00011461A460023E1EE103A83F30B880A4BE0
:101FB0002025A3F5205686F30B8883F3098863B6A2
:101FC0004FF0000383F31188BFF36F8FA04785F3B1
:101FD0001188BFF36F8FFEE70882012001491022AC
:101FE0000A60704710ED00E072B6404080F311883F
:101FF000BFF36F8FBFF34F8F30BF62B6BFF36F8FEA
:10200000704700BF72B6494081F3118820BF80F34A
:10201000118862B6704700BF37B505460C46C9B196
:102020008B6810480093D1E90023452103F0EDFCB3
:10203000636945210093D4E903230B4803F0E5FCD1
:102040004521E269094803F0E0FC4521A2690848FE
:1020500003F0DBFC2146284603B0BDE8304001F028
:1020600027BC00BFB76D0000EB6D00001F6E0000C5
:10207000336E000030BFFFF7FDBF00BF144A08B544
:10208000144B22F07F029A60BFF34F8FBFF36F8F24
:10209000D3F8882022F47002C3F88820D3F888206F
:1020A00042F4A002C3F888204FF04042C3F8342223
:1020B000BFF34F8FBFF36F8F0023E1EE103A01F0B3
:1020C00035FC01F08BFC00F061FA01F051FC00BF1F
:1020D0000000000000ED00E001B5EFF30580A0F185
:1020E00010004FEAC0000449014409C99847BDE8FF
:1020F00001400249084700000C630000F924000079
:10210000002080F31488BFF36F8F002080F30A88CB
:1021100080F30B8803F077FC00200E490860BFF3C2
:102120004F8F0D4880F3088800F00AFA202080F3D2
:1021300011880A484FF40061401880F30988EFF3D2
:1021400014800221084380F31488BFF36F8FFFF7D8
:1021500095FF000094ED00E0088201200882012034
:10216000EFF30880EFF3098101B5724600F008F93A
:1021700001BD00BF70B5224C06460D4621484521E1
:1021800003F043FCA26AD00603D545211E4803F0A4
:102190003CFCA36A190703D545211C4803F035FC14
:1021A000174CA36A9A0710D54521194803F02DFC56
:1021B000626BA36A1B0608D54521164803F025FC6F
:1021C0001EB1A36A23F08003A3620D4CA26AD0075C
:1021D00003D54521104803F018FCA36A990603D5DE
:1021E00045210E4803F011FC0020054B9A6AD206E7
:1021F00058BF9A6A9A6A42F0FF029A62287070BDCC
:1022000000ED00E0666E0000816E0000B96E000017
:10221000D16E0000EE6E0000096F00002D6F00000F
:1022200070B5234C06460D462248452103F0EDFBD0
:10223000A26AD10403D545211F4803F0E6FBA36A37
:102240001A0503D545211D4803F0DFFB184CA36A8E
:102250009B0510D51A48452103F0D7FBA26BA36A52
:10226000180408D54521174803F0CFFB1EB1A36A17
:1022700023F40043A3620E4CA36A590503D54521FC
:10228000114803F0C2FBA36ADA050BD545210F48BC
:1022900003F0BBFB0020064A936A43F47F4393623A
:1022A000287070BDA36A9B04F4D545210848EFE768
:1022B00000ED00E0616F00007C6F0000B96E00006F
:1022C000926F0000B06F0000CA6F0000EA6F00005C
:1022D0002D6F000038B5214C4521214803F095FBB6
:1022E000A26A950103D545211E4803F08EFBA36A1F
:1022F000DC0103D545211C4803F087FB174DAC6A70
:1023000014F4801404D04521184803F07EFB022405
:10231000AB6A180303D54521154803F076FB0F4D32
:10232000AA6A510303D54521124803F06EFBAB6A3C
:102330009A0303D54521104803F067FB074DAB6AAC
:10234000DB0303D545210D4803F05FFBAB6A204654
:102350006FEA03436FEA1343AB6238BD00ED00E060
:1023600007700000247000003C7000005B700000EB
:102370008A700000AD700000D7700000F670000099
:102380002DE9F0434A4B0025D3F804908BB0C9F3F4
:10239000080885F31188BFF36F8F02F07F43B3F114
:1023A0007F4F07D102F00C03082B05D1452141488E
:1023B00003F02BFB2F4604E012074EBF0F460746E3
:1023C00001250022A8F1030614468DF80720092EE6
:1023D0005BD8DFE806F0054F53335A5A5A5A5A571A
:1023E0004521354803F011FB314B8DF80740DC6A7D
:1023F00014F0020405D04521304803F006FB002408
:102400001FE0DB6A5B001CD545212D4803F0FDFA77
:102410002C4B1B782BB101200DF10701FFF7AAFE11
:102420000EE0294B1B782BB101200DF10701FFF7BE
:10243000F7FE05E0254B1B889BB213B1FFF74AFF5F
:1024400004469DF8073093B92022394602A803F0CC
:102450007BFC099B35B3C3F3080222B96FEA53230F
:102460006FEA43230993204602A9FFF7D5FD0BB07D
:10247000BDE8F08300200DF10701CFE700200DF14A
:102480000701D4E745211248B7E7124919F4F87F4C
:10249000114A124808BF0A46A8F11003452103F06B
:1024A000B4FAACE723F4FF7323F00103DAE700BFCB
:1024B00000ED00E05471000084710000A071000084
:1024C000C671000028ED00E029ED00E02AED00E0F3
:1024D000EA710000267100003B71000013720000D9
:1024E000044B5A6942F010025A615A6942F4806200
:1024F0005A61704700ED00E0704700BFBFF34F8F97
:102500000549064BCA6802F4E0621343CB60BFF38F
:102510004F8F00BFFDE700BF00ED00E00400FA05AB
:1025200000231846054A1168C1F307218B4200D1E8
:102530007047936010610133F8E700BF90ED00E051
:1025400010B572B6002484F31388FFF7E9FF0E4A32
:10255000234611464FF0FF3403F120000133102BC6
:1025600042F82040F8D100234FF0FF3003F1600221
:102570000133102B41F82200F8D162B6BFF34F8F20
:10258000BFF36F8F10BD00BF00E100E000232021EA
:102590000348C2180133412B82F80013F9D1704768
:1025A00000E100E00121024B024A034800F00CB9AF
:1025B0000000042000450120BC66000010B50B6837
:1025C0000C7A23F01F0204F01F031A43CB6864093E
:1025D00023F01F03044943EA440343F001038860E6
:1025E000CA600B6110BD00BF90ED00E030B54B68D4
:1025F0000C6885B00A898D7A0094013B24F01F0491
:10260000234402F01F0242EA451223F01F030F2861
:1026100004468DF80820039309D90246452106484F
:1026200003F0F3F96FF01504204605B030BD69469C
:10263000FFF7C4FFF8E700BF2F7200002DE9F04F4D
:102640008946144606464FF00008524D85B0C845ED
:1026500023DA7768002F42D01F2F17D9FB0615D138
:10266000D6F800A01AF01F0F10D1504603F035FB2A
:10267000834607EB0A00013803F02FFB834510D097
:102680006FF0150B5A464521434802E0424645216A
:10269000424803F0BAF96FF01504204605B0BDE8D2
:1026A000F08F1BF1160FEDD0631E5B45EADBC5F81A
:1026B00008B0E968C5F808B02F6921F01F01D6E914
:1026C00000321A44994247F01F0702F1FF3A1CD129
:1026D000574508D131465FFA8BF0FFF787FF08F1C5
:1026E00001080C36B3E73146C5F808B0EB6822F0B4
:1026F0001F0203F01F031A43EA60E0B2FFF776FF00
:1027000010F1160FC7D0441CE9E7013B5745E0B272
:1027100023F01F03C5F808B006D12A69314602F03C
:102720001F0213432B61E9E7296901F01F010B43E5
:102730002B613146FFF75AFF10F1160FABD0C5F8E9
:1027400008B0EA689DF80830013F62F304038DF891
:1027500008302B699DF808205B0863F347128DF859
:102760000820D6E900321344009323F01F033B44B2
:10277000441CA3EB0A0AE0B22AF01F030F280393BC
:1027800003D902464521064883E76946FFF716FF4D
:10279000B9E700BF90ED00E0827200005A720000BD
:1027A0002F7200000522034B5A60BFF34F8FBFF317
:1027B0006F8F704790ED00E0BFF35F8F0022014BF9
:1027C0005A60704790ED00E010B5034C2278FFF797
:1027D00035FF207010BD00BFF255012038B50E4CFA
:1027E0002568102D14D8FFF7E7FF00200B4B0C4A8B
:1027F0001A63854205D10B4B1D70FFF7D3FF0020F4
:1028000038BD616801EB0011FFF7D8FE0130F0E739
:102810004FF0FF30F4E700BFC866000090ED00E025
:10282000AAFF4400F2550120014B1860704700BF19
:1028300014450120064A00F01F0002EB8000D0F88A
:10284000003223F4403343EA0141C0F800127047DC
:102850000025845008B5094B1A786AB901210D206A
:1028600019700521FFF784FB0D20FFF763FB4FF084
:102870000042034BC3F80423002008BDF355012098
:1028800000D00050F7B50E46416806F01F05097AE2
:10289000B2F5A03F076945EA41150AD15C4805F049
:1028A0001F01803150F82110C80707D56FF085004F
:1028B00093E0B2F5005FF96800F091800121F868BB
:1028C000B1400143F96001217869B140B2F5A03F00
:1028D0000CBF0843884378610020BA69B3F5C02F64
:1028E0000CBF0A438A43BA613A69B3F5802F0CBF23
:1028F000114322EA0101474A3961D2F80433DBB2BD
:1029000000F5A27152F82110C1F304218D426BD160
:1029100023FA00F1C90767D5830003F1A04303F54B
:102920005043D3F8101521F00101C3F8101501230D
:102930008340C2F80833C0B200F070FE2846002180
:10294000FFF778FFF868F04010F0010045D0786993
:10295000F04010F001044ED0BB690DF10700F340C8
:10296000DB0757BF3969032621FA06F606F0010690
:102970005CBFC6F10206F6B200F072FE264B98422A
:1029800036D100209DF807102D028B0003F1A043E3
:1029900003F55043D3F8102505F4F85522F44732D7
:1029A00022F44072C3F81025D3F8102515438A008D
:1029B00002F1A04202F5514245EA0646C3F810650D
:1029C00010601268D3F8102542F00102C3F81025F8
:1029D0000123104A8B40C2F8043303B0F0BD01203C
:1029E000B04021EA00016DE70130082888D1A5E751
:1029F0006FF01200F1E739692846F14001F001015A
:102A0000C1F10301C9B2FFF715FF2046E5E700BF9A
:102A10000025845000D000500000AD0B284B70B54D
:102A200046682848134083423BD00DD8062B15D06A
:102A300005D89BB1022B36D06FF0150030E0B3F50E
:102A4000801FF9D1012309E01F4883422DD0B3F53F
:102A5000A00F2CD0B3F5800FEED10223D0064CBFCF
:102A60000325C2F3401582F4807412F4007FC2F390
:102A70004020C4F3002406D012F4006F766818D00A
:102A800001228A40B26040EA4402002042EA032365
:102A900001F01F010D4A43EA8503803142F82130DD
:102AA00070BD0723DAE70423D8E70523D6E703231D
:102AB000D4E7520542BF01228A40F260E3E700BF3B
:102AC0000600F000060010000200400000258450BF
:102AD0002DE9F84F414E3568002D5AD0404B4FF04C
:102AE0000108D3E90520D968024321EA02093D4AD9
:102AF0004F464FF0000B924614691B695C4029EA6F
:102B0000040477BB37603368002301261F4636482C
:102B1000D0F8042306FA03F1114211D09A0002F111
:102B2000A04202F55142116851B103F5A27150F86B
:102B300021101760C1F3042106FA01F112680C4359
:102B40000133082BE4D134BB4DB101260027244DBD
:102B5000EC68D5E905210A4324EA020464BBBDE818
:102B6000F88F18EA070F0FD018EA090F0BF01F00B3
:102B700008BF00F180034FF0000108BF5AF823306E
:102B8000FFF758FE27EA08070BF1010B4FEA480848
:102B9000B7E72C46B8E7124B59680029D4D00E6825
:102BA000124F8A68224002D038464B689847002E60
:102BB000CAD031463668F4E726420CD0296907F0BE
:102BC0001F00F94001F00101C1F10301C9B2FFF793
:102BD00031FE24EA060401377600BFE77CD10050BD
:102BE000A44F01200025845000D00050044601204D
:102BF000024B0B6001231360704700BFC44F0120DC
:102C0000004870473867000010B503F0ABFA034C7A
:102C1000206003F0A4FA6060002010BDC44F0120C2
:102C2000F8B50E46144603F09AFA2146054630469A
:102C300003F026F93746F8B1B6FBF5F305FB13634D
:102C400023B9B4FBF5F305FB134040B123463246EC
:102C500045210C4802F0D9FE6FF015000BE0A542AB
:102C600009D803F07CFA0546384600F03BFD641BAA
:102C70002F44F9D12046F8BD23463246452102486B
:102C8000E8E700BFC0720000E472000037B50C46F0
:102C9000194620460193154603F0F2F8019B40B90E
:102CA00009482246452102F0B0FE6FF0150003B03E
:102CB00030BD33B11A462146284603F045F80020BE
:102CC000F5E71846F3E700BFE4720000F8B50E46DA
:102CD0001946304617461C4603F0D2F840B9234641
:102CE00032464521124802F090FE6FF01500F8BD03
:102CF00044EA060515F0030504D023463246452173
:102D00000C48F0E78CB12B19032BA6EB050006D875
:102D1000094AD2F80034DB07FBD50020E7E77B1B2C
:102D2000196800F0FDFC043DEDE72046DFE700BF39
:102D3000E47200000673000000900350F0B54B7978
:102D4000012B2AD0032B25D110268B79032B21D1DF
:102D5000CC792CB1012C1DD143685B689B0719D03D
:102D60000A7912B1022A15D10E220B684568B3F513
:102D7000164F2D6865D02DD8B3F5165F64D016D8E0
:102D8000B3F5966F62D00AD8B3F5967F61D0B3F5EC
:102D9000167F61D06FF0850052E00026D5E7B3F5CD
:102DA000166F5CD0B3F5965FF4D1374B3CE0B3F5CA
:102DB000E14F57D007D8B3F5615F55D0B3F5964FC3
:102DC000E8D1324B30E047F61227BB42E2D14FF454
:102DD000000329E0B3F5613F48D013D8B3F5963F1F
:102DE00047D009D84DF6C027BB4244D0B3F5614F58
:102DF000D0D14FF46B0317E0B3F5E13FCAD14FF0E8
:102E0000EB7311E0B3F5612F38D008D8204FBB42E7
:102E100037D0B3F5E12FBDD14FF0E86304E01D4F8B
:102E2000BB42B7D14FF08053C5F824350369344312
:102E30002243043303C9C5F86C2583E8030000204E
:102E4000F0BD4FF41D03EFE7134BEDE74FF49E2366
:102E5000EAE74FF4A033E7E74FF41C33E4E74FF41D
:102E60001D23E1E70D4BDFE70D4BDDE74FF06C7302
:102E7000DAE70C4BD8E74FF46503D5E74FF0706302
:102E8000D2E74FF08063CFE700B0130000A04E0000
:102E900090D0030040420F000050270000C0750092
:102EA00000F03A0000903A01F8B505460F46066971
:102EB00003F0C4F910B9294B1B78A3B94FF02003D4
:102EC000EFF3118483F31188BFF36F8F284603F06B
:102ED0005FF800BB84F31188BFF36F8FEEE784F3D4
:102EE0001188BFF36F8F6424284603F051F828B986
:102EF000012003F024F9013CF6D1F4E74FF0200360
:102F0000EFF3118483F31188BFF36F8F284603F02A
:102F10003FF80028E3D0012206F8107F69680B68AB
:102F2000C3F84465C3F848250022C3F82021D3F82C
:102F30002001C3F85821D3F858214A68D20641BF6E
:102F40000822C3F800254FF48002C3F804230122AD
:102F50009A6084F31188BFF36F8FF8BD045A012083
:102F600043682DE9F0411C68002306690F46C4F848
:102F700000350546306008680121444B00F01F020F
:102F8000914099600321803243F822107A68511CE5
:102F90001FBF4FF00C0C02F01F01803143F821C01D
:102FA000B968C4F80C05481C18BF0C20C4F81425D7
:102FB0001EBF01F01F02803243F82200F868421C55
:102FC0000CD04FF0010C00F01F020CFA02FCC3F809
:102FD00008C04FF0030C803243F822C0C4F8080543
:102FE000C4F81015296928460431FFF7A7FE80466A
:102FF00080B96B685B6819071CD506F1120000F0F8
:10300000E3FA234B984208D04521224802F0FDFC08
:103010006FF004084046BDE8F081B37C43F0004304
:10302000C4F8A031C4F88C300123B27C93401A4A12
:10303000C2F804350823C4F800357B6801330CD08E
:103040000023C4F81031D4F8103106F11103C4F88C
:1030500034350123C4F8383523606B6810365B685B
:103060001A075CBF4FF48072C4F80423DB0644BF28
:103070004FF48003C4F804330023C4F84465C4F853
:1030800048350123A360E360C4E700BF00258450F6
:103090000000AD0B337300000070015030B585B0F7
:1030A0006C460546084B0FCB84E80F000022012137
:1030B0000820FEF75DFF0820FEF73CFF214628466A
:1030C000FFF74EFF05B030BD9065000030B585B00C
:1030D0006C460546084B0FCB84E80F000022012107
:1030E0000920FEF745FF0920FEF724FF2146284668
:1030F000FFF736FF05B030BDA065000040EA0103D0
:10310000C3F30E0330B58BB940F21515094CC90B4A
:10311000C0F3C730994201D1002030BDC218D2B2ED
:1031200002F5C07244F822500133F3E76FF0150046
:10313000F3E700BF003000500348452108B502F016
:1031400064FC0020FFF7DAF975730000816808B5A8
:10315000044A1023103902F0A3FC003818BF0120E4
:1031600008BD00BF6467000030B50C46816887B0B9
:10317000102302AA1039054602F075FC002811DB65
:103180001022284602A902F031FF68B10323237000
:10319000A968012328460DF10702283902F063FCD3
:1031A00000280BDA01202AE01022164902A802F0BA
:1031B000BBFD002814BF02230123E8E79DF8073078
:1031C000284603F00F021B096270237101220DF1E2
:1031D000070102F00BFF10B96378042B03D9012318
:1031E000637000232371AA682846203AA11C02F0CC
:1031F00025FF0028D6D12846E11C02F078FF07B051
:1032000030BD00BF646700002DE9F04385B069461A
:10321000032002F070FF18B1FF2005B0BDE8F08375
:10322000072002A902F067FF0028F5D102469DF8A9
:1032300000509DF808609DF803709DF80B809DF884
:1032400002901E4C2946207802F0E4FE00B331467D
:10325000607802F0DFFED8B1A378042B01D0BB4226
:1032600016D1E378042B01D0434511D12379042BE7
:103270000CD16379022B16D1114A1248492102F070
:10328000C4FB6079831E022BC7D9C5E74B45F0D03C
:103290000132032A04F10604D4D10B48492102F07B
:1032A000B4FB0120B9E7032B05D0084A0849042BD9
:1032B00018BF0A46E1E7074ADFE700BFE2730000F4
:1032C0009E730000BA730000CD7300009773000076
:1032D000A8730000A3730000054B1868043B1B682B
:1032E000092B03D1431E58425841704700207047B4
:1032F0003401FF0008B54C4B1B68092B01BF4FF090
:1033000050230022C3F81421C3F81821FFF7E4FF6B
:1033100030B10123454A1360A2F63822C2F878354D
:10332000414B1B68092B07D1414B1B68012B1EBF6A
:103330000122404BC3F87825FFF7CEFF10B10E22D3
:103340003D4B1A60384B1B68092B04D100223B4BC4
:103350001A6001225A600022D30003F57F03D3F8DC
:103360000013013108D0D3F800130132D3F804332D
:10337000B2F5807F0B60EFD1314BDA69D1073BD5D5
:10338000304B1946D3F80024012AFBD1C3F8042599
:10339000D1F80034012BFBD1294BDA69D20708D5CB
:1033A000DA69284922F00102DA61D1F80024012A01
:1033B000FBD11A6A01320AD11A6A22F0FF0242F0E6
:1033C00020021A621F4AD2F80034012BFBD10022DE
:1033D0001C4BC3F80425D3F80024012AFBD1BFF30A
:1033E0004F8F1949194BCA6802F4E0621343CB604E
:1033F000BFF34F8F00BFFDE71B6A0133C0D0124BF4
:10340000D3F88C2042F44062C3F88C20D3F8882093
:1034100042F47002C3F88820BFF34F8FBFF36F8F61
:103420000B4B0C4A1A6008BD3001FF00384A0050AF
:103430003401FF0000400050E4AE03500C47005040
:103440000080FF000090035000ED00E00400FA054A
:10345000404501200090D003044B1A7922B9012283
:1034600018601A710248704702487047D44F012013
:103470000000AD0B0C00AD0B10B1012820D070473F
:103480004FF05022D2F81834D2F81814C90311D5CD
:1034900003F00303022B0DD1C2F8183500220D4BA7
:1034A0001A601B6802224FF05023C3F80423012244
:1034B0009A6070474FF050230122C3F81825EDE7BA
:1034C0000022054B1A601B684FF05023C3F8040319
:1034D00018607047045100500051005038B510B1C9
:1034E000012818D038BD4FF050230222012142F2AA
:1034F00010751C46C3F80823154A10601268154A57
:103500001160D4F81834DB03ECD5012002F017FE6B
:10351000013DF6D1E6E74FF05024002242F210754B
:103520000D4BC4F808031A601B680C4B1860D4F8E4
:103530000C34D4F80C2403F00103D203D2D5002BB1
:10354000D0D0012002F0FBFD013DF0D1CAE700BF61
:10355000045100500C5000500051005004500050D5
:10356000164B10B51A6852B1002018601B68012272
:103570004FF05023C3F80823114B1B689847114B99
:103580001A688AB100221A601B684FF05023D3F8E2
:103590001824D3F8181402F00302012A4FF0020194
:1035A00003D1C3F818159A6010BDC3F80813044B73
:1035B0000120BDE810401B68184700BF00510050B3
:1035C000D44F012004510050F0B54FF02003EFF329
:1035D000118783F31188BFF36F8F0D4A1668F1438B
:1035E00089B291B10025ECB221FA04F3DB0705F1B1
:1035F0000105F8D50123A340334304700548136047
:1036000087F31188BFF36F8FF0BD0348F8E700BF61
:10361000DC4F01200000AD0B0200AD0B012303FACB
:1036200000F010F0FF0F12D04FF02003EFF31181E4
:1036300083F31188BFF36F8F064AD36C23EA00002F
:10364000D06481F31188BFF36F8F0348704703483C
:10365000704700BFE04F01200000AD0B0400AD0B30
:103660002DE9F041FF22002401260546DFF858E04D
:103670001448DFF85880E3B24FF02001EFF3118CCB
:1036800081F31188BFF36F8F22FA03F1C9070AD5BE
:10369000DEF84C1006FA03F7394201BF40463943C1
:1036A000CEF84C102B708CF31188BFF36F8F404510
:1036B00005D006FA03F39A4304F10104DBD1BDE817
:1036C000F08100BF0200AD0BE04F01200000AD0B08
:1036D0000022034BC3F88425C3F80425704700BFBC
:1036E0000090035008B5C0F30B0383B90222094BC5
:1036F000C3F88425C3F804254FF0FF320260D3F8E5
:103700000024D207FBD5FFF7E3FF034808BD0348B9
:10371000FCE700BF009003500000AD0B0A00AD0BAA
:103720000122074BC3F88425C3F80425D3F80824E5
:10373000D207FBD50160BFF35F8FFFF7C9BF00BFA2
:1037400000900350032310B5134C144A23616361A6
:10375000134BA261E3614FF4806323620023A362F1
:103760006362E36222660F4A0F4962661022E01D1F
:10377000A2662367E366636702F0B9FABFF35F8F5F
:103780000A49204602F0B3FABFF35F8F2023A371EA
:10379000BFF35F8F10BD00BF30500120F4730000F5
:1037A00004560120F4550120FD730000017400004F
:1037B000F8B51823174C00FB033503FB00402544E4
:1037C000C46A0F46012C16460FD0022C1AD0F4B949
:1037D000284602F0CAFC864205D8324639462846B9
:1037E00002F0D1FC34462046F8BD284602F0BDFC6C
:1037F0008642344628BF044639462246284602F00F
:10380000C2FCF0E72846BDE8F84002F0DABC00242C
:10381000E9E700BF305001200E4B70B553F820404F
:10382000013053F82060A64200D870BDD4E90035BD
:103830002846984765B1EB6830B10028B8BF4042D0
:10384000FF28A8BFFF2018705A7842F001025A7072
:103850000834E8E77467000070B5054610B9002425
:10386000204670BD0378002BF9D00F4A0F4C164646
:10387000944208D10D4CB442F1D0204602F0D5FC60
:1038800050B91834F7E7204602F0CFFC10B1236896
:10389000AB42E5D01834EBE72846216802F038FA4D
:1038A0000028EED1DCE700BF34460120A44501200A
:1038B00073B504460D464FF02003EFF3118683F3F2
:1038C0001188BFF36F8F0022042896BF114B124B53
:1038D00053F82030009245210246104802F095F836
:1038E0003DB1EB69C3F308031BB145210C4802F05D
:1038F0008CF800220B4B45210B4802F086F8294634
:103900002046FFF719FC86F31188BFF36F8F02B0D2
:1039100070BD00BF886700000874000016740000C6
:103920004374000069740000717400000248034A87
:103930000021121A02F033BA38460120085A012039
:10394000012208B5084B02201A70FFF765FF00F04E
:103950005FF80320FFF760FFFCF782FD034A137B4B
:1039600023F00103137308BD045A012038460120D7
:1039700008B5174B03F5006282F3088883F30A88C1
:103980000025E023134C84F82230E5772576657610
:10399000A576636A43F4E0236362FEF7A1FDFEF7B8
:1039A0001DFB4FF0FF33A362E362FEF717FFFEF744
:1039B000F9FD02F039FC2846FFF72EFF0120FFF742
:1039C0002BFF2B462A4629460348FEF7E7FA00BF9D
:1039D0000882012000ED00E04139000008B50648EA
:1039E000064A0749121A02F0AFF9BDE80840054A35
:1039F0000549064802F0A8B90045012034460120D7
:103A00002C75000000000000147500000045012026
:103A1000024A0349034801F03CBF00BF687400003C
:103A2000DB740000EB74000010B50A4C23681BB176
:103A300001230020236010BD00F048F80028F7D0D3
:103A40000138062803D8044B53F8200010BD034862
:103A500010BD00BFD85001209C670000FE8FFFFF03
:103A6000BFF34F8F0549064BCA6802F4E062134367
:103A7000CB60BFF34F8F00BFFDE700BF00ED00E05C
:103A80000400FA054FF0FE33002130B4064A074D1A
:103A9000074C2B6013602360064A074CEB60636899
:103AA000C2F8001530BC1847041484500014845028
:103AB000081484500000845044450120024BD0E992
:103AC0000012C3E9001270474445012010B500F010
:103AD00033F820B1032400F067F8204610BD00F051
:103AE00035F890B900F0B0F890B90F4B1B681B0E79
:103AF000F02B08D10D4A0E4B12689A420AD00724C7
:103B000000F01CF8E7E70624FAE70424204610BD7D
:103B10000024F5E7012000F097F804460028F7D1CB
:103B2000044B1860D9E700BF28198450241A845028
:103B30000000E0200C1A84500020704700207047DD
:103B4000014B1860704700BF041A845010B511482B
:103B500000F048F800B110BD0F4800F043F800280D
:103B6000F9D10E4C204600F03DF80028F3D10C4B63
:103B70000C481C6000F036F801460028EBD100F03C
:103B80002DF8044608B1204610BD00F03FF820464D
:103B9000FAE700BF584501204C450120544501205B
:103BA0005C4501205045012008B5084800F024F884
:103BB000074800F021F8074800F01EF8064800F01A
:103BC0001BF8BDE8084000F00BB800BF58450120C5
:103BD0004C450120544501205045012000207047EC
:103BE000704700BF08B5034B02681B681068984710
:103BF000002008BD6845012008B5034B02685B68DA
:103C000010689847002008BD6845012070B5094C30
:103C1000094D2069AB68984718B1084B08485B68A4
:103C200098470021074AEB6811602069BDE87040A1
:103C3000184700BF78450120684501204445012010
:103C4000B8670000DC50012070B51A4D1A4E0446CA
:103C5000B26828699047F0B95CB1184C2368ABB1E1
:103C6000012B1AD0013B23602869F3689847002094
:103C700070BD124C216839B90120114B114AC3F8AB
:103C800000051368002BFCD101312160F36828691D
:103C90009847002070BD0C4870BD0A4A1368002B7D
:103CA000FCD1074A6FF07E40C2F80035FFF748FFAD
:103CB0002368D7E77845012068450120DC500120C2
:103CC0000000845010198450E98FFFFF48B1436809
:103CD0002BB1BFF35F8F0023036018467047024883
:103CE00070476FF4E0407047EA8FFFFF10B504465D
:103CF00028B1636813B100232360636010BD024BD9
:103D000002485B689847F4E744450120D867000003
:103D100010B5044630B100226368226043F001030D
:103D2000636010BD0148FFF7ADFEF4E700680000D6
:103D300080B1436863B10122D0E8EF3FC0E8E12FD2
:103D40000029F9D1012BF7D0BFF35F8F0020704716
:103D5000024870476FF4E040704700BFEA8FFFFFF2
:103D600030B10268034B04489A4208BF00207047F4
:103D700002487047DD55AABB8208F0007108F000C8
:103D800038B50D460446B0B1A0220021043002F03F
:103D900079FA95B10822294604F1640002F078FA14
:103DA000082205F1200104F1840002F071FA0020DC
:103DB000034B236038BD0348FCE70348FAE700BF24
:103DC000DD55AABB7108F0008308F0002DE9F74328
:103DD00005460E4699461146FFF7C2FF04460028E5
:103DE00040F08480002E00F08580002900F084805F
:103DF000B9F1200F40F0828005F14404082205F15A
:103E00000408204602F044FA05F12407082231464E
:103E1000404602F03DFA06F120010822384602F041
:103E200037FA02A941F8049D4FF4807002F024FA99
:103E3000002865D14FF48073324A012113609360EA
:103E40000823314A00F034FB0121052308462F4A9C
:103E500000F02EFB0823424601211C2000F028FB25
:103E600008233A460121032000F022FB22460823C2
:103E70000121022000F01CFB0823254A01211A2001
:103E800000F016FB0523234A01211B2000F010FB44
:103E90000823214A0121142000F00AFB08231F4AAD
:103EA0000121152000F004FB082305F16402012123
:103EB000162000F0FDFA082305F1840201211720E5
:103EC00000F0F6FA0823164A01210B2000F0F0FA60
:103ED00000F04AFB0446019800F0D8FA114B002C80
:103EE00018BF1C46A421284602F0CEF9204603B094
:103EF000BDE8F0830C4CF9E70C4CF7E70C4CF5E708
:103F0000084CEFE79010845064680000DC68000003
:103F100024680000C868000088680000A8680000E5
:103F2000446800008408F0007608F0008008F00083
:103F30008108F000C2690C4B1A60826943F8042CB6
:103F4000426943F8082C026943F80C2CC26843F814
:103F5000102C826843F8142C426843F8182C02682D
:103F600043F81C2C704700BF5C1684500C4B1B6838
:103F7000C3610C4B1B6883610B4B1B6843610B4B8C
:103F80001B6803610A4B1B68C3600A4B1B68836094
:103F9000094B1B684360094B1B680360704700BFF7
:103FA0005C16845058168450541684505016845011
:103FB0004C16845048168450441684504016845041
:103FC00030B10268034B04489A4208BF0020704792
:103FD00002487047DD55AABB0202F0000002F00063
:103FE00038B5044668B1051D7021284602F04CF929
:103FF00028462022044902F043F90020034B2360A5
:1040000038BD0348FCE700BFF0680000DD55AABBDF
:104010000002F0002DE9F04385B015466F46274BAE
:1040200004460E460FCB87E80F002DB94FF000096C
:10403000484605B0BDE8F0832046FFF7C1FF814642
:104040000028F5D1231D0193636AA3BB236F8BB1B5
:10405000C3F14008A84528BFA84604F13000314606
:104060001844424602F00CF9236F46444344236748
:10407000A5EB0805226F402A06D104F1300138462D
:1040800000F0B4FB0023236705F03F0835F03F053F
:1040900005D031462A46384600F0A8FB2E44B8F138
:1040A000000FC3D04246314604F1300002F0E8F878
:1040B000C4F87080BCE7DFF80890B9E7B06500008D
:1040C0000C02F0002DE9FF4104466F46134B0E46EB
:1040D0000FCB87E80F002046FFF772FF8046B0B98C
:1040E000CEB1636A251D01953BB90123226F63623E
:1040F00004F13001384600F079FB2B46043E2434AD
:1041000053F8042B12BAA34246F8042FF8D14046C4
:1041100004B0BDE8F081DFF80880F8E7B065000082
:104120000502F000084B1B681B0EF02B08D1074B53
:104130001A68074B9A4205D10020064B1860704759
:10414000052070470620704728198450241A84508F
:104150000000E0200C1A8450002230B5134640F6CF
:10416000FC754900023802F1A15404F582349042F2
:104170004FEA840402F10102CABF236025605B1884
:104180001E2AF0D1034A13600B445360024B034ACA
:104190001A6030BD781084508410845020F80F00CD
:1041A0001E4B30B51A4685B0196800910099CC07AE
:1041B000FAD500F1A15000F5823080000168136843
:1041C0000193019BD807FAD5154B164C186820238C
:1041D0001F3090FBF3F0144D0138002810DA002353
:1041E0000130400153B14FF00042A0F120011342D1
:1041F00004D1013888424FEA5202F8D105B030BDEF
:1042000013680393039BDB07FAD5431823602B68DD
:104210000293029B002BE3D10138DEE7B4108450F7
:10422000AC108450E4108450DC108450F0B51D684C
:1042300085B001F01F040DB91F2C28D1174D2E4653
:104240002F680197019FFF07FAD500F1A15000F5F3
:1042500082308000006835680395039DED07FAD52C
:104260001F2C00EB611018BFC9430D4D18BF01F0A2
:104270001F0128600B480068029002981CBF00FADA
:1042800001F111604FF0000108BF10601960106863
:104290004300C00F136005B0F0BD00BFB4108450E0
:1042A000E4108450DC1084500C4B890118603F30BE
:1042B00020F03F004030586099600948D96019618A
:1042C000596199611C3382B0196002680192019AA8
:1042D000D207FAD5196002B0704700BF9010845021
:1042E000B410845038B5A0F12003B3F5426F0546F1
:1042F0002CD88F2826D800F1470300F16604DB068E
:104300004FEA541400D0013464013F34A40901344D
:1043100011B1A1421AD30C464FF48050E300B0FB18
:10432000F3F0202828BF202002B110600122084BA2
:1043300021461A60FFF710FF28462146FFF7B4FF19
:10434000002038BD00F11F046409DDE70148F8E7EB
:104350001C1884502221F000464BF0B51D4689B050
:104360001C680194019CE407FAD5434B00241344D4
:104370009B001A680B181E2B88BFC0F11E011F324C
:104380000B1852095343B3F5806F84BF4FF480611B
:10439000B1FBF2F1274688BF091ADFF8E4E000F12B
:1043A000A150DFF8E0C000F58230A14233DC2B6879
:1043B0000493049BDB07FAD5304B1B6829680591F1
:1043C0000599CF07FAD52E4C2E49236000231E46AF
:1043D000934203F1010040D11946002620F001026A
:1043E00028488A423CD8296806910699CE07FAD512
:1043F00025490968286807900798C007FAD5216001
:1044000000210C461F488B422DD100201D499A42A5
:104410002CD809B0F0BD2B680293029BDB07FAD5BC
:1044200003199B001B682E680396039EF607FAD5B6
:10443000CEF800300023934203F1010306D1164663
:1044400023F00103B34204D80134AEE7CCF8007086
:10445000F1E7CCF800700136F4E70E600346B7E7E9
:1044600006600131BDE704600131CCE7086001332B
:10447000CDE700BFB4108450240421147C10845074
:10448000D4108450D81084507810845008B540B1AE
:10449000202801464FF0070228BF20210020FFF707
:1044A0005BFF0022014B1A6008BD00BF1C1884503E
:1044B000F0B5294D85B02C462E680096009EF60773
:1044C000FAD500F1A15000F582308000056820681F
:1044D00001900198C707FAD52048214F056002EBEB
:1044E0008306B24229D100275A1C1D4E22F0010238
:1044F0009A4227D823680293029BDE07FAD5194B0C
:104500000B449B001B681F335B099A4213D221683E
:1045100003910399C907FAD500211544056008469F
:104520009B1A0F4A8B4210D800205A1C0C4922F0CB
:1045300001029A420CD805B0F0BD52F804CBC7F87E
:1045400000C0CEE737600133D2E710600131E9E700
:1045500008600133EDE700BFB4108450D4108450DC
:10456000D8108450240421142DE9F041814BA0B0CF
:104570001D68986820331E461A680192019AD70771
:10458000FAD57D4B7D4A1A6032680292029AD407AE
:10459000FAD57B4A1A607B4A144611680391039945
:1045A000C907FAD5784A1168C1F3402137680497E2
:1045B000049FFF07FAD5754F1F6027680597059F71
:1045C000FF07FAD51768002900F0CF80B90540F140
:1045D000CC80316806910699CF07FAD56C491960ED
:1045E000216807910799C907FAD51168C1F34021DD
:1045F00037680897089FFF07FAD5664F1F6027683E
:104600000997099FFF07FAD51268002900F0AF80CB
:10461000910540F1AC8032680A920A9AD207FAD525
:10462000564A1A6032680B920B9AD707FAD55A4A43
:104630001A6031680C910C99CC07FAD5574919606A
:1046400031680D910D99C907FAD55549196031683E
:104650000E910E99CF07FAD55249196031680F9122
:104660000F99CC07FAD550491960504B1E4619686E
:1046700010911099C907FAD53F4C4D4B2360336810
:104680001193119BDB07FAD54A4B236033681293D1
:10469000129BDF07FAD5484B23603A4B98461968BE
:1046A00013911399C907FAD5324F386033681493C0
:1046B000149BDB07FAD5226033681593159BD80746
:1046C000FAD53E4B236033681693169BD907FAD56B
:1046D0003B4B236033681793179BDA07FAD5394BA6
:1046E000236033681893189BDB07FAD5364B236099
:1046F00033681993199BD807FAD5344B2360336874
:104700001A931A9BD907FAD5314B236033681B9350
:104710001B9BDA07FAD52F4B236000F01DFC08BB6A
:10472000D8F800301C931C9BDB07F9D53D6033683B
:104730001D931D9BD907FAD5274B236033681E9321
:104740001E9BDA07FAD5254B2360D8F800301F935B
:104750001F9BDB07F9D50C4B1B6813F4805F204BC4
:1047600008BF184620B0BDE8F0811E48FAE71E4891
:10477000F8E700BF90108450801084500010025160
:10478000C01F7229B410845088108450C0CF0129F2
:10479000C01F0E29C03F002940010249003184A8F2
:1047A00000001649400108A180440888B0108450D8
:1047B000C044708880077A41C0077E4100006A4982
:1047C0008006164940006E49000200210082202127
:1047D000408220218082242140A161A100C8615132
:1047E0000308F1000108F1000208F100324B2DE945
:1047F000F74F80469246994644681A68002AFCD1D1
:104800002E4B9B461A68002AFCD14FF0FF300191D5
:1048100000F094FC802000F097FC01230720284A38
:10482000284DA2F59E722B60C2F83C011360636AAA
:10483000254F264E3B60A36A20463360D8F80030EF
:1048400042F8043CD8F8083098470199D9F800306C
:10485000002BFBD1BAF1000F20D104221C4B1A60AF
:10486000D9F80030002BFBD1DBF800A0BAF1000F23
:10487000FAD1D8F80C30204698473B686362336819
:10488000A362144BC3F800A0C3F844A1D9F80030C8
:10489000002BFBD12B6003B0BDE8F08F236A4020D2
:1048A000012B04BF0B4A13600B4B1960C3F804A023
:1048B00000F050FCD4E700BF10198450201C845035
:1048C0000019845018188450CC178450D017845085
:1048D000C817845084168450281C8450544B10B53B
:1048E000194698B01A680192019AD207FAD5514B2D
:1048F000514A1A600A680292029AD407FAD54F4ABE
:104900001A600A680392039AD007FAD54C481860D7
:104910000A680492049AD207FAD54A4A1A600A68C9
:104920000592059AD407FAD5474A1A600A68069292
:10493000069AD207FAD5454A1A600A680792079A7A
:10494000D407FAD5424A1A600A680892089AD20730
:10495000FAD5404A1A600A680992099AD407FAD52A
:104960003D4A1A600A680A920A9AD207FAD53B4A67
:104970001A600A680B920B9AD407FAD5384A1A6063
:104980000A680C920C9AD207FAD5364A1A600A685D
:104990000D920D9AD407FAD5334A1A600A680E921E
:1049A0000E9AD207FAD5314A1A600A680F920F9A06
:1049B000D407FAD52E4A1A600A681092109AD207C4
:1049C000FAD52C4A1A601A4B19461C681194119C8E
:1049D000E407FAD5174B1860086812901298C407BC
:1049E000FAD51A600A681392139AD007FAD5124AB8
:1049F0001A600A681492149AD207FAD51E4A1A60ED
:104A00000A681592159AD407FAD51C4A1A600A68E2
:104A10001692169AD007FAD5194A1A600A681792A0
:104A2000179AD207FAD5174A1A6018B010BD00BFFE
:104A3000B0108450801084500093652100043190A0
:104A4000409665900083612100C3302100C36490CB
:104A50000081619000461021008111210041442114
:104A600000C320290C4610C80086312100C36021F4
:104A700040C1282940966521001331904096252990
:104A8000594614C840043249494B10B5194694B0F0
:104A90001A680092009AD207FAD5464B464A1A6025
:104AA0000A680192019AD407FAD5444A1A600A6842
:104AB0000292029AD007FAD5414818600A68039218
:104AC000039AD207FAD53F4A1A600A680492049AF8
:104AD000D407FAD53C4A1A600A680592059AD207AB
:104AE000FAD53A4A1A600A680692069AD407FAD5A5
:104AF000374A1A600A680792079AD207FAD5354AE8
:104B00001A600A680892089AD407FAD5324A1A60DD
:104B10000A680992099AD207FAD5304A1A600A68D7
:104B20000A920A9AD407FAD52D4A1A600A680B929B
:104B30000B9AD207FAD52B4A1A600A680C920C9A83
:104B4000D407FAD5284A1A600A680D920D9AD2073E
:104B5000FAD5264A1A600A680E920E9AD407FAD538
:104B6000234A1A600A680F920F9AD207FAD5214A8F
:104B70001A600F4B19461C681094109CE407FAD574
:104B80000C4B1860086811901198C407FAD51A6088
:104B90000A681292129AD007FAD5174A1A600A6860
:104BA0001392139AD207FAD5144A1A6014B010BDA2
:104BB000B0108450801084508090652100040990CA
:104BC000409665908080612180200821802064903B
:104BD0000081619000461021008111210041442193
:104BE00080202029024610C80086092180206021EB
:104BF000402128294096652140962529594614C808
:104C0000504B10B51C4696B01A680192019AD20713
:104C1000FAD54D4B4D4A1A6022680292029AD20789
:104C2000FAD54B4A1A604B4A42EA80402268039206
:104C3000039AD207FAD5186022680492049AD00722
:104C4000FAD5454A1A60A2F5800242EA81412268FB
:104C50000592059AD207FAD5196022680692069A3B
:104C6000D007FAD53D4A1A6022680792079AD10701
:104C7000FAD53B4A1A6022680892089AD207FAD5F8
:104C8000384A1A6022680992099AD007FAD5364A3A
:104C90001A6022680A920A9AD107FAD5334A1A6032
:104CA00022680B920B9AD207FAD5314A1A60226811
:104CB0000C920C9AD007FAD52E4A1A6022680D92EF
:104CC0000D9AD107FAD52C4A1A6022680E920E9AD4
:104CD000D207FAD5294A1A6022680F920F9AD00794
:104CE000FAD5274A1A60216810911099C907FAD598
:104CF0001A60144B1A46196811911199C807FAD510
:104D0000114B20491960116812911299C907FAD5FF
:104D10001D491960116813911399CC07FAD50B49F5
:104D20001960116814911499C807FAD517491960C8
:104D3000116815911599C907FAD5154A1A6016B068
:104D400010BD00BFB01084508010845040044190CA
:104D500000862929D81001C8401441904014212907
:104D6000401465210034409000310C90C0400C90FC
:104D7000C030202940960D9000416090031645C830
:104D80000086112100416021594644C840144590D5
:104D900040142D90264870B5054688B004680094EC
:104DA000009CE607FAD5234C23480460234C44EAD0
:104DB00083432C680194019CE407FAD503609301B6
:104DC00043EA824242F0104444F4C0442B68029308
:104DD000029BDE07FAD504602B680393039BDB0775
:104DE000FAD5174B03608B0143EA814141F0104330
:104DF00043F4C0432E680496049EF607FAD5036078
:104E00002B680593059BDE07FAD5046041F05841F5
:104E10002B680693069BDC07FAD5016042F05842E6
:104E20002B680793079BDB07FAD5026008B070BDBB
:104E3000B0108450C02102298010845080710098E5
:104E400080611890354B8EB019461A680092009A0E
:104E5000D207FAD5324B334A1A600A680192019A96
:104E6000D007FAD5304A1A600A680292029AD2072D
:104E7000FAD52E4A1A600A680392039AD007FAD527
:104E80002B4A1A600A680492049AD207FAD5294A72
:104E90001A600A680592059AD007FAD5264A1A6060
:104EA0000A680692069AD207FAD5244A1A600A6856
:104EB0000792079AD007FAD5214A1A600A68089221
:104EC000089AD207FAD51F4A1A600A680992099A05
:104ED000D007FAD51C4A1A600A680A920A9AD207C1
:104EE000FAD51A4A1A6008680B900B98C007FAD5D1
:104EF0001A600A680C920C9AD007FAD5144A1A6004
:104F00000A680D920D9AD207FAD5124A0E211A603C
:104F100000200D230F220EB0FFF73CBFB0108450CD
:104F20008010845080430129406339218070012919
:104F30008020542100D13490C0403490C0302029CA
:104F4000C0530D9000413890832308C880E310219E
:104F500000413821CF4308C801232DE9F04192B028
:104F6000CDE90333624B1D461A680592059AD207B4
:104F7000FAD5604B604C2360604B19461A68069264
:104F8000069AD707FAD55E4B1A68D60400F1A880B6
:104F90002A680792079AD007FAD55A4A22600A6807
:104FA0000892089AD207FAD51E68C6F30036002E7A
:104FB00040F098801220FFF7F3F807461320FFF720
:104FC000EFF887428CBF12201320FFF7E9F8471E45
:104FD000FFF738FF03AB01AA39461220FFF726F985
:104FE00004AB804602AA39461320FFF71FF900EBF5
:104FF0004800022832D003283ED0012874D12B6803
:105000000993099BDB07FAD53F4B23602B680A9372
:105010000A9BD807FAD53D4B23602B680F930F9B53
:10502000D907FAD53A4B23602B681093109BDA0707
:10503000FAD5384B23602B681193119BDB07FAD507
:10504000354B2360013F25D510231922182100205C
:10505000FFF7A0FE304612B0BDE8F0812B680B933D
:105060000B9BD907FAD52D4B23602B680C930C9B17
:10507000DA07FAD52A4BCFE72B680D930D9BDB0798
:10508000FAD5284B23602B680E930E9BD807FAD5D0
:10509000254BC1E703AB01AA39461220FFF7C6F83A
:1050A00004AB044602AA39461320FFF7BFF810EB01
:1050B000440402D1FFF712FCC4E7FFF7E5FC022C21
:1050C00008D0032C09D0012C10D117211620FFF78E
:1050D00097FDB7E715211420F9E70F210E20F6E719
:1050E000124EB7E7124EB5E7124EB3E7124EB1E7D4
:1050F000B010845000084A5180108450B41084507D
:105100008810845000084E5100065A4940065E49F6
:10511000000442410014424940042E49000652490D
:105120004006564900063A4940063E490608F10045
:105130000708F1000408F1000508F100014B1860B0
:10514000704700BF081A8450014B1860704700BFB9
:10515000041A8450034A13681842FCD0024A1060B3
:1051600018467047001A8450081A845029B1012942
:1051700014BF6FF015000720704703207047704779
:105180002DE9F7430E4617469946044628B94FF0D5
:10519000FF38404603B0BDE8F0830029F7D0002A6D
:1051A000F5D0CB680D8938461D44042329460DEB04
:1051B000030200F058FC80460028E8D146F60812A9
:1051C000BDF804107389914223D1BDF806109942AD
:1051D000DDD1042338460DEB0302294400F043FCE3
:1051E0000028D4D146F60713BDF804209A42CED148
:1051F0009DF82830BDF80620A3727389C4E90067C2
:105200002B44E36004351344A4F8089063612561DE
:10521000BFE7002BE6D0BAE72DE9F7430F469046EB
:105220001E46044620B94FF0FF3003B0BDE8F083BE
:105230000368002BF7D04368002BF4D04FF6FF79BA
:10524000D4E904239A4216D223685B8923B1E36828
:10525000934204BF043323610423216960680DEB8A
:10526000030200F000FC0028DDD1A37A256923B1F8
:10527000E368AB4201D80120D7E72189BDF80630A9
:10528000494503F1040203D0BDF804C08C450BD19D
:1052900016B1BDF80410318004353D60A8F8003027
:1052A000236913442361C0E715442561C8E773B53A
:1052B0000C46064611460223204601AA00F03CFA9D
:1052C0000546E8B9019A1F2A0ED9A2F120013046FD
:1052D00020222368194400F037FD2368019A134403
:1052E0002360284602B070BD0146C2F1200230465C
:1052F00000F055FD019A2168C2F120003044EAE730
:105300006FF00205EDE700F00FBD4FF4C073584396
:10531000303070470B7803F0FB03032B14BF4FF0C2
:10532000FF304FF4C070704710B5044600F01AFC0F
:105330004FF4C072A368303B02FB103010BD81688F
:105340000122203900F0C4BE13B50446019100F0DB
:105350005EFE0423A0F108010DEB0302204600F0DD
:105360008AFE02B010BDF7B5054600200C46174670
:10537000FFF7FCFE6946C0B2FCF79AFB30B101258D
:10538000009800F06FFB284603B0F0BD2C2101FB14
:1053900004542189E3680098CE18042331460DEBAC
:1053A000030200F060FB05460028E8D146F608132A
:1053B000BDF8042064899A421AD1BDF806309C4297
:1053C00001D00325DCE7042300980DEB0302A119AB
:1053D00000F049FB0028D2D146F60713BDF804209F
:1053E0009A42EED1BDF80610214431443960C7E736
:1053F000002CF1D0E5E773B5134601920E46024644
:1054000000210546FBF7C0FC044650B9012128469F
:10541000019B05F12C02FBF7B7FC10B1002E18BF61
:105420000446204602B070BD37B580250446426A66
:1054300001A903200195FCF74FFB48B9019B072008
:10544000226DA36201A90195FCF746FB054608B150
:10545000012505E0019B206A636500F083FBE065A0
:10546000284603B030BD0123036003F101234360EC
:105470000023C0E9023370474379012B07D1036849
:10548000012B04D10079431E584258417047002037
:10549000704770B586B006460D46032003A9FCF799
:1054A00007FB30BB0398FFF73FFFF16D044628462A
:1054B00000F0E4F80444039800F054FB01900398D2
:1054C00000F059FB0822014604A800F068FC2A7984
:1054D00021468DF81020019B039804AA00F0E0FA01
:1054E000041E18BF0124039800F0BCFA204606B041
:1054F00070BD0124F7E700F005BB2DE9F8430E4627
:10550000002107460846FFF731FE0446012100202E
:10551000FFF72CFE33789C4221D0984221D1012400
:105520002C2303FB0474F86DA56AFFF7EEFE4FF021
:1055300000080746013D636A304603EBC50253F895
:105540003510D2F804901B684A46C91AC844FFF7C0
:10555000D2FFB84505F1FF35EDD3BDE8F88300244F
:10556000DEE70120F9E737B515460C460720694606
:1055700000F0C1FDE979012903D00022204600F0A6
:10558000CEFD9DF80330012B02D1204600F0AAFD8C
:10559000A9682046FFF7D8FE2046FDF7D7FD00207A
:1055A00003B030BD73B50D460646FBF7D5FC044687
:1055B000E86038B102282FD1032001A9FCF778FA5E
:1055C00018B10124204602B070BD2A463146019828
:1055D000FBF728FC0446D8B9019800F018FD012318
:1055E00001460DF10302019800F03DFA044600283F
:1055F000E7D1012201980DF1030100F019FD10B16E
:1056000001238DF803309DF8033003F00F03EB7195
:10561000019800F027FAD5E70724D3E713B5032054
:1056200001A9FCF745FA48B90198FFF788FE04463E
:10563000019800F017FA204602B010BD0124FAE7E5
:105640001FB5032001A9FCF733FAA8B9019802A9F4
:10565000FDF78AFD044668B99DF80B30032B03D192
:10566000019800F03FFD0446019800F0FBF9204648
:1056700004B010BD0124F7E70124F8E730B5437901
:105680000468012B0ABF01220222002501FB02F25D
:1056900004F1FF3402FB04F2037918BFCD01013B92
:1056A00001FB0321481930BD036870B5CD1A002DE8
:1056B0000DDD93F900601C78002E0BDB5C1C046090
:1056C0001B7813600368C91A13688B4232D96FF0D4
:1056D0005F0070BD04F07F04013C032C27D8DFE895
:1056E00004F00209121E012DF1D05C78023314601F
:1056F0000360E7E7022DEADDB3F80140033364BA43
:10570000A4B21460F4E7032DE1DD9C785D782402F7
:1057100044EA0544DD7804332C431460E8E7042DA3
:10572000D5DDD3F80140053324BA1460E0E76FF00B
:105730006300CEE70020CCE770B404680E1B002E97
:1057400007DD26789E4208D10134046070BCFFF763
:10575000ABBF6FF05F0070BC70476FF06100FAE79D
:1057600038B5032304461546FFF7E6FF58B913681A
:105770005A1E012B2A6004D923685A1C22601B7808
:105780000BB16FF0670038BD2DE9F74390461F4617
:1057900001AA302305468946FFF7CEFF0446F8B933
:1057A0002E68A9EB0609B9F1000F35DD42460199D3
:1057B00033780E4442F8043B314606232846FFF76F
:1057C000BBFF044660B92A68D8F80410C8F808205E
:1057D0005318B3422B6007D10C213846FBF776FDF6
:1057E000204603B0BDE8F083515C3A46013342F8ED
:1057F000041B284631462B60FFF756FF044600285D
:10580000EED12B687A68BB601344B3420CBF0446E8
:105810006FF065042B60E3E76FF05F04E0E7F8B535
:10582000B1F1005F0546144600AF10D26E46D31D9D
:1058300023F00703ADEB030D684600F085FA6946D7
:1058400022462846FEF7E6FBB546BD46F8BDFEF704
:10585000E1FBFAE760B1436803F00303012B03D0D7
:10586000032B05D103681BB10023836018467047E2
:105870006FF01500704700224368816003F0030356
:10588000032B14BF1346036842601846704700207C
:1058900070470FB407B504A951F8040B0191FBF749
:1058A00089FD03B05DF804EB04B07047038B13F07F
:1058B000070305D10368002B0CBF002003207047AD
:1058C000022B05D1438B002B14BF0020042070470E
:1058D000012B05D10368002B0CBF00200520704769
:1058E0000020704773B50D4606461946281D0192E3
:1058F0000093FFF7C0FF044640B1DDE900322946BE
:105900003046A44602B0BDE87040604702B070BDAA
:1059100010B44FF02004EFF3118284F31188BFF329
:105920006F8F41615DF8044B0121FBF751BD10B54C
:105930000C4640B139B1081DFFF78CFF28B9A368A8
:1059400033F0030301D06FF0150010BD38B50C46DD
:10595000054658B151B10B6843B14B6833B11C22B5
:10596000002100F01CFA00202C6138BD6FF01500FA
:10597000FBE770B504460E46FFF7D9FF051E31DB85
:105980004FF02003EFF3118183F31188BFF36F8F82
:105990004FF6FF75638B208BAB4200F007022ED0D1
:1059A000022A0ED1013363831546012381F3118846
:1059B000BFF36F8FB3B1002331462046FFF792FF4C
:1059C00010E0830701D0062A0ED1002333606368FC
:1059D00093B9C4E90066154662B90A462046022119
:1059E000FBF7F6FC284670BD052A0CBF6FF0850555
:1059F0006FF004050023D9E71E606660EBE76FF0E7
:105A00000A05F7E77047FDF775BC0FB407B504A9A1
:105A100051F8040B0191FBF7CDFC03B05DF804EBEA
:105A200004B07047FDF718BF70B502684C68A24219
:105A300016D38B6823449A4206D2D1E90435AB428F
:105A400004D36FF00B038B6100200AE0CD68121BBA
:105A500045F83320426805EBC306013372600B61E1
:105A6000012070BD704773B51E46836805468B42A2
:105A70000C46019210D371188B420DD3C068FFF70A
:105A8000D1FF696821448368019A1C683346A446A3
:105A900002B0BDE8704060476FF0150002B070BD05
:105AA0002DE9F8431F46836805468B420C46914614
:105AB00025D37A18934222D3C068FFF7B3FF6D68ED
:105AC00006462544D0F80880D8F80C306BB93B4620
:105AD000D8F804404A4629463046A047D8F80C304A
:105AE000044643B92046BDE8F883002198470446A0
:105AF0000028ECD0F6E7012130469847F2E76FF036
:105B00001504EFE783682DE9F0418B4205460C460A
:105B1000174624D30A44934221D3C068FFF782FF7B
:105B20006D6806462544D0F80880D8F80C3063B973
:105B3000D8F808303A46294630469847D8F80C300D
:105B4000044643B92046BDE8F08100219847044649
:105B50000028EDD0F6E7012130469847F2E76FF0D4
:105B60001504EFE708B5C068FFF75CFF83681B69A1
:105B70009847007808BD08B5C068FFF753FF8368F1
:105B80001B699847007908BDCBB20C21026903FB61
:105B90000121086C00F0070070474FF02003EFF37D
:105BA000118283F31188BFF36F8F036813F0C00372
:105BB00001D08B4207D101230360002082F31188BA
:105BC000BFF36F8F70474FF0FF30F7E710B54FF01E
:105BD0002003EFF3118283F31188BFF36F8F036803
:105BE00003F00704012C06D10160002082F3118824
:105BF000BFF36F8F10BD03F0C0038B4214BF4FF093
:105C0000FF306FF07700F1E74FF02003EFF31182E0
:105C100083F31188BFF36F8F036803F0C00343F071
:105C20000203036082F31188BFF36F8F70476FF038
:105C30008500704710B41C240069CBB203FB04003C
:105C400000215DF8044B10470020FDF715BC002033
:105C5000FDF744BC38B50C24C9B24C430546006975
:105C600004F1400380211844FFF797FF002804DB6C
:105C700069680C4463689847002038BD2DE9F041FD
:105C80000C24C9B24C430569064604F1400080214A
:105C9000284490461F46FFF799FF002806DB25445D
:105CA000C5E90E8773681B5998470020BDE8F0814D
:105CB000704770470020FBF7ADBE70470021012000
:105CC000FCF7AAB901460068FCF7A6B908B5FCF7CD
:105CD000D1F9BDE80840FCF70FBC40E800F0C3B2C2
:105CE00010F4803F14BF18466FF01500704703464C
:105CF000013911F8012F0AB91A70704703F8012B06
:105D0000F7E7034600201A5C02B970470130FAE752
:105D10000138013910F8013F11F8012F934201D1E8
:105D2000002BF7D1981A704710B55AB10139841871
:105D300010F8012B11F8013FA04201D09A42F7D090
:105D4000D01A10BD1046FCE7F0B581EA0004A507A3
:105D500003460BD0013B0A4491421BD1F0BD002AFF
:105D6000FCD011F8014B013A03F8014B9C07F6D126
:105D700022F003041D1F96080F19B94205D16FF0D8
:105D80000305234405FB0622E4E751F804CB45F85C
:105D900004CFF2E711F8014B03F8014FDCE70346AB
:105DA00070B5C9B29C0711D141EA012422F0030663
:105DB00044EA04451E449408B3420DD16FF0030534
:105DC00005FB04221A44934209D170BD002AFCD07D
:105DD00003F8011B013AE5E743F8045BECE703F83D
:105DE000011BF0E74FF0FF307047436800205B680D
:105DF0001B690B60704743685B68586842400A4003
:105E000042405A6000207047436800205B689960F8
:105E10007047436800205B68D96070474368002082
:105E20005A685368594051607047036930B55868E3
:105E300058B10024814213D108685CB99C6858604D
:105E4000A14200D198600020086072B9002030BDE6
:105E50002846EFE720609868814208BF9C60F2E71F
:105E600005680446002DF3D13AB15A680A60986873
:105E700059600028EAD19960E9E76FF01500E6E77C
:105E800038B504460D4600F067F9844209D2002C6B
:105E900007DBA84205D3611981428CBF0020012095
:105EA00038BD0020FCE72DE9F0470024836886B068
:105EB000884691465B6902AA01A99847A2462546F1
:105EC000029BAB4202D806B0BDE8F0870026019FD6
:105ED00007EBC5077B6804933A680AEB0603B242F6
:105EE00002D89A460135EBE7494603A80394059387
:105EF000C0470028E7D0049B01361C44ECE7436808
:105F00001B68D3F80423D10518D5D3F82021AAB1F2
:105F10004FF02001EFF3118281F31188BFF36F8FEF
:105F2000D3F8201131B10021C3F82011D3F820118A
:105F30000121D96082F31188BFF36F8F42685268E4
:105F4000D20615D54FF02001EFF3118281F31188AD
:105F5000BFF36F8FD3F8581111B10021C3F80015AA
:105F60004FF48001C3F8081382F31188BFF36F8FD9
:105F700070470B460269D2E9010183E80300002063
:105F8000704743681B68D3F88004C3F880047047E7
:105F900042681368D3F8580140B95268120706D412
:105FA000D3F82001003818BF012070470120704746
:105FB000436802691B68D3F8100148B10020527C85
:105FC0000A70C3F81001D3F8102101221A6070473B
:105FD0004FF0FF307047FDF727BD08B5FBF794FF82
:105FE000FFF76BFEBDE80840FDF71EBD38B50C4657
:105FF0001546FFF7C0FD21462544A94201D10120E5
:1060000038BD11F8013B9842F7D00020F8E78068CE
:1060100028387047042809D0052803D1481E18BF26
:1060200001207047431A5842584170470120704779
:1060300011B10AB1FFF7DABF0020704738B50C463E
:106040000123114622460546FFF70DFD002810DB0F
:10605000012221462846FFF7EBFF18B10323002059
:10606000237038BD2378012B0CBF0123022323703A
:10607000F7E70120F5E72DE9F7431D4606460F46F1
:106080009046FFF76FFD4419013C40420440E4B2E2
:10609000082C1AD83046FFF76EFD81462A46414645
:1060A0006846FFF751FE4946621B0DEB0500FFF7FE
:1060B00076FE23466A4639463046FFF7F1FC003843
:1060C00018BF012003B0BDE8F0834FF0FF30F9E7BF
:1060D00007B501238DF8042001AAFFF7CCFF03B018
:1060E0005DF804FB816801221839FFF7F1BF82686F
:1060F000183AFFF7A3BF13B50C46C0B201A9FBF7CE
:10610000D7FC50B921460198FDF72EF804460198B6
:10611000FFF7A8FC204602B010BD0124FAE707B53E
:1061200041EA021281688DF8072001230DF1070270
:106130002839FFF7A0FF03B05DF804FB004700F02B
:1061400083B808B50520FBF705FF20B9BDE8084076
:106150000520FBF7EFBE08BD4FF4801070474FF4E9
:10616000805070474FF4807070470369C1688B425C
:1061700097BF826803F1FF33D21802F1FF3294BF58
:10618000501A581A70472DE9F843D0E90294054691
:10619000A9EB04084068904520440F46144406D9F2
:1061A000FFF7D2FDBFF35F8FEC60BDE8F883424696
:1061B000A4EB0904FFF7C8FD2246686807EB080155
:1061C000EEE72DE9F8430646894617464FF00008EA
:1061D000C5683469B368A54228BFE418013C621B56
:1061E0005C1BBC4228BF3C46944228BF14467068E2
:1061F000494622462844FFF7A7FDB3682544AB4231
:1062000008BF0025A044A1443F1BBFF35F8FF5608A
:10621000002FDED14046BDE8F883FDF793BA08B5FC
:10622000FFF7FBFF002008BD7047C3681888C0F364
:106230000800A0F58073584258417047EFF305807D
:10624000003818BF0120704708B1FBF70FBC70473A
:1062500070472DE9F041069F044615461E46FDF79E
:106260008FFD38B93B46324629462046BDE8F0410D
:10627000FDF7ACBDBDE8F0810A460021FEF732B85B
:10628000FFF762BDFFF78BBD0A460021FFF787BD10
:1062900001EB820204388A4201D10020704752F893
:1062A000043D1BBA40F8043FF5E7FFFFC89EFF7F9F
:1062B00001000000451A0000000000001F620000FD
:1062C00000000000291B000000000000D75F000054
:1062D00000000000251C0000A4450120CD30000076
:1062E000BC4501209D300000D4450120B51E0000B2
:1062F000EC4501205528000004460120DB5F00002A
:1063000000000000092C00001C46012000000000D5
:10631000BD5C000000000000BD5C0000000000004B
:10632000BD5C000000000000BD5C0000000000003B
:10633000BD5C0000613500003D6100000000000010
:10634000BD5C000000000000BD5C0000D4450120E1
:10635000FF5E0000BC450120FF5E00000000000061
:10636000BD5C000000000000BD5C000000000000FB
:10637000BD5C000000000000D12A00000000000009
:10638000BD5C000000000000BD5C000000000000DB
:10639000BD5C000000000000BD5C000000000000CB
:1063A000BD5C000000000000BD5C000000000000BB
:1063B000BD5C000000000000651E00000000000041
:1063C000BD5C000000000000BD5C0000000000009B
:1063D000BD5C000000000000BD5C0000000000008B
:1063E000BD5C000000000000BD5C0000000000007B
:1063F000BD5C000000000000BD5C0000000000006B
:10640000BD5C000000000000BD5C0000000000005A
:10641000BD5C000000000000BD5C0000000000004A
:10642000BD5C000000000000BD5C0000000000003A
:10643000BD5C000000000000BD5C0000000000002A
:10644000BD5C000000000000BD5C0000000000001A
:10645000BD5C000000000000BD5C0000000000000A
:10646000BD5C000000000000BD5C000000000000FA
:10647000BD5C000000000000BD5C000000000000EA
:10648000BD5C000000000000BD5C000000000000DA
:10649000BD5C000000000000BD5C000000000000CA
:1064A000BD5C000000000000BD5C000000000000BA
:1064B000BD5C000000000000BD5C000000000000AA
:1064C000BD5C000000000000BD5C0000000000009A
:1064D000BD5C000000000000BD5C0000000000008A
:1064E000BD5C000000000000BD5C0000000000007A
:1064F000BD5C000000000000BD5C0000000000006A
:10650000BD5C000000000000BD5C00000000000059
:10651000BD5C00009F6D0000030000008B73000055
:10652000030000002973000003000000206A00003F
:10653000030000002B72000003000000D87400006C
:1065400003000000896D0000030000006573000077
:1065500001000000FF7FFF7FFF7FFF7FFF7FFF7F46
:10656000FF7FFF7FFF7FFF7FFF7FFF7FFF7FFF7F3B
:10657000FF7FFF7FFF7FFF7FFF7FFF7FFF7FFF7F2B
:10658000FF7FFF7FFF7FFF7FFFFFFFFFFFFFFFFF1B
:106590001D0000001C0000001A0000001B0000008D
:1065A00001000000000000000F0000000E000000CD
:1065B0000200000000000000353F00006D3F0000B9
:1065C0000338FDD87047000001000000F56C0000A2
:1065D000D46500005B0000002F5C0000555C0000EB
:1065E0007D5C000000000000895B0000DD1C0000F5
:1065F000411D0000936D0000495C00004F5C0000ED
:10660000996D0000D11B0000891B000000000000F4
:10661000000000000000000000C000002969000028
:106620000100000000C000000040000029690000D7
:1066300002000000000001000002000029690000C3
:1066400003000000000001000000070029690000AD
:10665000040000000002010000FE0600296900009D
:10666000050000000002010000000100296900008F
:10667000060000000002020000FE0500296900007B
:106680000700000000000800000007002969000062
:106690000800000000000F0000E000002969000071
:1066A0000900000000E00F00002000002969000040
:1066B0000A00000000000000B55C00000045012059
:1066C000000000000600010002000000D06600008B
:1066D00000000000AA72000002000000E0FF0F00AE
:1066E000E8440120B272000021000000E0FF032016
:1066F0001D2A0000EB5D0000F75D0000095E000050
:10670000135E00001D5E0000852800002B5E000067
:1067100000000000FFFFFFFF002584500000000084
:106720008D2C0000CD2C0000212C0000000000006A
:10673000012C0000F12B000004000000FF0000000D
:10674000B15F0000A92E0000835F00003D2D000016
:10675000735F0000008000500B00000000900050AC
:106760000B00000077C295F360D2EF7F3552500FD7
:106770002CB67980B4620000EC620000F462000084
:106780000C6300000C6300008E7400009C74000019
:10679000B0740000BF740000CB740000FF8FFFFFD7
:1067A000FF8FFFFFFE8FFFFFFE8FFFFFFD8FFFFFBD
:1067B000FC8FFFFFFC8FFFFF436F756C64206E6FD3
:1067C00074206C6F636B20706F77657220736176D5
:1067D00065206D75746578006D757465785F667297
:1067E00065652063616C6C65642077697468204E10
:1067F000554C4C20706172616D65746572000000CB
:1068000043616E277420696E697469616C697A6589
:10681000206D757465782C20776173204E554C4C33
:106820000D0A0000FFFFFFFFFFFFFFFFFFFFFFFF5D
:106830000000000000000000000000000100000057
:10684000FFFFFFFFFCFFFFFFFFFFFFFFFFFFFFFF5B
:106850000000000000000000000000000100000037
:10686000FFFFFFFF512563FCC2CAB9F3849E17A73F
:10687000ADFAE6BCFFFFFFFFFFFFFFFF00000000D7
:10688000FFFFFFFF0000000096C298D84539A1F431
:10689000A033EB2D817D0377F240A463E5E6BCF8DD
:1068A00047422CE1F2D1176BF551BF376840B6CBA8
:1068B000CE5E316B5733CE2B169E0F7C4AEBE78EA4
:1068C0009B7F1AFEE242E34FFFFFFFFF7F000000C5
:1068D000800000000000000000000000FFFFFFFF3C
:1068E0007F000000800000000000000000000000A9
:1068F00067E6096A85AE67BB72F36E3C3AF54FA551
:106900007F520E518C68059BABD9831F19CDE05B7C
:1069100025633A205374617274696E6720626F6FE9
:10692000746C6F616465720A004E52465F464C415A
:1069300053485F4452565F4E414D450025633A200F
:10694000466C6173682064657669636520257320F1
:106950006E6F7420666F756E640A0025633A205569
:106960006E61626C6520746F2066696E6420626F70
:106970006F7461626C6520696D6167650A002563EB
:106980003A20426F6F746C6F616465722063686156
:10699000696E6C6F61642061646472657373206FEB
:1069A00066667365743A20307825780A0025633A64
:1069B000204A756D70696E6720746F207468652059
:1069C000666972737420696D61676520736C6F749A
:1069D0000A0025633A2050726F74656374206D63FA
:1069E00075626F6F7420666C617368206661696C94
:1069F00065642C2063616E63656C207374617274CE
:106A000075702E0A0025633A204E657665722073F4
:106A1000686F756C642067657420686572650A002C
:106A20006D6375626F6F740025633A20696E7661DD
:106A30006C696420666C6173682049442025643B5E
:106A40002065787065637465642025640A002A8671
:106A500048CE3D0201002A8648CE3D03010700735F
:106A600065636F6E64617279007072696D617279CD
:106A70000025633A20496D61676520696E2074685E
:106A80006520257320736C6F74206973206E6F749A
:106A90002076616C6964210A0025633A2025642010
:106AA00073746174757320777269746520666169A7
:106AB0006C7320706572666F726D696E67207468A2
:106AC0006520737761700A0025633A204661696C1E
:106AD00065642072656164696E6720736563746FB5
:106AE00072733B20424F4F545F4D41585F494D47B1
:106AF0005F534543544F52533D2564202D20746FFE
:106B00006F20736D616C6C3F0A0025633A2046610B
:106B1000696C65642072656164696E6720696D6186
:106B2000676520686561646572733B20496D6167C4
:106B3000653D25750A0025633A204661696C6564E8
:106B40002072656164696E6720626F6F7420737470
:106B5000617475733B20496D6167653D25750A0059
:106B600025633A2070616E6963210A0025633A202B
:106B7000446574656374656420696E636F6E7369E0
:106B80007374656E7420737461747573210A0025C3
:106B9000633A2043616E6E6F742075706772616432
:106BA000653A206E6F74206120636F6D7061746947
:106BB000626C6520616D6F756E74206F6620736501
:106BC00063746F72730A0025633A2043616E6E6FBF
:106BD0007420757067726164653A206D6F7265200C
:106BE000736563746F7273207468616E20616C6C7E
:106BF0006F7765640A0025633A2043616E6E6F7497
:106C000020757067726164653A206E6F74207361DD
:106C10006D6520736563746F72206C61796F757434
:106C20000A00676F6F6400756E736574006261645B
:106C3000005072696D61727920696D616765002528
:106C4000633A2025733A206D616769633D25732C93
:106C500020737761705F747970653D307825782C8A
:106C600020636F70795F646F6E653D307825782C96
:106C700020696D6167655F6F6B3D307825780A002C
:106C80005365636F6E6461727920696D6167650039
:106C900025633A20426F6F7420736F757263653A93
:106CA000207072696D61727920736C6F740A0025AF
:106CB000633A20426F6F7420736F757263653A2078
:106CC0006E6F6E650A0025633A204E6F7420656E04
:106CD0006F756768206672656520737061636520F3
:106CE000746F2072756E2073776170207570677293
:106CF0006164650A003059301306072A8648CE3D84
:106D0000020106082A8648CE3D030107034200041B
:106D10002ACB403CE8FEED5BA44995A1A91DAEE855
:106D2000DBBE1937CD14FB2F245737E5953988D9A9
:106D300094B9D65AEBD7CDD5308AD6FE48B24A6A36
:106D4000810EE5F07D8B6834CC3A6AFC538EFAC133
:106D50002D002B00307800305800286E696C290017
:106D60004661696C656420746F207265626F6F7430
:106D70003A207370696E6E696E6720656E646C652B
:106D800073736C792E2E2E0A00736F6300434C4F81
:106D9000434B006866636C6B006C66636C6B0063EE
:106DA0006C6F636B5F636F6E74726F6C007379737B
:106DB0005F636C6F636B0025633A2072302F613123
:106DC0003A2020307825303878202072312F6132F7
:106DD0003A2020307825303878202072322F6133E5
:106DE0003A20203078253038780A0025633A20721E
:106DF000332F61343A2020307825303878207231B2
:106E0000322F69703A20203078253038782072315E
:106E1000342F6C723A20203078253038780A0025DB
:106E2000633A2020787073723A2020307825303809
:106E3000780A0025633A204661756C74696E672094
:106E4000696E737472756374696F6E2061646472C5
:106E500065737320287231352F7063293A2030789A
:106E6000253038780A0025633A202A2A2A2A2A203F
:106E70004D5055204641554C54202A2A2A2A2A0A88
:106E80000025633A202020537461636B696E67208C
:106E90006572726F722028636F6E746578742061FA
:106EA000726561206D69676874206265206E6F7419
:106EB0002076616C6964290A0025633A20202055F8
:106EC0006E737461636B696E67206572726F720AAC
:106ED0000025633A2020204461746120416363658A
:106EE00073732056696F6C6174696F6E0A00256355
:106EF0003A2020204D4D4641522041646472657312
:106F0000733A20307825780A0025633A20202049FA
:106F10006E737472756374696F6E20416363657319
:106F2000732056696F6C6174696F6E0A0025633A4D
:106F3000202020466C6F6174696E672D706F696EDA
:106F400074206C617A792073746174652070726545
:106F5000736572766174696F6E206572726F720A02
:106F60000025633A202A2A2A2A2A204255532046FD
:106F700041554C54202A2A2A2A2A0A0025633A20FD
:106F80002020537461636B696E67206572726F7243
:106F90000A0025633A2020205072656369736520DA
:106FA0006461746120627573206572726F720A0089
:106FB00025633A2020204246415220416464726594
:106FC00073733A20307825780A0025633A20202010
:106FD000496D7072656369736520646174612062D4
:106FE0007573206572726F720A0025633A20202043
:106FF000496E737472756374696F6E206275732065
:107000006572726F720A0025633A202A2A2A2A2A98
:10701000205553414745204641554C54202A2A2AA1
:107020002A2A0A0025633A20202044697669736978
:107030006F6E206279207A65726F0A0025633A20AC
:107040002020556E616C69676E6564206D656D6F9B
:107050007279206163636573730A0025633A2020A7
:1070600020537461636B206F766572666C6F772056
:1070700028636F6E746578742061726561206E6F2D
:10708000742076616C6964290A0025633A20202007
:107090004E6F20636F70726F636573736F722069D8
:1070A0006E737472756374696F6E730A0025633A48
:1070B000202020496C6C6567616C206C6F616420D6
:1070C0006F66204558435F52455455524E20696EB5
:1070D000746F2050430A0025633A202020496C6CCD
:1070E0006567616C20757365206F66207468652024
:1070F000455053520A0025633A202020417474659C
:107100006D707420746F2065786563757465207583
:107110006E646566696E656420696E73747275630A
:1071200074696F6E0A0052657365727665642045F6
:107130007863657074696F6E20280053707572698A
:107140006F757320696E746572727570742028494A
:107150005251200025633A20535053454C20696E0C
:1071600020746872656164206D6F646520646F656A
:1071700073206E6F7420696E64696361746520505A
:1071800053500A0025633A202A2A2A2A2A204841F5
:107190005244204641554C54202A2A2A2A2A0A00C1
:1071A00025633A202020427573206661756C742037
:1071B0006F6E20766563746F72207461626C6520F7
:1071C000726561640A0025633A2020204661756C6F
:1071D0007420657363616C6174696F6E20287365D8
:1071E000652062656C6F77290A0025633A202A2A98
:1071F0002A2A2A204465627567206D6F6E69746F54
:107200007220657863657074696F6E202A2A2A2A55
:107210002A0A0025633A202A2A2A2A2A20257320AE
:10722000256429202A2A2A2A2A0A006D7075002539
:10723000633A204661696C656420746F20616C6CF0
:107240006F63617465206E6577204D5055207265BF
:1072500067696F6E2025750A0A0025633A20506120
:1072600072746974696F6E2025753A2073616E6956
:10727000747920636865636B206661696C65642E50
:107280000A0025633A20496E76616C696420756E48
:107290006465726C79696E6720726567696F6E20CC
:1072A000696E6465782025750A00464C4153485F35
:1072B00030005352414D5F30004750494F5F30001E
:1072C00025633A20756E616C69676E656420616440
:1072D00064726573733A2030782530386C783A25BB
:1072E0007A750A0025633A20696E76616C696420BC
:1072F000616464726573733A2030782530386C7835
:107300003A257A750A0025633A206E6F7420776FEC
:1073100072642D616C69676E65643A20307825303F
:10732000386C783A257A750A00666C6173685F6E0E
:1073300072660025633A204661696C656420746F4B
:1073400020616C6C6F636174652050504920436804
:10735000616E6E656C0A00554152545F31005541B3
:1073600052545F3000756172745F6E7266785F753B
:10737000617274650025633A20526573657474699F
:107380006E672073797374656D0A00666174616C51
:107390005F6572726F7200726576657274007465F3
:1073A0007374007065726D004255473B2063616ED7
:1073B00027742068617070656E0025633A205377EA
:1073C000617020747970653A2025730A0025633A4C
:1073D000205377617020747970653A206E6F6E6506
:1073E0000A0004010403040204010401040301036C
:1073F000030401045465726D696E616C005254544B
:107400000053454747455200556E6B6E6F776E20AF
:107410006572726F720025633A203E3E3E205A45E7
:107420005048595220464154414C204552524F52E7
:107430002025643A202573206F6E20435055202567
:10744000640A0025633A204661756C742064757285
:10745000696E6720696E74657272757074206861F8
:107460006E646C696E670A0A00756E6B6E6F776E7C
:107470000025633A2043757272656E7420746872D9
:107480006561643A20257020282573290A0043503D
:107490005520657863657074696F6E00556E68611C
:1074A0006E646C656420696E7465727275707400C8
:1074B000537461636B206F766572666C6F77004BF7
:1074C00065726E656C206F6F7073004B65726E65D0
:1074D0006C2070616E6963006F730076322E362EF9
:1074E000302D7263312D6E637331002A2A2A2042B7
:1074F0006F6F74696E67205A6570687972204F5398
:10750000206275696C64202573202573202A2A2A3D
:107510000A000000FFFFFFFFFFFFFFFFFFFFFFFF6D
:10752000FFFFFFFFFFFFFFFFFFFFFFFFFFFFFFFF6B
:10753000FFFFFFFF9F5D00008F58000010660000F6
:10754000E55D00000000000000C201000001030032
:1075500000000000000000000000000000C2010068
:107560000001030000000000000000000090D003B4
:1075700000000000613A00007C45012088450120A0
:10758000804501207845012054450120E05001202C
:1075900001000000113D0000ED3C0000313D000005
:1075A000CD3C00009C450120604501209445012010
:1075B000000000008C450120E45001200100000083
:1075C000E850012001000000EC5001200100000003
:1075D0008D6D0000EC650000D8650000244F01208F
:1075E000384F01207E650000577300005C67000083
:1075F00040670000D04F01202C4501207465000039
:107600005E7300005467000040670000CC4F01200B
:10761000184501206A650000AD6D00000000000003
:1076200000000000904F0120000000006465000091
:10763000B972000014670000F0660000A04F01203E
:10764000A44F01205C6500002969000000000000D3
:1076500020670000C04F01200000000054650000BA
:020000040001F9
:100000003DB8F396000000000002000038B903007C
:1000100000000000000000000000000000000000E0
:10002000FFFFFFFFFFFFFFFFFFFFFFFFFFFFFFFFE0
:10003000FFFFFFFFFFFFFFFFFFFFFFFFFFFFFFFFD0
:10004000FFFFFFFFFFFFFFFFFFFFFFFFFFFFFFFFC0
:10005000FFFFFFFFFFFFFFFFFFFFFFFFFFFFFFFFB0
:10006000FFFFFFFFFFFFFFFFFFFFFFFFFFFFFFFFA0
:10007000FFFFFFFFFFFFFFFFFFFFFFFFFFFFFFFF90
:10008000FFFFFFFFFFFFFFFFFFFFFFFFFFFFFFFF80
:10009000FFFFFFFFFFFFFFFFFFFFFFFFFFFFFFFF70
:1000A000FFFFFFFFFFFFFFFFFFFFFFFFFFFFFFFF60
:1000B000FFFFFFFFFFFFFFFFFFFFFFFFFFFFFFFF50
:1000C000FFFFFFFFFFFFFFFFFFFFFFFFFFFFFFFF40
:1000D000FFFFFFFFFFFFFFFFFFFFFFFFFFFFFFFF30
:1000E000FFFFFFFFFFFFFFFFFFFFFFFFFFFFFFFF20
:1000F000FFFFFFFFFFFFFFFFFFFFFFFFFFFFFFFF10
:10010000FFFFFFFFFFFFFFFFFFFFFFFFFFFFFFFFFF
:10011000FFFFFFFFFFFFFFFFFFFFFFFFFFFFFFFFEF
:10012000FFFFFFFFFFFFFFFFFFFFFFFFFFFFFFFFDF
:10013000FFFFFFFFFFFFFFFFFFFFFFFFFFFFFFFFCF
:10014000FFFFFFFFFFFFFFFFFFFFFFFFFFFFFFFFBF
:10015000FFFFFFFFFFFFFFFFFFFFFFFFFFFFFFFFAF
:10016000FFFFFFFFFFFFFFFFFFFFFFFFFFFFFFFF9F
:10017000FFFFFFFFFFFFFFFFFFFFFFFFFFFFFFFF8F
:10018000FFFFFFFFFFFFFFFFFFFFFFFFFFFFFFFF7F
:10019000FFFFFFFFFFFFFFFFFFFFFFFFFFFFFFFF6F
:1001A000FFFFFFFFFFFFFFFFFFFFFFFFFFFFFFFF5F
:1001B000FFFFFFFFFFFFFFFFFFFFFFFFFFFFFFFF4F
:1001C000FFFFFFFFFFFFFFFFFFFFFFFFFFFFFFFF3F
:1001D000FFFFFFFFFFFFFFFFFFFFFFFFFFFFFFFF2F
:1001E000FFFFFFFFFFFFFFFFFFFFFFFFFFFFFFFF1F
:1001F000FFFFFFFFFFFFFFFFFFFFFFFFFFFFFFFF0F
:1002000090260020AD1F0100856801000D2001002F
:100210000D2001000D2001000D2001000D20010026
:10022000000000000000000000000000091E0100A6
:100230000D20010000000000B11D0100B3670100A6
:100240006D1F01006D1F01006D1F01006D1F01007A
:100250006D1F01006D1F01006D1F01006D1F01006A
:100260006D1F01006D1F01006D1F01006D1F01005A
:100270006D1F01006D1F01006D1F01006D1F01004A
:100280006D1F01006D1F01006D1F01006D1F01003A
:100290006D1F01006D1F01006D1F01006D1F01002A
:1002A0006D1F01006D1F01006D1F01006D1F01001A
:1002B0006D1F01006D1F01006D1F01006D1F01000A
:1002C0006D1F01006D1F01006D1F01006D1F0100FA
:1002D0006D1F01006D1F01006D1F01006D1F0100EA
:1002E0006D1F01006D1F01006D1F01006D1F0100DA
:1002F0006D1F01006D1F01006D1F01006D1F0100CA
:100300006D1F01006D1F01006D1F01006D1F0100B9
:100310006D1F01006D1F01006D1F01006D1F0100A9
:100320006D1F01006D1F01006D1F01006D1F010099
:100330006D1F01006D1F01006D1F01006D1F010089
:100340006D1F010000000000000000000000000020
:10035000000000000000000000000000000000009D
:10036000000000000000000000000000000000008D
:10037000000000000000000000000000000000007D
:10038000000000000000000000000000000000006D
:10039000000000000000000000000000000000005D
:1003A000000000000000000000000000000000004D
:1003B000000000000000000000000000000000003D
:1003C000000000000000000000000000000000002D
:1003D000000000000000000000000000000000001D
:1003E000000000000000000000000000000000000D
:1003F00000000000000000000000000000000000FD
:10040000DEE61E284CBBCE8F025B00003C000000E5
:10041000007E000001000000000201000002010057
:10042000FFFF02910000000000000000000000003B
:1004300000000000000000000000000053B94AB9AD
:10044000002908BF00281CBF4FF0FF314FF0FF30DC
:1004500000F084B9ADF1080C6DE904CE00F006F8A7
:10046000DDF804E0DDE9022304B070472DE9F04F28
:10047000099E0D4604468A46002B40F085808A423C
:10048000174644D9B2FA82F24AB1C2F1200105FA04
:1004900002F39740944020FA01F141EA030A4FEA3F
:1004A00017484FEA144C1FFA87F9BAFBF8FE08FB0D
:1004B0001EA30EFB09F14CEA0343994207D9FB182E
:1004C0000EF1FF3002D2994200F230818646591A6D
:1004D000A3B2B1FBF8F008FB101100FB09F943EAE5
:1004E0000144A14507D93C1900F1FF3302D2A145CF
:1004F00000F219811846A4EB090440EA0E400021DD
:100500001EB1D4400023C6E90043BDE8F08F02B914
:10051000FFDEB2FA82F2002A51D1CB1B4FEA174E0E
:100520001FFA87F80121250CB3FBFEFC0EFB1C30E3
:1005300008FB0CF945EA0045A9450BD97D190CF1DA
:10054000FF332CBF01200020A94502D9002800F06C
:10055000F1809C46A5EB0905A3B2B5FBFEF00EFBAE
:10056000105508FB00F843EA0544A04507D93C199B
:1005700000F1FF3302D2A04500F2D2801846A4EB6E
:10058000080440EA0C40BBE78B4208D9002E00F07B
:10059000BE800021C6E900050846BDE8F08FB3FA29
:1005A00083F100294DD1AB42C0F0B480824240F2C9
:1005B000B1800846002EA8D0C6E9004AA5E7C2F1DE
:1005C0002000974001FA02F34FEA174EC14024FA87
:1005D00000F51FFA87F894401D43B1FBFEF02B0C89
:1005E0000EFB101100FB08FC43EA01439C450ED9A9
:1005F000FB1800F1FF312CBF4FF001094FF000094B
:100600009C4503D9B9F1000F00F098800846A3EB90
:100610000C03ADB2B3FBFEF10EFB113301FB08FC82
:1006200045EA0345AC4507D97D1901F1FF3302D2F4
:10063000AC4500F28A801946A5EB0C0341EA004163
:1006400071E7C1F120048B4002FA01F705FA01FCC1
:10065000E24020FA04F8E54000FA01FE134348EABC
:100660000C024FEA13484FEA124C1FFA83F9B5FB0C
:10067000F8FA08FB1A550AFB09F04CEA054C6045EC
:100680000ED913EB0C0C0AF1FF352CBF4FF0010B08
:100690004FF0000B604502D9BBF1000F51D0AA46C4
:1006A000ACEB000C92B2BCFBF8F008FB10CC00FBEA
:1006B00009F942EA0C4CE14507D913EB0C0C00F1A7
:1006C000FF3201D2E14543D8104640EA0A40ACEB84
:1006D000090CA0FB0789CC4545464A4602D306D102
:1006E000C64504D20138B8EB070569EB030296B39F
:1006F000BEEB05036CEB020C23FA01F20CFA04F4D6
:100700002CFA01F300211443C6E90043FDE631460B
:100710003046FAE6841A65EB030301209A4649E75E
:1007200002383C442BE702383C44E4E6AEF1020ECA
:100730003B44CCE6ACF1020C3D440BE702383B44B1
:1007400065E7AAF1020A9C44AAE702393D4473E72F
:1007500002389C44B9E73146D7E600BF704700BF76
:100760002DE9E04F2746A046A146A246A346A4464F
:10077000A2B02DEC000A84F3008825462646A44743
:100780003DEC000A22B0BDE8E08F00000B680133A9
:100790000B60014B1B6818470000002007B50B4693
:1007A000002102460191034801A900F0E5F803B0D9
:1007B0005DF804FB8D0701002DE9F84FB0F81890A3
:1007C000044619F0080893460DD001290CBF49F0E2
:1007D000100949F02009A0F818908BF31188BFF395
:1007E0006F8FBDE8F88F09F00709022907D120466D
:1007F00005F022FE0028F0D00128238B4ED1676936
:10080000218B002F15DA256821F00701C4E9008843
:1008100041F0010121830026218B01F0070ACA451E
:1008200002D0A368002B5AD10DB9002E71D000233D
:1008300056E001F007035A1F012A1ED821F00701D4
:10084000062B256889B2C4E900880AD13DB12A4641
:10085000638B126801339BB2002AFAD1638341F0A3
:1008600002012046218305F0E7FD06460028D3D08B
:10087000238B43F020032383CDE7042B0CD121F0FD
:10088000070189B22046218305F0D6FD05460028E0
:10089000C1D041F0200121830025BCE7032809D104
:1008A000226923F00703166843F00603002523831B
:1008B0002F46B1E7042806D1226923F007035668C2
:1008C00043F00403F2E7052806D1226923F0070369
:1008D000966843F00503E9E700252E46E8E7012383
:1008E00041F0080121838BF31188BFF36F8FFBB9AF
:1008F00085BB16B120461F49B0474FF02003EFF3E8
:10090000118B83F31188BFF36F8F238B23F00803C0
:100910002383238BDA0625D5012123F010032383BB
:10092000B4F8189009F0070900297FF45EAF54E786
:10093000A1680029DCD0D1F800903B465246204601
:10094000D1F804B0D847B9F1000FD1D04946D9F851
:100950000090F2E729463B46524620462D6805F0B6
:1009600087FDC5E713F020011EBF23F020030221FD
:100970002383D5E79D6401002DE9F04F8B46924615
:100980001C46002591B002909AF8000008B928464C
:100990005EE325280AF1010707D05946029B9847D4
:1009A0000028C0F25583013510E2182200210AA860
:1009B00005F0FCFF9AF80130252B78D000229446F0
:1009C000164696461046394617F8013B2B2B00F089
:1009D0009D8000F29480202B00F09B80232B00F060
:1009E0009A8028B19DF8300040F004008DF8300066
:1009F000BEF1000F05D09DF8300040F008008DF8E2
:100A000030002EB19DF8300040F010008DF830001D
:100A1000BCF1000F05D09DF8300040F020008DF8AB
:100A200030002AB19DF8302042F040028DF830208D
:100A30009DF8302002F04400442803D16FF3861261
:100A40008DF830209DF830202A2B42F080028DF85E
:100A500030207BD19DF831204B1C42F001028DF8F3
:100A600031201A782E2A0CBF012100219DF8312057
:100A700061F341028DF8312074D15A782A2A6AD064
:100A800000210A260133184610F8012BA2F1300785
:100A9000092F40F28E809DF830200E91C2F3400065
:100AA00040EAD17161F341028DF830205AE00AF139
:100AB00002078DF833309DF83130D90740F1498174
:100AC00054F8049BB9F1000F07DA9DF83020C9F102
:100AD000000942F004028DF830205A0740F14281AB
:100AE00054F8048BB8F1000F80F241819DF8313049
:100AF0006FF341038DF831304FF0FF3837E12D2B84
:100B00000CD0302B7FF46DAF01225CE74FF0010E6B
:100B100059E7012657E74FF0010C54E7012052E74F
:100B200033460CFB0202303A1E4616F8010BA0F1C8
:100B30003007092FF4D9994293D09DF830100D92C7
:100B4000D20F62F341018DF830108AE70B46002284
:100B50004FF00A0CE8E79DF83120023342F004021E
:100B60008DF831201F4617F8012B6C2A41D025D86B
:100B7000682A2BD06A2A46D04C2A4CD01F4617F838
:100B8000012B9DF83130782A8DF8332000F2D9807E
:100B9000572A4DD8412A03D0453A022A00F2D18083
:100BA00004229DF8323062F302038DF832300123C3
:100BB0009EE006FB01210346303964E7742A26D003
:100BC0007A2ADBD106229DF831300DE05A78682A66
:100BD0009DF8312006D1012161F3C6028DF8312044
:100BE0009F1CCCE71346022262F3C6038DF8313016
:100BF000C5E75A786C2A9DF8312001D10421EBE732
:100C000013460322F0E705229DF83130ECE7072276
:100C10009DF83130E8E7BDF8303023F4F04323F09D
:100C2000020343F4804343F00203ADF83030A6E7FB
:100C3000A2F15801202900F2848001A050F821F08F
:100C4000050D0100430D0100430D0100430D01009E
:100C5000430D0100430D0100430D0100430D010050
:100C6000430D0100A10B0100430D0100050D010022
:100C7000C50C0100A10B0100A10B0100A10B01009B
:100C8000430D0100C50C0100430D0100430D01009F
:100C9000430D0100430D01000D0D0100050D010084
:100CA000290D0100430D0100430D0100290D010034
:100CB000430D0100050D0100430D0100430D01002E
:100CC000050D010001209DF8321003F0780360F358
:100CD0000201402B8DF8321002BF9DF8301041F018
:100CE00001018DF83010632A31D1003B18BF012378
:100CF0009DF83020C2F340010B4363F341028DF8AD
:100D00003020D8E602209DF83210DEE703219DF85E
:100D1000322003F07803A3F1400061F30202434262
:100D20008DF832204341E3E703219DF8322013F090
:100D3000780F61F3020214BF012300238DF83220E3
:100D4000D6E79DF8303043F001038DF830300023B2
:100D5000CEE79DF93020002AACBF4FF0FF39DDF817
:100D60003490BAE69B077FF5C7AEDDF838800023E4
:100D7000CDE90D339DF832309DF8312003F00703A3
:100D8000012BC2F3C30236D1D31E042B20D8DFE8D7
:100D900003F00307071F1F0054F8040BC11704E0FA
:100DA000073424F00704F4E80201CDE90A019DF8B4
:100DB000303013F0030654D03B4652465946029851
:100DC00005F03AFC0028C0F243810544BA46DBE551
:100DD00054F8040B012A4FEAE071CDE90A0105D16C
:100DE0009DF828300A9300230B93E0E7022ADED116
:100DF000BDF92800D2E7022B23D1D31E042B13D830
:100E0000DFE803F0030A0A12120000212068231D04
:100E10000A900B911C46CAE7073424F00703F3E855
:100E20000201CDE90A01F5E754F8043B012A0A93CF
:100E30004FF000030B93D3D0022AB8D1BDF828306D
:100E4000D0E7042B07D1073424F00704F4E80201AB
:100E5000CDE90A01ABE7032B04BF54F8043B0A9326
:100E6000A5E79DF833007828B0D8622822D8252835
:100E70003FF493AD5828A9D1DDE90A010DF126030D
:100E800000930CAA04AB05F08CFB8246B8F1000F6E
:100E90000DF126000CDB9DF83020A0EB0A036FF368
:100EA000861298458DF8302002D9A8EB03030D93E4
:100EB00080463DE06338152888D801A151F820F01C
:100EC000410F0100A50F0100CD0D0100CD0D010066
:100ED000CD0D0100CD0D0100A50F0100CD0D0100CC
:100EE000CD0D0100CD0D0100CD0D0100031001005D
:100EF000D10F0100D50F0100CD0D0100CD0D010076
:100F0000190F0100CD0D0100D10F0100CD0D010021
:100F1000CD0D0100D10F0100B8F1000FDDF828A0C0
:100F20000ADB4146504605F0E6FC00260AEB0008C5
:100F3000BAF1000F0CD149E7504605F0D5FCF4E7B3
:100F400000260A9B0DF111088DF810300DF1100AE2
:100F5000A8EB0A0306B101339DF83220D0066BD509
:100F6000023352060D9948BF0E9A0B4448BF9B1896
:100F7000B9F1000F79DD9DF83020A9EB0309C2F328
:100F800080030393530770D4500664D546B1594685
:100F90003046029B984700285ADB039B01351E46CA
:100FA000302359E01E0711D413F0100618BF202675
:100FB000DDE90A23002A73F10001BFF65DAF52425A
:100FC00063EB43032D26CDE90A2355E72B26EFE7F4
:100FD000002651E70A9848B30DF12603009300213B
:100FE00004AB0CAA05F0DDFABDF83230824603F0FE
:100FF000EF0343F4F04343F010030026ADF8323022
:1010000044E70A9B072A3FF6E1AEDFE802F00D0451
:10101000060D08080D0D1D70D8E61D80D6E6284681
:10102000E917C3E90001D1E61D60CFE6DFF8C4800F
:101030000646A8F1050A8BE7110748BF013390E780
:10104000184603935946029B98470028039B04DAED
:1010500011B0BDE8F08F20234D444A46002AA5EB8D
:10106000090109F1FF39EBDC0D4636B1594630462E
:10107000029B98470028EBDB01359DF83230D906FA
:1010800001D41A0706D559463020029B98470028FC
:10109000DEDB01359DF83230DB0607D559469DF879
:1010A0003300029B98470028D2DB01350D9E2E4469
:1010B000731B002B16DC434652465946029805F036
:1010C000BBFA0028C4DB0544A944A9EB0503002BA7
:1010D0007FF77CAE59462020029B98470028B7DB5B
:1010E0000135F2E759463020029B98470028AFDBD4
:1010F0000135DDE7C8720100044608B54FF0200253
:10110000EFF3118382F31188BFF36F8F05F053FB68
:10111000204601F09DF8034805F081F900F0EEFE4D
:10112000FCE700BFC97201004FF02002EFF311830A
:1011300082F31188BFF36F8F0121044AC2F8401572
:1011400083F31188BFF36F8F002070470090035026
:1011500020B1034B800143F001031847704700BFE3
:10116000906F010084B004AB03E907009DF80430E0
:10117000062B07D10122044BC3F80025BFF34F8F84
:1011800020BFFDE704B0704700400050F8B50546A9
:101190004FF02003EFF3118683F31188BFF36F8FB5
:1011A000094B1C685CB1094FD4E90132002D08BF1E
:1011B00013460BB1387898472468002CF4D186F395
:1011C0001188BFF36F8FF8BD480200205002002045
:1011D000084B10B51C685CB901221A60064B93E8F5
:1011E000070005F042FA2046BDE81040FFF7CEBFE9
:1011F00010BD00BF0400002050020020F0B585B0F3
:101200006E46184C01460546304605F039FA96E818
:10121000070084E80700207808B30021124B19600A
:101220006B1C0ED017464FF4004600210F480023D8
:10123000E6FB07010E4AFFF701F90121281A05F024
:1012400031FD01F077FF0120FFF7A0FF94E80700D0
:10125000FFF788FFFFF7BCFF02F05EF8207805B0CB
:10126000F0BD00BF50020020040000203F420F00EC
:1012700040420F000E4A70B5841A05460C200E46F7
:101280004021A3100B4C5C43E4B200FB0420084453
:1012900005F004FA011E05DB074B03EBC404636889
:1012A0009847002128463346BDE87040184700BFE4
:1012B00070020020B76DDBB6AC6F01002DE9F04184
:1012C0000C25104E8046841BA3100F4C0F465C4328
:1012D000E4B2654305F140004021304405F0F7F9E0
:1012E000011E09DB094A7319C3E90E27084B53F89D
:1012F0003430BDE8F041184740463B46BDE8F04178
:10130000184700BF70020020B76DDBB631670100DF
:10131000AC6F010070B5002201210446052000F0E9
:10132000A1FD052000F080FD0F4801F019FB0F4BD7
:10133000984215D105F06FFB26690D49304605F03E
:10134000CAF800280BDB012535642469084904F13B
:101350001C0005F0C0F8002801DB0020E56470BD2A
:101360006FF00400FBE700BFA91301000000AD0B04
:10137000BC6F010001460C2300224B43084870B5A6
:10138000C4184033D4E90E561844A26305F0BDF9E1
:101390002DB132462B46BDE870400248184770BD5B
:1013A00070020020A400002010B1012804D0704772
:1013B000034B1B6C5B0701D1FFF7DCBF704700BF1D
:1013C0007002002008B54FF02003EFF3118183F382
:1013D0001188BFF36F8F124A136843F0020013F0B5
:1013E000010310600CD04FF05022D2F80C34D2F828
:1013F0000C2413F0010303D00A4805F086F90123F9
:1014000081F31188BFF36F8F23B1BDE8084000203E
:10141000FFF7B0BF0120BDE8084001F0B1BA00BF3E
:10142000C0020020B0020020074BD3E8EF2F22F0CB
:101430000201C3E8E01F0028F7D1D30702D401203E
:1014400001F0D0BA704700BFC00200201FB50022D3
:101450000123CDE902236B46084ACDF800D0CDF830
:1014600004D005F08BF9002805DB4FF480420023FF
:10147000684601F0DBFD05B05DF804FB4F67010035
:101480002DE9F843012206463949D1E8EF3FC1E88A
:10149000E02F0028F9D133B9364937484B60CB608B
:1014A0008A6005F02BF8731E012B32D8012E07D16C
:1014B0004FF05023D3F81C3403F00303022B28D041
:1014C00005F014FB044618B92C4B1B78002B47D1B0
:1014D0004FF02003EFF3118583F31188BFF36F8F73
:1014E0000124274FDFF89C80DFF89C904FF05022BA
:1014F000D2F81834D2F81824D2030CD503F0030321
:10150000022B01D0012E06D124B385F31188BFF33D
:101510006F8FBDE8F883C4B1284600F0FDFC4FF0A2
:101520005022D2F81835DBB2012BDFD139680029FF
:10153000DCD00021396039680221C2F81815202258
:10154000C8F88021C9F80030D0E70021212002F03E
:1015500073F8E4E74FF050230222C3F80423D8E7DE
:101560004FF0502302220546C3F80823B9E700BF15
:10157000C4020020600200208C0200208D16002092
:101580000451005000E100E008500050044A136884
:10159000C81A20F07F400344136002F0B9B900BFBD
:1015A000D80200202DE9F0474FF480374FF00009B2
:1015B000860000F1500406F15026A40006F580369E
:1015C000A4B204F15024D6F84035DFF86C8021F045
:1015D0007F4504F580348740D8F804A5A3EB0A03BF
:1015E00023F07F432AF07F42012BC6F8402502D129
:1015F000132005F075FB0AF10202AB1A23F07F43BA
:10160000B3F5000F88BF1546C4F80090236825F095
:101610007F43C8F84473C6F84035D8F804359A4576
:1016200006D0EB1A023B23F07F43B3F5000F01D83D
:10163000BDE8F0872B46CFE700500150F8B50024F5
:1016400027460F4E0F4B104A18461D6804B1F8BDCF
:10165000D2F80413C903FAD531680029F7D03460F1
:1016600031684FF48031C2F848130124D2F8401594
:1016700025B100205A681F60A847E3E70560E6E748
:1016800040510150CC0200200050015038B50024D8
:101690004FF480334FF400120D4D0121C5F8084579
:1016A000C5F804330B4B1520C3F88021224600F007
:1016B000D9FB152000F0B8FB0123074A0220136074
:1016C000064A2B601360FFF7DBFE204638BD00BFE3
:1016D0000050015000E100E008500150D402002009
:1016E000134BB0F1FF3F08BF1846013800281CDD3E
:1016F0009842A8BF18460F4BD3F804250E4B196823
:10170000521A12F4000F18BF002022F07F43013359
:101710000A4A03440A48106000205060044A934279
:1017200094BFC9188918FFF73DBF0020E3E700BF49
:10173000FFFF7F0000500150D8020020CC020020A3
:101740008D150100044BD3F80405044B1B68C01A27
:1017500020F07F40704700BF00500150D8020020A9
:1017600000280DDB0122430900F01F0002FA00F0FF
:10177000044A203342F82300BFF34F8FBFF36F8F2B
:10178000704700BF00E100E0F7B500281C4614BF19
:101790004FF400534FF400438A42154640D90A469D
:1017A000204F002839D002F5E07647F82640561C35
:1017B000B54230D15D431C484B43009504F02FFEE9
:1017C0001A4B14F0100F1A491A4808BF194604F0B2
:1017D00026FE14F0040F14BF72212D21164804F0C8
:1017E0001EFE14F0020F14BF77212D21124804F0C1
:1017F00016FE14F0010F0CBF2D2178210E4804F0C5
:101800000EFE6C210C4804F00AFE0C4803B0BDE843
:10181000F04004F004BE3246C3E702F5C076C4E7E8
:1018200003B0F0BD003000501173010005730100DA
:10183000FC720100907401002B73010072760100AC
:1018400030B5274C85B021462648274D04F0E7FDEA
:101850002168264804F0E3FD2968254804F0DFFDEF
:1018600010220021684605F0A1F82368684600931D
:10187000029400F053FD012000F080FD002000F0F4
:1018800069FD002000F08EFD0121002000F0A8FD80
:1018900000F09CFD17482C6804F0C1FD0820FFF7FC
:1018A0005FFF154A24F00104D2F82038002B07DA34
:1018B00003F00303023B012B9CBF104BC2F82038FE
:1018C0000121082004F0A5FFBFF34F8FBFF36F8FF6
:1018D000640864002046214622462346FEF740FF66
:1018E000000202002E730100040202004573010091
:1018F0005A7301007873010000300050000100802D
:101900002DE9F843494804F08AFD002140F21713FD
:1019100008460422FFF738FF40F207132022042173
:101920000020FFF731FF424804F079FD414B424A65
:10193000C3F3C431C3F30E03C3F50043C3F343132E
:10194000C2F80015C2F80435D2F80015D2F8042503
:101950003A48520104F063FD354804F060FD00F0A0
:10196000A7F8014610B1364804F059FD0024354867
:1019700004F055FD40F21713082200210120FFF763
:1019800003FF2D4D40F20713202208210120FFF70D
:10199000FBFE274804F043FDC5F880442A4804F0C4
:1019A0003EFD2A4EC5F8C044294F2A4DDFF8B480C9
:1019B00095F805902146B9F1000F14BF33463B4618
:1019C00040462A6804F02BFDB9F1000F0CD12248E3
:1019D000013404F024FD1C2C05F10805E8D114485D
:1019E000BDE8F84304F01BBD95F8049095F9040098
:1019F000FFF7B6FE4FEA890303F1A04303F5405316
:101A0000B9F1310FD3F8002806D0002A07DA02F026
:101A10000302023A012A02D8104AC3F80028012121
:101A2000484604F0F6FE0E48D2E700BFAE73010050
:101A300072760100E07F010000300050D273010097
:101A400018740100487401006A740100A373010056
:101A500009730100C86F0100937401000001008048
:101A60009A740100867401002DE9F04307460026B0
:101A700085B0DFF83490DFF8348001AD59F8044BBD
:101A800098E807003C4485E807000C2229462046D8
:101A900004F03AFF00B91CB90136052EEED100243E
:101AA000204605B0BDE8F083A8700100606F01001A
:101AB00000220248114602F007B800BFDC020020F5
:101AC00070B50C461546064650B96FF01500BDE8D6
:101AD0007040714672467346F4468EF3008C74472C
:101AE000002AF2D004F0DEFE0128EED0B4F5803FEB
:101AF00017D32B19B3F5813F06D90B4A94420AD963
:101B000002F61D22934209D82A462146304604F0A7
:101B100022FF0020DBE7054A944202D9044A93429F
:101B2000F2D94FF0FF30D2E70302FF002F01FF0090
:101B30003801FF0070B506460D46144604F0B2FEAB
:101B400001280DD0204604F0ADFE012808D0234620
:101B50002A463146084801F0EBFF2368AB4201D02A
:101B60006FF01500BDE87040714672467346F4464A
:101B70008EF3008C744700BFDC02002070B5054670
:101B800010460E46144604F08DFE01280AD16FF06F
:101B90001500BDE87040714672467346F4468EF3F8
:101BA000008C74472846FFF75FFF05463046FFF775
:101BB0005BFF0346CDB1296A0E4A914215D148B167
:101BC0000120196A0B4A914202D138B92070E0E72E
:101BD0000028DCD0012300202370DAE75B696A6902
:101BE0009A4234BF00230123F5E7002BCFD0002019
:101BF000E7E700BFFFFF0291014801F05DBF00BFB2
:101C0000BC70010008B5B0B14368042B0DD10022AF
:101C10000368D3E8EF1F012903D1C3E8E02F0028B0
:101C2000F7D1074808BF104608BD3BB1006801F076
:101C300097F90020F8E76FF4E040F5E70148F3E793
:101C4000E98FFFFFEA8FFFFF10B5044618B90D4B6F
:101C50000D485B689847616808290DD031F004038E
:101C60000AD011F0020108D02146084804F015FFFF
:101C7000002323600023636010BD1422206804F059
:101C800095FEF7E734000020AB75010098040020B2
:101C900010B5044618B9164B16485B689847636838
:101CA000042B23D0082B21D0CBB92368BBB94FF02C
:101CB000FF324FF0FF3321460F4801F005F808B915
:101CC00023681BB90A4B0D485B6898471422002112
:101CD000206804F06BFE636843F0020363602068D1
:101CE00004F011FF636843F00103636010BD00BF9F
:101CF00034000020AB75010098040020D17501006C
:101D000008B5E8B14368042B0CD101220368D3E87D
:101D1000EF1F002903D1C3E8E02F0028F7D10BD132
:101D2000002008BD53B100684FF0FF324FF0FF3381
:101D300001F09EF80028F3D00348F2E70348F0E7EB
:101D40006FF4E040EDE700BFE98FFFFFEA8FFFFF90
:101D500008B5064940231422054804F083FEBDE877
:101D600008400449044801F04FBF00BFB4040020FC
:101D700098040020D4700100C4700100094A0A4987
:101D8000936809685867996708494B6843F080531E
:101D90004B60002383F31188BFF36F8F9368986FB4
:101DA000704700BF900B00203871010000ED00E08B
:101DB00013498A684FF030001044EFF3098C80E833
:101DC000F01F202080F31188BFF36F8F0D4F4FF06D
:101DD00000664A6A8A603E60506F0023536780F352
:101DE000118802F1300090E8F01F8CF3098802F1AD
:101DF000000004B504F03CFDBDE80440704700005D
:101E0000900B002004ED00E01EF0040F0CBFEFF378
:101E10000880EFF30980816911F8021C0229FFD0C4
:101E200001B504F02BFD01BD43B2002B08DB0122FC
:101E300000F01F0002FA00F0024A5B0942F823009A
:101E4000704700BF00E100E0054B420953F8222033
:101E5000012300F01F0003FA00F01040704700BF9C
:101E600000E100E043B2002B01F10101ACBF03F13E
:101E70006043064B4FEA4111C9B2ABBF03F5614362
:101E800000F00F0083F800131954704714ED00E0C0
:101E900042F8203C009B0B4942F81C3C019B21F07E
:101EA000010142F8183C029B42F8081C42F8143C1D
:101EB0004FF0807342F8043C0023203A02654367E8
:101EC000704700BF8F650100084B9860436E83F335
:101ED0000B88104681F30988002163B681F31188CD
:101EE000BFF36F8F0022002304F051FB900B002002
:101EF000014910220A60704710ED00E072B64040C0
:101F000080F31188BFF36F8FBFF34F8F30BF62B67E
:101F1000BFF36F8F704700BF72B6494081F31188DD
:101F200020BF80F3118862B6704700BF30BFFFF753
:101F3000FDBF00BF0B4A08B50B4B22F07F029A6031
:101F4000BFF34F8FBFF36F8FD3F8882022F4700256
:101F5000C3F8882000F0DCFD01F0E8FB00F0C0F9D8
:101F600000F0FAFD0002010000ED00E001B572B6DC
:101F70000B4A106A00281EBF0021116204F0BCFD4C
:101F800062B6EFF30580A0F110004FEAC0000549EA
:101F9000014409C99847BDE80140034908470000CA
:101FA000900B0020346D010035220100002080F3E9
:101FB0001488BFF36F8F002080F30A8880F30B88AA
:101FC00004F051FB00200E490860BFF34F8F0D480D
:101FD00080F3088800F05EF9202080F311880A4819
:101FE0004FF40061401880F30988EFF31480022158
:101FF000084380F31488BFF36F8FFFF79BFF000047
:1020000094ED00E090260020D0270020EFF3088018
:10201000EFF3098101B5724600F074F801BD00BF0D
:102020000E4B9A6A9A6A9A6A920708D55A6B9A6A0C
:10203000120604D518B19A6A22F080029A62002032
:10204000064B9A6A9A6A9A6AD20658BF9A6A9A6A3C
:1020500042F0FF029A620870704700BF00ED00E096
:102060000D4B9A6A9A6A9A6A920508D59A6B9A6A8F
:10207000120404D518B19A6A22F400429A62002030
:10208000054B9A6A9A6AD20558BF9A6A9A6A42F4CC
:102090007F429A620870704700ED00E0094B9A6A2F
:1020A0009A6A986A9A6A9A6A9A6A9A6A9A6A10F412
:1020B00080106FEA02426FEA124218BF02209A6251
:1020C000704700BF00ED00E00D4B9A695A695A69EC
:1020D000D0070FD45A6991070CD45A69520709D412
:1020E0005A69100706D45A69D10603D45A69920670
:1020F00058BF5A695A6942F0FF025A61704700BFDF
:10210000D0ED00E0F0B5414B0E465B6800258BB08A
:10211000C3F3080385F31188BFF36F8F02F07F418B
:10212000B1F17F4F1CD112F0010118D0540602F01A
:10213000080165D482F00402C2F3800561B1EFF3B7
:1021400089860022033B8DF80720042B49D8DFE85D
:1021500003F0094A4E3F4600EFF38886F1E70D464B
:102160002E46EEE7294BDA6A92073AD4DC6A14F07D
:10217000804408D028331B78EBB101200DF1070112
:10218000FFF74EFF04469DF8073093B920223146F1
:1021900002A804F0E0FB099B6DB3C3F3080222B967
:1021A0006FEA53236FEA43230993204602A904F000
:1021B00063FB0BB0F0BD164B1B782BB101200DF16A
:1021C0000701FFF74DFFDDE7124B1F88BFB217B1C4
:1021D000FFF764FFD6E7104B5C69002CD3D0FFF704
:1021E00073FF0024CFE700200DF10701C8E70020AE
:1021F0000DF10701E5E723F4FF7323F00103D3E7B3
:1022000000299ED1064601259BE700BF00ED00E0B6
:1022100029ED00E02AED00E0D0ED00E0044B5A6922
:1022200042F010025A615A6942F480625A61704762
:1022300000ED00E0044B9968586A884203D00349D6
:102240004FF080520A607047900B002004ED00E0D0
:10225000BFF34F8F0549064BCA6802F4E06213438F
:10226000CB60BFF34F8F00BFFDE700BF00ED00E084
:102270000400FA0500231846054A1168C1F3072136
:102280008B4200D17047936010610133F8E700BFC3
:1022900090ED00E010B572B6002484F31388FFF7C8
:1022A000E9FF0E4A234611464FF0FF3403F12000A8
:1022B0000133102B42F82040F8D100234FF0FF30BB
:1022C00003F160020133102B41F82200F8D162B60D
:1022D000BFF34F8FBFF36F8F10BD00BF00E100E071
:1022E000002320210348C2180133412B82F8001338
:1022F000F9D1704700E100E0064B9B68834207D1AB
:10230000EFF3058323B1044A536843F080535360CD
:1023100001F0BAB9900B002000ED00E082680C4B90
:102320009A60036883F38888436883F38988027B13
:1023300002F00101EFF3948323F00303920748BFF7
:1023400043F0020309B143F0010383F3948870471B
:1023500000ED02E0084AD36848B123F400531B049F
:102360001B0C43F0BF6343F40033D36070479BB250
:1023700043F40053F5E700BF00ED00E0084AD368DE
:1023800040B19BB243F4804343F0BF6343F4003356
:10239000D360704723F480431B041B0CF4E700BF99
:1023A00000ED00E0084AD36840B19BB243F0080357
:1023B00043F0BF6343F40033D360704723F0080356
:1023C0001B041B0CF4E700BF00ED00E0034AD2F849
:1023D0008C3043F44063C2F88C30704700ED00E06D
:1023E000084B1A6818B142F001021A60704722F0D7
:1023F00001021A601A6811B142F00202F5E722F0F8
:102400000202F2E7D0ED00E01FB5094C094A23466D
:102410000121094800F0DCF800230393074B012158
:10242000E41A01A80193029400F0DCF804B010BD96
:102430000000012000000020E870010040010020A1
:1024400010B50B680C7A23F01F0204F01F031A4327
:10245000CB68640923F01F03044943EA440343F0B3
:1024600001038860CA600B6110BD00BF90ED00E001
:102470002DE9F04F8846144606464FF000094A4DB4
:1024800085B0C14505DA7768BFB31F2F05D86FF057
:102490001504204605B0BDE8F08FFB06F7D1D6F84D
:1024A00000A01AF01F0FF2D1504604F0F2F9834653
:1024B00007EB0A00013804F0ECF98345E7D11BF182
:1024C000160FE4D0631E5B45E1DBC5F808B0E96890
:1024D000C5F808B02F6921F01F01D6E900321A446F
:1024E000994247F01F0702F1FF3A1CD1574508D126
:1024F00031465FFA8BF004F0DAF909F101090C3684
:10250000BFE73146C5F808B0EB6822F01F0203F0C0
:102510001F031A43EA60E0B204F0C9F910F1160F84
:10252000B5D0441CE9E7013B5745E0B223F01F0357
:10253000C5F808B006D12A69314602F01F021343DC
:102540002B61E9E7296901F01F010B432B6131463B
:1025500004F0ADF910F1160F99D0C5F808B0EA688B
:102560009DF80830013F62F304038DF808302B69B1
:102570009DF808205B0863F347128DF80820D6E920
:1025800000321344009323F01F033B44441CA3EB8D
:102590000A0AE0B22AF01F030F2803933FF677AF31
:1025A0006946FFF74DFFBCE790ED00E00522034BC5
:1025B0005A60BFF34F8FBFF36F8F704790ED00E00D
:1025C000BFF35F8F0022014B5A60704790ED00E02F
:1025D00010B5034C2278FFF74BFF207010BD00BFF1
:1025E0008C1600202DE9F74F264D8A4606464FF0FF
:1025F0000008AB46244FD0451BDAD6F80490B9F159
:10260000000F39D031680846019104F042F9019970
:10261000044609EB0100013804F03BF984424FF015
:1026200014021A4B08D06FF0150302FB08F84BF8A0
:10263000083003B0BDE8F08F14F1160F2C60F8D00D
:102640001978A142F5DD02FB08B0BC60BC60FC68F3
:1026500000F10801007B64F30400087138690C790B
:10266000400860F347140C71F96821F01F0169609C
:10267000396921F01F01296108F1010814350C3670
:10268000B9E700BFB409002090ED00E08C160020EF
:1026900038B50E4C2568102D14D8FFF791FF002097
:1026A0000B4B0C4A1A63854205D10B4B1D70FFF78B
:1026B0007DFF002038BD616801EB0011FFF7C0FE0F
:1026C0000130F0E74FF0FF30F4E700BFF470010095
:1026D00090ED00E0AAFF44008C1600202DE9F341A4
:1026E0000F4616464FF4806500246FF01500DFF8A2
:1026F0003880A64202D802B0BDE8F081331BB3F5A2
:10270000806F38BF1D46404601AB2A46391901F09B
:102710000FFA019BAB4203D10028ECD12C44E8E72F
:102720006FF01500E7E700BFCC090020002208B5D4
:102730001146044801F0C8F9002818BF6FF01500D1
:1027400008BD00BFCC0900202DE9F0430025214C35
:10275000214E54F8048CDFF8889085B0A84503D842
:10276000002005B0BDE8F083636A96E807001F68A3
:1027700001AB83E807000C221946384604F0C4F880
:1027800090B98FB1636A21691B681A6991420BD1B4
:102790009A69A169914207D8E169914204D96269B5
:1027A0005B6932EA03030AD0276A67B10B4803F07A
:1027B00036FE404080F311884FF0040002DFE368EA
:1027C00001351C44CAE7484603F029FE636A1F60CE
:1027D000F5E700BF3C0401006C6F010018760100B2
:1027E00041760100054B1868043B1B68092B03D197
:1027F000431E584258417047002070473401FF0083
:102800004A4A08B5136843F002031360484B1B683B
:10281000092B01BF4FF050230022C3F81421C3F845
:102820001821FFF7DFFF30B10123424A1360A2F6FF
:102830003822C2F878353E4B1B68092B07D13E4B36
:102840001B68012B1EBF01223C4BC3F87825FFF704
:10285000C9FF10B10E223A4B1A60354B1B68092B89
:1028600004D10022374B1A6001225A600022D300A3
:1028700003F57F03D3F80013013108D0D3F8001318
:102880000132D3F80433B2F5807F0B60EFD12E4BC9
:10289000DA69D1073BD52D4B1946D3F80024012A1C
:1028A000FBD1C3F80425D1F80034012BFBD1264B12
:1028B000DA69D20708D5DA69244922F00102DA611F
:1028C000D1F80024012AFBD11A6A01320AD11A6A0E
:1028D00022F0FF0242F020021A621C4AD2F80034B1
:1028E000012BFBD10022194BC3F80425D3F8002497
:1028F000012AFBD1BFF34F8F1549164BCA6802F46A
:10290000E0621343CB60BFF34F8F00BFFDE71B6A4C
:102910000133C0D00E4AD2F88C3043F44063C2F881
:102920008C300D4B0D4A1A6008BD00BFD0ED00E0A1
:102930003001FF00384A00503401FF0000400050D1
:10294000E4AE03500C4700500080FF00009003509D
:1029500000ED00E00400FA05280000200090D003FC
:10296000044B1A7922B9012218601A710248704783
:1029700002487047880B00200000AD0B0C00AD0B27
:1029800010B1012820D070474FF05022D2F81834EF
:10299000D2F81814C90311D503F00303022B0DD18B
:1029A000C2F8183500220D4B1A601B6802224FF046
:1029B0005023C3F8042301229A6070474FF050233C
:1029C0000122C3F81825EDE70022054B1A601B68A9
:1029D0004FF05023C3F804031860704704510050AF
:1029E0000051005038B510B1012818D038BD4FF053
:1029F00050230222012142F210751C46C3F808231D
:102A0000154A10601268154A1160D4F81834DB03B7
:102A1000ECD5012003F0FDFF013DF6D1E6E74FF0D4
:102A20005024002242F210750D4BC4F808031A60BE
:102A30001B680C4B1860D4F80C34D4F80C2403F049
:102A40000103D203D2D5002BD0D0012003F0E1FF47
:102A5000013DF0D1CAE700BF045100500C500050B6
:102A60000051005004500050164B10B51A6852B176
:102A7000002018601B6801224FF05023C3F8082380
:102A8000114B1B689847114B1A688AB100221A60D3
:102A90001B684FF05023D3F81824D3F8181402F011
:102AA0000302012A4FF0020103D1C3F818159A60FE
:102AB00010BDC3F80813044B0120BDE810401B688B
:102AC000184700BF00510050880B002004510050EF
:102AD0000E4B70B553F82040013053F82060A642E9
:102AE00000D870BDD4E900352846984765B1EB6839
:102AF00030B10028B8BF4042FF28A8BFFF2018709F
:102B00005A7842F001025A700834E8E72471010053
:102B10000248034A0021121A03F048BF4001002076
:102B200090160020012208B5094B02201A70FFF709
:102B3000CFFF04F0D9F80320FFF7CAFF00F024F913
:102B400003F046FC034A137B23F00103137308BD13
:102B50008D160020C00100202DE980483F4BA7B012
:102B600003F5006787F3088883F30A880024E023CD
:102B70003B4D4FF0010B85F82230EC772C766C76CC
:102B8000AC76EC766B6A374E43F4E0236B626B6A8B
:102B9000DFF8E8A043F400236B62AC63EB68DFF876
:102BA000E0809BB243F0BF6343F40833EB60FFF770
:102BB00035FBFFF79DF94FF0FF33AB62EB62FFF798
:102BC00067FDFFF721FC40F20113274DADF82430DB
:102BD00006ABAB60CDE91F4403F028FF2046FFF7AA
:102BE00077FF0120FFF774FF00F0CAFC1F4B6E62F5
:102BF0004FF480521E49059330465346CDE9034BAE
:102C0000CDE90144009400F08FF8737B814623F0F6
:102C100004033046737303F0D5FF0F234FF4A07203
:102C2000CDE902431349144B4046CDE904B4CDE944
:102C3000005400F079F898F80D30524623F0040360
:102C400088F80D3005F1180349463046C5E90633CA
:102C5000C5F80C802C756F60FFF736F9D02700207F
:102C600000ED00E0C0010020900B00207476010010
:102C70009016002090260020452E0100252B0100F3
:102C80004001002070B50E4B0E4CA34201D3002032
:102C900070BDD3E9030141EA000212F003020BD137
:102CA0009D685A61AA4201D11C33EEE75E69013288
:102CB0000E6059610144F5E76FF01500E8E700BFC9
:102CC000EC000020EC000020D3B50C4616461F4651
:102CD0004FF02003EFF3118183F31188BFF36F8F5F
:102CE00043695BB123601B6843618369013383617E
:102CF000002081F31188BFF36F8F11E056EA0702BD
:102D000003D16FF00B002360F3E70246CDE90067C3
:102D1000083000F081FA18B9024B9B685B692360A8
:102D200002B0D0BD900B00202DE9FF410E9E00F1B6
:102D3000580506730426C0E9165500250446467357
:102D40000D9EC0E906558673D61D0C9A26F007061F
:102D5000C0E919168560C573C56602920B9A01EB2E
:102D6000060801920A9A00924246FFF791F8054B35
:102D700065659B6803B11B6F4046236704B0BDE8DF
:102D8000F08100BF900B00202DE9F0472A4E2B4D1B
:102D9000B04686B0B54205F1300410D300F0CAF950
:102DA0004FF4004940F2E7360027244CDFF890A0AA
:102DB000444521D306B0BDE8F04700F0ADBA54F861
:102DC000043C059354F8103C049354F8143C0393CA
:102DD00054F8183C029354F81C3C019354F8203CDE
:102DE000009354E90A2354E90C01FFF79DFF54F8BE
:102DF000303C5D652546CDE7636A5A1C0DD03046F0
:102E0000394623EAE373C9FB0301B94208BFB04264
:102E1000256804D1284600F04DFB3034C8E74FF454
:102E20007A720023FDF70AFB02460B4605F11800F3
:102E3000514600F0E5FCF0E7EC000020EC0000203B
:102E4000E56B010008B5094C4FF02002EFF3118348
:102E500082F31188BFF36F8F03F014FF2062FEF737
:102E6000CDF90028F0D1FFF749F8EDE7900B0020ED
:102E70002DE9F341044616461F464FF02003EFF3B9
:102E8000118883F31188BFF36F8FC368324A6BB127
:102E900080689168884219D056EA070318D188F3F0
:102EA0001188BFF36F8F6FF00F000CE0916891F9FC
:102EB0000E100133E36093682161A36088F31188E9
:102EC000BFF36F8F002002B0BDE8F0812169F0E709
:102ED00090F90E3091F90E109942A8BF194621EAD7
:102EE000E1718B422CDD00F003FB05462246414692
:102EF000CDE90067194800F08FF90028E3D04FF0C2
:102F00002003EFF3118683F31188BFF36F8F2368DB
:102F100021699C4207D033B193F90E309942A8BF82
:102F2000194621EAE171A06890F90E30994209D161
:102F30006DB13146094800F0EBF86FF00A00C2E7C6
:102F40000025D3E700F0D4FA0028F2D1F0E786F3A9
:102F50001188BFF36F8FF0E7900B00208E160020D2
:102F600038B583680446002B36D01E4A92689342D7
:102F700035D1DA7B013ADA73C368012B05D0013B06
:102F8000C36000F0C9F9002038BD4FF02003EFF313
:102F9000118583F31188BFF36F8F0169806890F901
:102FA0000E30994201D000F0A3FA204603F03CFE17
:102FB000A06058B190F90E2022610022826703F0D0
:102FC00001FE2946084800F0A3F8DAE7E06085F33F
:102FD0001188BFF36F8FD4E76FF01500D4E74FF07F
:102FE000FF30D1E7900B00208E16002038B5044644
:102FF0004FF02003EFF3118583F31188BFF36F8F38
:1030000003F012FE48B10022826703F0DBFD29467F
:10301000BDE83840044800F07BB8D4E902329A4257
:1030200018BF0133A360F2E78E16002037B51446AF
:103030001D464FF02003EFF3118183F31188BFF396
:103040006F8F836843B1013B836081F31188BFF3C5
:103050006F8F002003B030BD54EA050306D181F321
:103060001188BFF36F8F6FF00F00F3E70246CDE9D1
:103070000045024800F0D0F8ECE700BF8E160020B3
:1030800010B5084C23685BB1FEF75CFB0346206873
:10309000054A03440021BDE81040136103F002BE5D
:1030A00010BD00BFC80B0020900B0020F8B50446EF
:1030B0000D464FF02003EFF3118683F31188BFF321
:1030C0006F8F00224FF4004740F2E73000210D4B94
:1030D000E7FB04011A6100234FF47A72FDF7AEF9A1
:1030E000002C094B09DC1860084B1D60FFF7C8FF76
:1030F00086F31188BFF36F8FF8BD0228B8BF022096
:10310000F1E700BF900B0020C80B0020C40B00208B
:1031100049B9EFF3058030B9054B5A6A9B689A426A
:1031200001D0FEF72BBE81F31188BFF36F8F70477C
:10313000900B00204FF02003EFF3118183F31188EF
:10314000BFF36F8F044B9A68D37B013BD37381F33A
:103150001188BFF36F8F7047900B002038B502467F
:103160000C4803F0FFFC0C4D044600B9EC68AB685A
:103170004AB95A7BD20606D1A26922B9DA897F2AD6
:1031800001D96B6238BD9C4201D0FFF779FF6C62B8
:10319000F8E700BFB80B0020900B002008B590F9AD
:1031A0000D200146002A437B04DA03F07F034373BA
:1031B00003F0B0FC044B9868431A58425841BDE8EC
:1031C0000840FFF7CBBF00BF900B00202DE9F04176
:1031D000064614461D464FF02003EFF3118783F394
:1031E0001188BFF36F8F03F0C3FC87F31188BFF31F
:1031F0006F8F6B1C08BFB4F1FF3F08D022462B46EF
:1032000006F118000349BDE8F04100F0F9BABDE845
:10321000F08100BFE56B010010B50C46064B11466E
:103220009868064B1860DDE90223FFF7CFFF2046C0
:10323000BDE81040FEF7A2BD900B0020C00B00209F
:103240002DE9F04105460F4603F046FD04464FF0D8
:103250002003EFF3118883F31188BFF36F8F124EB1
:10326000124BB0682C441860FFF798FFB068104903
:103270002A463B46183000F0C3FAB2684046537BFA
:10328000002543F010035373FEF778FD03F024FD8F
:10329000241A65F10005002C75F10003B8BF002465
:1032A0002046BDE8F08100BF900B0020C00B00203D
:1032B000E56B010070B50446183003F0CDFC4FF00B
:1032C0002003EFF3118683F31188BFF36F8F94F916
:1032D0000D20637B002A05DA03F07F032046637329
:1032E00003F018FC0B4D637BA86843F01003637375
:1032F000031B58425841FFF731FF86F31188BFF393
:103300006F8FAB68A34203D1BDE8704003F020BCCF
:1033100070BD00BF900B002010B54FF02003EFF3FD
:10332000118483F31188BFF36F8F084B00209A68D4
:10333000D37B0133D373FFF711FF84F31188BFF3FD
:103340006F8FBDE8104003F003BC00BF900B00205E
:1033500070B590F90D200146002A437B04DA03F092
:103360007F03437303F0D6FB4B7B154A63F07F0367
:103370004B7302F12800D2E90A3583421BD0D3B146
:1033800091F90E6093F90E40A6420FD0A41B002CB9
:103390000CDD5868C1E90030016059609068BDE8F3
:1033A0007040431A58425841FFF7D8BEAB4202D092
:1033B0001B68002BE6D1C1E900052960D162EDE769
:1033C000900B0020014670B54FF02003EFF31184FD
:1033D00083F31188BFF36F8F164B174A98681568EF
:1033E000A8421D4606D1FFF74BFE84F31188BFF3B8
:1033F0006F8F70BD00261660104A1268BAB1C2897C
:103400007F2A14D8427BD20611D10D4A90F90E6062
:10341000126896420BDB0B4A904208D01A698A4226
:1034200002DCFFF795FFDEE7521A1A61DDE70023A1
:103430002B61DAE7900B0020C00B0020C80B0020A6
:10344000C40B00204001002070B490F90D20437B94
:10345000002A2ADBDA0628D1826932BB144A63F0DB
:103460007F03437302F12801D2E90A358B4217D05A
:10347000B3B190F90E6093F90E40A6420BD0A41B95
:10348000002C08DD5A68C0E9003210605860002046
:1034900070BCFFF763BEAB4202D01B68002BEAD1C1
:1034A000C0E900152860D062F1E770BC704700BF2A
:1034B000900B002010B54FF02002EFF3118482F33F
:1034C0001188BFF36F8F427B510704D484F31188B6
:1034D000BFF36F8F10BD22F004024273FFF7B4FFF9
:1034E0002146BDE810400148FFF712BE8E160020AD
:1034F000F8B504464FF02003EFF3118583F31188EC
:10350000BFF36F8F437B49B2DA0633D182698ABB3E
:1035100003F07F03437303F0FDFA437B174A63F024
:103520007F0343738173104650F8283F83421BD0BA
:10353000D3B1D76A93F90E60B14210D0761A002E3B
:103540000DDD5A68C4E9003214605C600120FFF7A9
:1035500005FE012085F31188BFF36F8FF8BDBB42D4
:1035600002D01B68002BE5D1D36AC4E900031C60BC
:10357000D462EBE70020A173ECE700BF900B0020C2
:103580000021044B084603F12802C3E90A22FFF791
:103590008DBD00BF900B00202549F8B58A68254BEA
:1035A0009A423BD04FF02003EFF3118583F311884B
:1035B000BFF36F8F8868437B03F07F03437303F08F
:1035C000A9FA08468B685A7B62F07F025A7350F85A
:1035D000282F82421CD0DAB1CF6A93F90E6092F99B
:1035E0000E40A6420FD0A41B002C0CDD5168C3E98D
:1035F00000210B6053600120FFF7B0FD2846BDE8B5
:10360000F840FEF7BBBBBA4202D01268002AE6D1EE
:10361000CA6AC3E900021360CB62ECE74FF02003F3
:10362000EFF3118083F31188BFF36F8FE7E700BFDB
:10363000900B002040010020B1F1FF3F08BFB0F126
:10364000FF3F08B502460B4606D10B4B9868FFF7C3
:1036500031FE4FF0FF3008BD13430AD1FFF79CFF46
:1036600000204FF47A7380FB0323D00B40EA4340E1
:10367000F1E7FFF7E5FDF4E7900B0020014B9868B8
:10368000704700BF900B00202DE9F04104464FF039
:103690002003EFF3118683F31188BFF36F8F437B11
:1036A0001A0705D586F31188BFF36F8FBDE8F08147
:1036B00023F0200242F00801D20920D14173A3680F
:1036C00013B1204603F02EFA04F1180003F0C4FAF7
:1036D0004FF0000804F15807A56DBD4200D0B5B900
:1036E0000120FFF73BFD104B9B68A342DAD1EFF3BB
:1036F0000583002BD6D13046FEF740FBD2E703F01E
:103700005F0343F00803437303F004FAD7E7284646
:1037100003F008FA05F1180003F09EFA2846C5F8F0
:103720007880FFF791FED7E7900B002008B5064898
:10373000064A0749121A03F00EF9BDE80840054A87
:103740000549064803F007B9000000203C010020AD
:10375000807601000000000080760100000000205B
:10376000034B1B680BB9FDF7EDBF0020704700BF8E
:10377000CC0B002030B5036868B10A4A5268904209
:1037800009D043B1D3E90421D0E90445121945EB2E
:103790000101C3E90421426813605A600023C0E9B3
:1037A000003330BD2C00002038B5134B1C689C4200
:1037B00008BF0024FFF7D4FF0546BCB1D4E90401DB
:1037C000401B61EBE571012871F1000311DB6FF023
:1037D00000420023824273EB010400DA1046074BDB
:1037E0001B6913B19842A8BF184638BD6FF000405E
:1037F000F5E70020F3E700BF2C000020900B00202D
:10380000B3F1FF3F08BFB2F1FF3F2DE9F74F044688
:1038100092469B4673D081604FF02003EFF31185F1
:1038200083F31188BFF36F8F6FF001034FF0FF3206
:10383000B3EB0A0862EB0B09B8F1000F79F1000154
:103840001CDB3048D0E900105B1A62EB0002B3EBDE
:103850000A0662EB0B07012E77F10003BCBF0126BD
:103860000027C4E90467284AD2E9003C93421ED1EC
:10387000C4E9002CCCF8004054602DE0FFF770FF45
:103880001AF1010300934BF100030193DDE90023DA
:10389000121843EBE073C4E90423E4E7B6EB080035
:1038A00067EB09016345C4E90401E1D01B68002B03
:1038B000DED0D3E90489D4E90467464577EB0901F2
:1038C000ECDAB8EB060069EB0701C3E904015968BB
:1038D000C4E900310C605C60136893420BD09C42D9
:1038E00009D1FFF761FF18B1084B1B69834202D071
:1038F0000021FDF7F5FE85F31188BFF36F8F03B04C
:10390000BDE8F08F400200202C000020900B00202A
:103910002DE9F74F0646FFF755FD4FF02003EFF373
:10392000118483F31188BFF36F8FDFF8B0A02A4DA5
:103930005146DFF8ACB02E60D5F800C0DBF80000CF
:103940006246DAE90089D3175845CDE900230DD046
:1039500060B1D0E90467B445BB411DDA009BB6EB0A
:10396000030C019B67EB0306C0E904C60026009B1D
:103970002E6013EB0802019B43EB0903C1E900230E
:10398000FFF712FF3146FDF7ABFE84F31188BFF35A
:103990006F8F03B0BDE8F08F0022002318EB0608FC
:1039A00049EBE679C0E90423ACEB0606CAE90089D5
:1039B0002E60FFF7DFFE84F31188BFF36F8F8368FB
:1039C00098474FF02003EFF3118483F31188BFF37E
:1039D0006F8F0249B0E700BFCC0B002040020020EF
:1039E0002C00002010B54FF02003EFF3118483F377
:1039F0001188BFF36F8FFDF7A5FE064BD3E90023B7
:103A0000121843F1000384F31188BFF36F8F10463F
:103A1000194610BD4002002010B50C4C236813B1AC
:103A20000B4B1B682BB900F099FA30B90122084BF7
:103A30001A6001230020236010BD0138062801D937
:103A4000044810BD044B53F8200010BDD00B0020DB
:103A5000D40B0020FE8FFFFF3C710100BFF34F8F9E
:103A60000549064BCA6802F4E0621343CB60BFF31A
:103A70004F8F00BFFDE700BF00ED00E00400FA0536
:103A80004FF0FE33002130B4064A074D074C2B603F
:103A900013602360064A074CEB606368C2F80015A8
:103AA00030BC184704148450001484500814845007
:103AB0000000845034000020024BD0E90012C3E91A
:103AC00000127047340000202DE9F043154CDFF858
:103AD0005C80002818BF0446206883B040451DD094
:103AE00016460D4620464FF4DE7104F1040900F03D
:103AF00079FE04F58C77484600F01CF9384601F051
:103B000047FA4A4638462B460749009601F052FAD2
:103B100008B9C4F8008003B0BDE8F083002003B00A
:103B2000BDE8F083D80B0020B53D0100A5BCC95A03
:103B3000F0B50D4C0D4E002808BF2046076883B035
:103B4000B7420ED100261D4600F58C703346009614
:103B5000144601F07FFA002818BF34462C6003B0E9
:103B6000F0BD0348FBE700BFD80B0020A5BCC95A35
:103B7000E88FFFFF48B143682BB1BFF35F8F00238D
:103B8000036018467047024870476FF4E040704782
:103B9000EA8FFFFF10B5044628B1636813B1002314
:103BA0002360636010BD024B02485B689847F4E7EE
:103BB000340000205871010010B5044630B10022D5
:103BC0006368226043F00103636010BD0148FFF7A2
:103BD00057FFF4E78071010080B1436863B10122AF
:103BE000D0E8EF3FC0E8E12F0029F9D1012BF7D051
:103BF000BFF35F8F00207047024870476FF4E040CA
:103C0000704700BFEA8FFFFF70B40B4B0668C268B5
:103C1000D0E90154C3E90242C3E90065D1E90302D6
:103C20000E68064BD1E90154C3E90065C3E90240BF
:103C30001A6170BC704700BF44000020540000208F
:103C40002DE9F043202B1D460646894690468BB051
:103C500026D8DBB202AF31688DF804908DF80530BC
:103C600006F1040921B9484600F062FE044640B955
:103C7000012302224846336001A900F06DFE04468C
:103C800038B13846202100F0ADFD20460BB0BDE82C
:103C9000F0832A464146484600F05EFE0446F0E7BF
:103CA00002AF1946104600233A4601F0ADFA044629
:103CB0000028E6D12023B8461D46CCE7F0B5D0F861
:103CC000F430A7B0002BD8BF02AE2CDD0546002390
:103CD000D0F8084102AE0193A4F101073146D5F8AE
:103CE000F8409022D0F8FC0001ABB7FA87F7A04764
:103CF0007F09044610B9019B3BB9A7B1304690211A
:103D000000F070FD204627B0F0BD0146324628463F
:103D1000FFF796FF50B9D5F80031019A1344C5F862
:103D20000031002FEAD16FF03C04E7E7044620465B
:103D300027B0F0BD70B50025044629461422C0F80E
:103D4000F450F83002F032FE164B04F586761B680C
:103D500030469847204640F8045B00F0CFFD124BF8
:103D600030461B689847D8B9D4F8F430AB4211DC20
:103D70000121202503EB830204EB8202C2F8FC0040
:103D80000A480B44C2F80451C2F8F800C2F80811FE
:103D9000C4F8F430064B3046BDE870401B68184745
:103DA00070BD00BF980000209C000020F947010072
:103DB000A00000202DE9F047202A88B078D83E4B9B
:103DC00000F5867904461B6848461746884698479A
:103DD000054640BB40F20116D4F8F430002B63D006
:103DE0002046FFF76BFF054600285FD1D4F8F4307A
:103DF000002B07DDD4E94002904203D3D4F8082118
:103E0000012A14D0013EE9D16FF03B056E463046E1
:103E1000202100F0E7FC294B48461B689847002802
:103E200018BF6FF01D05284608B0BDE8F0871F28B1
:103E3000E8D96E4629462022304604F1040A02F0F1
:103E4000B5FD3146504600F08FFD05460028DED115
:103E5000504600F067FD504600F050FD29465046A0
:103E600000F066FD05460028D1D15046202231469B
:103E700000F072FD05460028C9D1034632462021D4
:103E8000304601F0C1F905460028C0D1D4F8F4301D
:103E90003A46002BC8BF002340463146C8BFC4F88D
:103EA000003102F058FDB2E76FF03F056E46AEE715
:103EB0006FF03B05B7E700BF9C000020A00000208A
:103EC000002130B58DB0282202A8019102F06EFDCC
:103ED00002A801F0C1F9044610B120460DB030BD72
:103EE000184D4FF0FF31286800F03AF90446C0B988
:103EF000002000F065F900BB134A02A901A800F0F8
:103F000063FC0446012000F05BF990B9286800F0DA
:103F10002FF90028E1D00D48FFF7B2FD20460DB083
:103F200030BD0B48FFF7ACFD012C08BF0524EDD0D8
:103F3000DEE70848FFF7A4FDE8E70748FFF7A0FD24
:103F4000DAE700BF940000200C0E0020FC71010095
:103F5000A4710100DC710100BC71010010B582B0D8
:103F600000F054F828B100F0A3F80324204602B072
:103F700010BD00F06FF8D0B900F022F9D8B91E4B8F
:103F80001B681B0EF02B0AD11C4A1D4B12689A426B
:103F900029D000F03DF8072400F08AF8E6E706246F
:103FA00000F036F800F084F8204602B010BD04247A
:103FB000204602B010BD00F02BF800F079F8FFF7B2
:103FC0007FFF044658B902460146FFF77DFD30B930
:103FD00068220C4901ABFFF7ABFD0028C6D00524D1
:103FE000204602B010BD012000F0EAF80028E2D11E
:103FF000054B1860E3E700BF28198450241A845049
:104000000000E020A40D00200C1A8450002070470E
:1040100000207047430503D54FF0FF32024B1A6072
:10402000024B1860704700BF08118450081A845072
:10403000014B1860704700BF041A845008B100F0AB
:104040006DB84FF47500704708B100F04FB84FF4E9
:104050007500704710B5114800F06EF800B110BD42
:104060000F4800F069F80028F9D10E4C204600F006
:1040700063F80028F3D10C4B0C481C6000F05CF88E
:1040800001460028EBD100F02DF8044608B1204687
:1040900010BD00F077F82046FAE700BF900000203E
:1040A000840000208C000020940000208800002064
:1040B00008B5084800F04AF8074800F047F80748F4
:1040C00000F044F8064800F041F8BDE8084000F070
:1040D0000BB800BF90000020840000208C0000205E
:1040E0008800002000207047704700BF0246074844
:1040F00003681342FCD021B1054B06481B680B60D6
:104100000360054B00201A60704700BF001A8450FE
:104110000411845008118450081A8450024604493E
:104120000B681A42FCD0034B00201A60704700BF96
:10413000001A8450081A845008B5034B02681B68A3
:1041400010689847002008BD4400002008B5034BC4
:1041500002685B6810689847002008BD4400002092
:10416000024B02689B681068184700BF440000209B
:1041700008B5034B0268DB6810689847002008BD4B
:104180004400002070B5094C094D2069AB68984780
:1041900018B1084B08485B6898470021074AEB684C
:1041A00011602069BDE87040184700BF540000202E
:1041B0004400002034000020147201002C10002064
:1041C00070B51A4D1A4E0446B26828699047F0B986
:1041D0005CB1184C2368ABB1012B1AD0013B2360B2
:1041E0002869F3689847002070BD124C216839B9DE
:1041F0000120114B114AC3F800051368002BFCD1B4
:1042000001312160F36828699847002070BD0C488F
:1042100070BD0A4A1368002BFCD1074A6FF07E403C
:10422000C2F80035FFF704FF2368D7E754000020E9
:10423000440000202C1000200000845010198450ED
:10424000E98FFFFF014B1B68184700BF44000020A7
:10425000014B9B68184700BF44000020014BDB68FE
:10426000184700BF440000202DE9F843002878D00B
:104270000C46002975D01D46002B72D006461AB197
:10428000012200232A6003602B68002B65D0294699
:10429000204601F0DDF8074600285FD12146286856
:1042A00001F0B8F80746002858D12B68082B67D0D2
:1042B000042B68D0A3F10208B8FA88F84FEA58181E
:1042C00001239C46314A3249136010460B60943AF0
:1042D000C0F800C0636A136011688B42F8D14FF0D8
:1042E00000092C4B4FF0FF30C3F80090FFF792FE0F
:1042F0006FF01B02284B48461A60FFF799FE274AC9
:10430000274BC2F80080186840F48060FFF790FEE9
:104310000A22244B1A60089A2369012A616A24D070
:10432000214AA2FB03231B09012203FB01F303EB38
:1043300043031E49DB039B090B60164B38461A608A
:1043400033682A6823F07F4343EA026333602A68B4
:1043500043EA02233360BDE8F883154F3846BDE8D1
:10436000F883144F3846BDE8F8834FF47F03D3F841
:104370000C2C013202D0D3F80C3CD1E71623D3E742
:104380004FF003089CE74FF0020899E7C4118450EE
:10439000401184502C118450001184500C11845011
:1043A000041A845038118450ABAAAAAAD811845098
:1043B000310CF100350CF100F0B40024C9002646A0
:1043C000274601F1FF3C06E09F4215D001266545D6
:1043D00018D82C461F46630950F8233004F01F01FB
:1043E000CB401F2904F1010518BF03F00103002C85
:1043F000EAD101263546ECE701369642E7D103487B
:10440000F0BC70470020F0BC704700BF360CF100D4
:1044100000285FD02DE9F0414C1EB4F5047F26D270
:104420002BB322B3CC00012B04F1FF3E2FD000218F
:104430008C460F460D4603F1FF384C0950F82440D6
:1044400001F01F06F4401F2E18BF04F0010421B92B
:104450000125AC4629462746EFE7AB4213D0A742D9
:1044600001D10CF1010C454504D1624502D21A4834
:10447000BDE8F0813C4601318E4505F10105EAD2E7
:104480000020BDE8F08100254FF0010CF3E7002685
:10449000B446374631464B0950F8233001F01F052A
:1044A000EB401F2D18BF03F0010339B15FB99C45E4
:1044B00001D0634608E06346013605E00126314637
:1044C0009C460127E7E73E46B242D0D30131A142E4
:1044D000F6D1D5E700487047370CF1002DE9F04FD1
:1044E0008DB0189E07460C46179D002E4CD1D1F872
:1044F00010B000211D60169B1960002A00F0228177
:104500009C4A9D4B1168626A1B689A4247D10A29EE
:1045100045D1FB7804930423B8460293974BA3FB41
:104520000B234FEA930A0AEB4A0305F108020392B0
:10453000ABEB430A169BC3F800B0BBF1000F00F0D1
:10454000C7805D464FF00009039E00F091FF0023F5
:104550000593B8F1000F00F0E980002C00F0E68030
:10456000049B002B00F0E080204604A900F070FFBF
:10457000B8B1834B984240F0AB80029000F078FFD6
:1045800002980DB0BDE8F08F4FF47F01D1F80C0C0C
:1045900001300CBF4FF4047BD1F80CBCA9E779487B
:1045A000EBE72146049800F035FF0028E1D1049F95
:1045B000082F00F0BD80042F00F0BC80A7F1020797
:1045C000B7FA87F77F09012319466F48036040F85F
:1045D000843C6D4B68481960636A036000688342DD
:1045E000F7D10023694A4FF0FF301360FFF712FD47
:1045F00000236FF01B011846654B1960FFF718FD8B
:104600006449654B0F6018685C4F40F48060FFF7A9
:104610000FFD0A210122574B604819602169636A26
:10462000A7FB01C1090903FB01F303EB4303DB0310
:104630009B090360554B05A81A600499D8F800201F
:104640000B0243EA016322F07F421343C8F80030B3
:1046500000F0D0FE059B03F01A03034338D1504B02
:10466000A7FB05271A681433069253F8102CB9EBF0
:10467000970F079253F80C2C089253F8082C0992C4
:1046800053F8042C0A921B680B9302D1BAF1000F65
:1046900041D1182230460DEB020100F01BFE183DFF
:1046A000183609F10109002D7FF44FAFBBF5047FE7
:1046B0005DD8039D594628466269FFF77DFE0028B4
:1046C0004BD00023169A13602D4B98423FF455AF00
:1046D000049D082D34D0002204AB214640466D00D5
:1046E00000920495FFF7C0FD2E4B984224D000287D
:1046F0007FF443AFD8F80020130A03F47F03134379
:1047000023F07F43C8F80030029B013B02937FF403
:1047100011AF002031E73046524606A900F0DAFD1D
:10472000A5EB0A055644BCE71E4822E71E4820E7D1
:10473000032748E7022746E7236A002B3FF41DAF13
:104740001A481AE7012221463846009604ABFFF7C3
:104750008BFD00283FF4DFAE0FE74FF4806359462E
:104760002846A269FFF754FE0028AAD1D1E7169B7C
:104770001D60ADE73811845030118450ABAAAAAA4D
:10478000020CF100300CF100C41184502C11845043
:10479000001184500C118450041A8450D811845094
:1047A00014118450310CF100350CF100320CF10081
:1047B000002330B4DDE903450493029BCDE90245B3
:1047C00030BCFFF78BBE00BF10B5012486B005AB2F
:1047D000CDE901240093002204ABFFF77FFE06B071
:1047E00010BD00BF38B131B1002201440346013091
:1047F00081421A70FAD170472DE9F04188B00592D4
:10480000002968D01C46002B65D01546002A62D0CE
:10481000DFF8E4800E46D8F800004FF0FF31FFF7D4
:104820009FFC00284CD10020FFF7CAFC002843D190
:104830002A4800F011FDE8B101204FF0FF37FFF7E3
:10484000BFFC002834D14FF408712548FFF7CAFF98
:1048500004212448FFF7C6FF20482821FFF7C2FFA4
:10486000D8F80000FFF784FC00282DD1384608B0A6
:10487000BDE8F0811A4907AB02460390029100930C
:1048800016491848019405ABFFF792FF0028D3D1D1
:104890002368AB42D0D3079907462A4630460831F1
:1048A00000F018FD01202560FFF78AFC0028CAD01F
:1048B0000D48FFF7E5F8C6E70C48FFF7E1F8B7E762
:1048C0000B48FFF7DDF8AEE70A48FFF7D9F838469E
:1048D00008B0BDE8F0814FF0FF37C7E75412002061
:1048E0003410002030100020DC710100BC71010088
:1048F000A4710100347201009400002010B5044638
:1049000028B12046BDE81040F02100F0E7BC044883
:10491000FFF7B6F82046BDE81040F02100F0DEBCFD
:104920004C72010010B1F021FFF75CBF704700BF6F
:1049300008B561B1012907D1022100F039F800283A
:1049400018BF6FF0360008BD6FF0360008BD0121BA
:1049500000F02EF8F3E700BF08B500F06BF8002870
:1049600018BF6FF0360008BD70B5E8B10E46D9B17A
:10497000044600F031F80546B0B92368012B0BD08E
:10498000022B01D0284670BD30461C2204F10801DC
:1049900000F0A0FC284670BD3046202204F108013A
:1049A00000F098FC284670BD6FF03605EAE700BFBE
:1049B00078B138B50D46F021044600F08FFC402355
:1049C00020462560E36500F099FD003818BF0120FE
:1049D00038BD0120704700BF70B5056EA4B0044615
:1049E00004AEE5B901220023626030462946CDE9D4
:1049F000003302AA00F04AFD10B1012024B070BDBE
:104A00002A46204602A900F0A3FD0028F5D1204641
:104A100000F0C8FE0028F0D1206624B070BD802DC3
:104A20002A46304628BF802204F1640100F052FC7F
:104A3000256ED7E7002855D0F0B51546A5B0B2B120
:104A40000E4651B30446D0E917301A1AB2FBF3F7F9
:104A500003FB1727AF4228BF2F46002F44D18342C4
:104A600008D0B5FBF3F703FB07F7CFB96DBB2846BA
:104A700025B0F0BD802B28BF802304F164011A46C5
:104A800004A800F027FC0023CDE9003304A8E16D61
:104A900002AA00F0FBFC002833D0012025B0F0BDB5
:104AA000002339463046CDE9003302AA00F0EEFC7F
:104AB0000028F2D13A46204602A900F049FD00281C
:104AC000EBD1ED1B3E44002DD1D0206E2A4619308B
:104AD000314604EB800000F0FDFB226E00202A44EA
:104AE0002266C5E70120704704F1640318443A4682
:104AF00000F0F0FBD4E9173038443E44ED1B20664B
:104B0000ADE72046E26D02A900F022FD0028C4D1E5
:104B1000E36D2066A5E700BF2DE9F04120220446A1
:104B200088B00D4668460021A6186F4601F03EFF8A
:104B3000E27B0132D2B2E273002A4DD1A27B013274
:104B4000D2B2A273002A47D1637B0133DBB2637315
:104B5000002B41D1237B0133DBB22373002B3BD1EC
:104B6000E37A0133DBB2E372002B35D1A37A013350
:104B7000DBB2A372002B2FD1637A0133DBB26372F5
:104B800053BB237A0133DBB223722BBBE3790133AE
:104B9000DBB2E37103BBA3790133DBB2A371DBB9F1
:104BA00063790133DBB26371B3B923790133DBB2CB
:104BB00023718BB9E3780133DBB2E37063B9A37877
:104BC0000133DBB2A3703BB963780133DBB26370AE
:104BD00013B92378013323703B4622460121304626
:104BE00000F050FE804600282AD1103708AB9F42C3
:104BF0009ED100992B686A684B40019930464A4023
:104C0000AE68029900937140EB68039E0192734075
:104C10002A69049E0291564005996A69039351409E
:104C2000D5E90623069D05915540079A69465340EC
:104C30008022CDE90653049600F00AFE804638B182
:104C400068462021FFF7CEFD404608B0BDE8F08160
:104C5000102220460DEB020101F07DFEF0E700BFBF
:104C60002DE9F04F06468069AFB0B0F5C07F00F285
:104C70007C811D46C0F5C073AB42C0F07681C5F59E
:104C8000C073181A90421746C0F06F81DFF8E8929F
:104C90004FF4C07288464846002101F087FE49461D
:104CA000D6F89430B269D6F898009847002840F0BA
:104CB0005F81B46955B12A464946D6F89430D6F892
:104CC00098009847002840F053812C44B8F1000F19
:104CD00002D0002F40F02281B4F5C07F88BF6FF072
:104CE000370500F21281DFF8A4824FF4D072002160
:104CF000404601F05BFE11A800F094FD2023002146
:104D000065BA2246A8F81010A8F812509A4988F8F7
:104D1000173008F1180001F01EFE8022974B984DC5
:104D2000984908EB0400CDE902510276019311A8DD
:104D300003F10C3301A9049300F08AFD0546002815
:104D400040F0F48004F119070DF114090DF1240B62
:104D500010220021484601F029FEBA468A4C9DF8EF
:104D6000142014F8103C9DF815C014F80F1C9DF881
:104D70001600534014F80E2C8CEA010C50409DF89C
:104D8000171014F80D2C9DF818E0514014F80C2C55
:104D90008DF814308EEA020214F80B3C9DF819E0ED
:104DA0008DF815C08EEA030314F80ACC9DF81AE0BA
:104DB0008DF816008EEA0C0C14F8090C9DF81BE017
:104DC0008DF817108EEA000014F8081C9DF81CE0FE
:104DD0008DF818208EEA010114F8072C9DF81DE0CB
:104DE0008DF819308EEA02029DF81E3014F806EC98
:104DF0008DF81AC083EA0E038DF81B008DF81C1085
:104E00008DF81D208DF81E309DF81F1014F8053CFC
:104E10009DF820C09DF821004B4014F8042C14F894
:104E2000031C8CEA020241409DF822C014F8020CD7
:104E30009DF823E08CEA000014F801CC8DF81F30B7
:104E40008EEA0C0C8DF820208DF821108DF82200B0
:104E50004B464A46012111A88DF823C000F012FDEF
:104E6000BAF1100F94BFAAEB0A0AAAF1100A00289F
:104E700079D11034BAF1000F7FF471AF0BEB05005C
:104E80001022494601F067FD98F8033010350133D0
:104E9000202D88F803307FF45BAF8022594611A89B
:104EA00000F0D6FC0546002844D1334C04F120071D
:104EB0000DAB1A46012111A800F0E4FC05460028BC
:104EC00038D1102220460DA9144401F044FDBC4203
:104ED000EED111A800F0B6FC4FF4D0712B48FFF7CB
:104EE00081FC58462021FFF77DFC102101A8FFF727
:104EF00079FC48461021FFF775FC30461E49FFF744
:104F00000BFE054608B9012333614FF4C0711A48FE
:104F1000FFF768FC28462FB0BDE8F08F09EB0400CE
:104F200041463A4601F017FD3C44D5E60DF114091F
:104F30000DF1240B11A800F085FC4FF4D07113483B
:104F4000FFF750FC58462021FFF74CFC01A8102128
:104F5000FFF748FC48461021FFF744FC2021064893
:104F6000FFF740FCD1E70546E4E76FF03705D1E7EE
:104F70006FF03305CEE700BF1C14002000010203D0
:104F80000405060708090A0B8C1200207C12002079
:104F900010B5A4220021044601F008FD4FF0FF32B5
:104FA000034B226104F19C001B68BDE810401847C8
:104FB000980000202DE9F04104460E46154684B0C5
:104FC0001022002100F1200868461F4601F0EEFC87
:104FD000404600F027FCA269C4E92565D2B9202229
:104FE0002669A261002E2FDB4FF6F073694640461A
:104FF0008022E36100F02CFC054638B9134B04F124
:105000009C0840461B689847054658B1284604B09E
:10501000BDE8F0812669002EE6DA172A14D801329D
:105020005608E1E7334639460A9A2046FFF718FE4C
:10503000074B05461B6840469847002818BF0546A1
:10504000284604B0BDE8F0810026CDE79C00002092
:10505000A00000202DE9F047B2F5806F8CB0149FBE
:1050600000F2CB80B7F5807F00F2C480044615467D
:105070000E462022002104A8984601F097FC2169E1
:10508000E269914200F387806369002B40F08380DE
:10509000002F40F0A7806F46002D00F098806F46EB
:1050A00004F120080EE0102DA94628BF4FF010098A
:1050B000304639464A4601F04EFCB5EB09054E44F0
:1050C00000F08580E37B0133DBB2E373002B4DD12D
:1050D000A37B0133DBB2A373002B47D1637B013386
:1050E000DBB26373002B41D1237B0133DBB223732B
:1050F000002B3BD1E37A0133DBB2E372002B35D1D5
:10510000A37A0133DBB2A372002B2FD1637A013370
:10511000DBB2637253BB237A0133DBB223722BBB46
:10512000E3790133DBB2E37103BBA3790133DBB273
:10513000A371DBB963790133DBB26371B3B923794E
:105140000133DBB223718BB9E3780133DBB2E37057
:1051500063B9A3780133DBB2A3703BB96378013341
:10516000DBB2637013B92378013323703B462246C8
:105170000121404600F086FB8146002893D0202183
:1051800004A8FFF72FFB38461021FFF72BFB4846FA
:105190000CB0BDE8F0871A4B04F19C0A50461B681E
:1051A000984781460028F2D103463A4641462046B8
:1051B000FFF756FD134B07461B685046984781463C
:1051C0000028E4D1002F3FF466AFB946DFE7204660
:1051D00004A9FFF7A1FC81460028D0D1236901333F
:1051E0002361CCE7064B04F19C001B6898476F468F
:1051F0008146C4E76FF03709C9E76FF03509C6E7A4
:105200009C000020A0000020F8B51C46054611486F
:105210000E461746FFF772FB21460E48FFF788FB44
:10522000044620B10B48FFF77DFB2046F8BD32460F
:1052300029460848FFF790FB04460028F2D139467A
:105240000448FFF791FB04460248FFF76BFB20463A
:10525000F8BD00BF9C1500201C2330B583B001A908
:105260000446019300F03EF8054638B9019B1C2B1B
:1052700007D0164D20461C2100F030F8284603B018
:1052800030BD0121D4E90032003B18BF0123E161A8
:105290000AB143F00203A26832B9E26842B9C4E934
:1052A00008328BB90A4DE5E7E26843F004033AB1EE
:1052B0000022284643F00803C4E9083203B030BD99
:1052C0001546C4E90832D9E71546D7E7370CF00090
:1052D0000E0CF00001F028BB01F068BB0A4600216B
:1052E00001F064BB002866D0002964D00B681C2B39
:1052F00061D14FF47F033B4AD3F8101C91425CD03C
:10530000D3F8102C013258D0D3F8102C4FF47F036F
:105310000260D3F8141C344A914260D0D3F8142CA4
:1053200001325CD0D3F8142C4FF47F034260D3F8E1
:10533000182C12F5947F4FD0D3F8182C01324BD093
:10534000D3F8182C4FF47F038260D3F81C1C274A33
:1053500091423ED0D3F81C2C01323AD0D3F81C2C09
:105360004FF47F03C260D3F8002C70322FD0D3F8F3
:10537000002C01322BD0D3F8002C4FF47F030261B4
:10538000D3F8042CAF3220D0D3F8042C01321CD037
:10539000D3F8042C4FF47F034261D3F8081C144A5D
:1053A00091420DD0D3F8082C013209D0D3F8083C33
:1053B0008361002070470120704740F6FC02A5E79A
:1053C00040F237338361002070475122E2E7902298
:1053D000D3E742F60412C3E740F6D862B2E742F2DE
:1053E000D002A1E7FCF8FFFFD020FFFF0429FFFF58
:1053F00037F3FFFF014608B54FF48060FEF724FE47
:1054000000230249024A0B60136008BDC811845092
:105410002C1184500138072805D8DFE800F00A0E67
:1054200004120404040609487047CB6800204B624C
:1054300070470B6800204B6270474B6800204B623E
:1054400070478B6800204B62704700BF310CF10041
:105450000B6802E0082B0B6006D8026A13424FEA81
:105460004303F7D00020704700487047310CF1002B
:1054700000230449044A0B604FF480601360FEF778
:10548000C9BD00BF2C118450C41184502DE9F041D6
:10549000002682B0B0F1005F8DF80760099E27D327
:1054A0000C460444B4F1804F054621D8174698466F
:1054B00001220DF1070300F00FFA0446C0B99DF870
:1054C00007303D603B71AEB1B8F1000F09D0024624
:1054D000089940460DF1070300F0FEF940B99DF828
:1054E00007302046C6F80080337102B0BDE8F08175
:1054F0004FF47504204602B0BDE8F081E8B110B564
:105500000468012C04D0022C10D044B10C4810BD0A
:1055100020220C490830FFF7DDFE002010BD1422C8
:1055200009490830FFF7D6FE204610BD2022074962
:105530000830FFF7CFFE002010BD4FF47300704716
:105540000100F300907201005C72010070720100B2
:105550002DE9F041002900F0EF800446002800F01A
:10556000EF80036817460E46002B00F0B980013B20
:10557000012B00F2CD804FF0FF3173484FF002084D
:10558000FEF7EEFD002840F0B5800020FEF718FE83
:105590000546002840F0B8806C4A1368002BFCD107
:1055A0006B480368002BFCD14FF0FF30FEF732FD53
:1055B000684B186820F04000FEF73AFD01230720F1
:1055C000654A66491360086042F8543CA16C644B1C
:1055D000483A1960E16C116043F80C8C236863B1A0
:1055E000013B012B18D8616A5E4BA2F5BC721960B1
:1055F000216A1160E26943F8082CA1695A4B5B4AA1
:10560000196061691160216943F8081CE16842F87A
:10561000081CA26843F8102C554A1368002BFCD1D3
:10562000002F59D063684020012B04BF514A1360FA
:105630003168514A514B11601F60FEF7FFFC05466F
:105640004B4A1368002BFCD1414A1368002BFCD154
:1056500023685BB1013B012B16D8424B484A1968BD
:10566000083B6162126822621B68E3613E4B3F4A5D
:105670001968083AA1619168103B616199682161DC
:105680001268E2601B68A3600121002334483D4A90
:105690000068A0641068E06442F80C1C35483A4980
:1056A000036002F5A0720B601368002BFCD12A4A3C
:1056B0001360002D3AD1274B186840F04000FEF7E8
:1056C000B7FC0120FEF77CFD60BB1F48FEF750FDD4
:1056D00010BB2846BDE8F08104222B4B1A60AFE7CF
:1056E0004FF0FF3118484FF00108FEF739FD002850
:1056F0003FF44BAF2548FEF7C3F90020FEF760FDED
:10570000054600283FF448AF2148FEF7B9F943E7C2
:10571000204D2846BDE8F0811F48FEF7B1F9284624
:10572000BDE8F0811D48FEF7ABF9CEE7102104F18A
:105730000800FFF7D3FDBEE7194D2846BDE8F0810C
:105740004FF47305C5E700BF900000201C1984507A
:10575000201C8450041A8450181884500019845056
:10576000CC1784505C168450501684504C168450CC
:105770001019845084168450281C84502C1C84508A
:1057800058168450D0178450C8178450A471010053
:10579000BC7101000100F300FC710100DC7101002B
:1057A0000300F30000283AD02DE9F041D0E90623A8
:1057B00092FA82F893FA83FE026A436AD0E90441BE
:1057C00012BA24BA1BBA04610262846A826B436211
:1057D000C36BD0E9026509BA36BA2DBAC76A8660CA
:1057E000C560066B456B416194FA84FC19BA14BA22
:1057F000436C026C3FBA36BA2DBA12BA1BBAC0E972
:105800000C65C0E90E41C0F81880C0F81CE0C0F873
:1058100028C0C762C0E910230020BDE8F0814FF422
:105820007300704710B5044630B100220123C4E96B
:105830001522C4E9173310BD0148FEF721F9F4E73A
:10584000B072010018B174220021FFF745BD704706
:1058500088B199B110B50024802A846380F83C4057
:1058600006D1046310221030FFF734FD204610BD2E
:105870006FF01F0010BD6FF0210070476FF01F0028
:10588000704700BF28B322B31BB3012921D870B5DC
:105890000446816B86B017D0012917D1102500214D
:1058A0000DEB0506616310462946009502AA019694
:1058B000FFF7ECFD50B92B463246204602A900F016
:1058C000EBF818B906B070BD0029E7D06FF02100E1
:1058D000F8E76FF02100704700201870704700BF94
:1058E00000284DD038B5044690F83C00022816D068
:1058F00003283DD0002830D02348244D2A68244B6B
:10590000126824491A602B68234A5C68234B0C6098
:105910002968896811602A68D2681A6038BD216BCD
:10592000206C00F0CBFB194D0028E7D12A68184BFA
:105930001068184918602868174A40680860296884
:10594000896811602A68D268DA60216B206C00F0E7
:10595000D9FB0028D2D1002038BD21690C4A0D4B5B
:10596000116061691960A1699160E2699A6038BD4E
:10597000216B206C00F0B8FB0028BED1034DD5E7A9
:105980004FF47100704700BF0900F1008000002053
:105990000014845004148450081484500C1484504F
:1059A00010B50446314A1368002BFCD1304A136805
:1059B000002BFCD12F4A1368002BFCD12E4A136810
:1059C000002BFCD12D4A1368002BFCD12C4A136804
:1059D000002BFCD14FF0FF30FEF71CFB636B23F074
:1059E0000403032BE36D36D0012B264B18680CBF44
:1059F00020F0800020F02000FEF71AFB0121224B4E
:105A00001A4A19601368002BFCD1194A1368002B3D
:105A1000FCD11E49154A0B601368002BFCD1144AB7
:105A20001368002BFCD1626B22F00401032918BF1C
:105A3000A36B4FEA820218BF03F00103144902F07E
:105A40001C0213430B60636B072B02D10122114B25
:105A50001A60002010BD012B0A4B18680CBF20F003
:105A6000400020F01000FEF7E3FAC7E71019845059
:105A700070148450201D8450201C8450381D845084
:105A8000381C8450041A845000198450BC1484506B
:105A9000C01484507C1484502DE9F04F87B0002945
:105AA00000F0A5801646002A00F0A18004460028D8
:105AB00000F041811F46C36D0D46002B50D1B7F554
:105AC000805F52D294F83C30042B00F00B814FF0F1
:105AD00000084FF0FF31A948FEF742FB002840F0D4
:105AE000E0800020FEF76CFB002840F0E3800121FD
:105AF000A34BA44A19601368002BFCD1636B032BE2
:105B000039DC002B3ADADFF8C8929E4A1368002B82
:105B1000FCD1B8F1000F40F0DC80636B23F004038C
:105B2000032BE36D58D0012B974B18680CBF40F046
:105B3000800040F02000FEF77BFA0022904B01200D
:105B40001A60FEF73DFB002840F0BF808B48FEF74F
:105B50000FFB002840F0B280484607B0BDE8F08F48
:105B6000012BAFD1B7F5803FACD3DFF86892484640
:105B700007B0BDE8F08F063B012BC4D8A36B012B07
:105B800000F2D680E36D012B37D8236E012B00F293
:105B900034812046FFF704FF81460028B5D1204616
:105BA000FFF79EFE81460028AFD1636B072BAAD872
:105BB00001A252F823F000BF175C0100015C010054
:105BC000735D0100015C0100075B0100075B0100E0
:105BD000735D0100015C0100012B6B4B18680CBF69
:105BE00040F0400040F01000FEF722FAA5E7DFF891
:105BF000E891484607B0BDE8F08FDFF8E09184E710
:105C00002168624A624B116061681960A168916005
:105C1000E2689A60636B23F00403032B2A6809D0BF
:105C2000216E3368012907BF5A485B495B485C49CC
:105C300003600F60E36D012B0BBF5A4B5A4B5B495E
:105C40005B490A601F60636B23F00403032B75D06C
:105C5000236E012B0CBF80202020FEF7EFF9814638
:105C600000287FF452AF474B1A68002AFCD1636BBF
:105C70009146013B062B11D8DFE803F004BC041069
:105C800010BC0400414A424B116808322160196877
:105C9000083361601268A2601B68E3600123A3659A
:105CA00033E74448FDF7ECFE0020FEF789FA0028B0
:105CB0003FF41DAF4048FDF7E3FE18E73F48FDF70E
:105CC000DFFE484607B0BDE8F08F3D48FDF7D8FE3F
:105CD0003CE70423202184F83C3004F11000FFF756
:105CE000FDFA1AE7216B206C00F0D2F9E8B9DFF871
:105CF000F080DFF8F0B0D8F80030DFF8ECA01B68D7
:105D0000DFF8E890CBF80030D8F800302D4A5B6817
:105D1000CAF80030D8F800309B68C9F80030D8F8CD
:105D20000030DB681360216B71B14FF00108D0E6E1
:105D3000DFF8BC90E9E64FF471090DE7E36D012B44
:105D40000CBF4020102088E7D4E9133200931023C1
:105D500004F11000CDE9012003930590D4E911234B
:105D6000206C00F04DFA00284AD1002384F83C3022
:105D7000DBE72168144A154B45E700BF900000207F
:105D80001018845010198450041A84504014845000
:105D900044148450281D84502C1D8450301D845080
:105DA000341D84502C1C8450341C8450281C845076
:105DB000301C8450A4710100BC710100FC71010011
:105DC000DC7101000C1484506014845064148450FD
:105DD0000100F1000500F1000B00F1000300F100EB
:105DE000800000200014845004148450081484504F
:105DF0000200F1000F4A104B46E7DFF8449084E6BA
:105E0000D8F8003005981B680C4ACBF80030D8F859
:105E1000003010215B68CAF80030D8F800309B6869
:105E2000C9F80030D8F80030DB681360FFF756FA85
:105E30009BE700BF60148450641484500C14845099
:105E40000400F1002DE9F04101B3FAB10446002845
:105E50007AD01D46436B0E46072B1BD05DB9032B32
:105E600010D1836D73B9C0E91955C0E91B551025D0
:105E700000F164030B602B4631462046BDE8F0413B
:105E8000FFF70ABE2F463846BDE8F081684F384616
:105E9000BDE8F081C36D002B59D1B5F5805F5BD2B1
:105EA00015B9A36D002B57D14FF0FF316148FEF7B4
:105EB00057F9002840F09A800020FEF781F9002869
:105EC00040F0908001215C4B5C4A19601368002B04
:105ED000FCD1636B032B20DD063B012B1FD8A36B8A
:105EE000012B3BD8E36D012B00F28880236E012B40
:105EF00000F286802046FFF753FD074680B9204612
:105F0000FFF7EEFC074658B9636B072B07D8DFE8AD
:105F100003F03127552706065527002BDFDA484FB7
:105F2000464A1368002BFCD1434A01201360FEF758
:105F300047F900285ED13F48FEF71AF90028A2D0A1
:105F40004048FDF79DFD9EE74FF471079BE7012B4D
:105F5000A6D1B5F5803FA3D33B4F94E73B4FDFE796
:105F600021683B4A3B4B116061681960A1689160F0
:105F7000E2689A6001233849384A0B601560002DA9
:105F800040D1A26D0AB9364A13602C4B1F68002F0E
:105F9000FCD1636B013B062BC2D801A252F823F05F
:105FA000C55F0100DF5F0100C55F0100215F0100E7
:105FB000215F0100DF5F0100C55F01002168294A00
:105FC000294BD0E7224A234B116808322160196817
:105FD000083361601268A2601B68E360A0E7214A91
:105FE000214BF1E72148FDF74BFD6BE72048FDF71A
:105FF00047FD61E71F48FDF743FD9CE71E4F8FE714
:106000001E4F8DE7E26D3368012A0AD010201C492B
:106010001C4A0B601560FEF711F807460028B4D043
:106020007EE71949194A0B6040201560F3E700BF6D
:106030000B00F100900000201018845010198450BB
:106040000100F100FC7101000500F1000200F10007
:1060500040148450441484507C148450BC148450E4
:10606000241584506014845064148450BC71010061
:10607000A4710100DC7101000300F1000400F100D3
:10608000301C8450341C8450281C84502C1C845098
:106090007F280CD849B1032901D00648704706492A
:1060A0007F280CBF0846002070470846704702480A
:1060B000704700BF0300F7000100F700831E7D2B2F
:1060C0000CD849B1032901D00548704705497F28FC
:1060D0000CBF0846002070470846704701487047CB
:1060E0000300F7000100F70028B9044B002918BF8E
:1060F0001946084670470249084670470300F700F2
:106100000100F700002858D009B13348704730B477
:106110000124324B324A84B0C2F80045C3F808115A
:10612000D3F8082105190292029AC3F80011D3F896
:10613000002180300292029AC3F80411D3F80411AE
:10614000284A02910299C3F8005552F83010264AA5
:1061500003910399914236D11A461C6005E09DF8DF
:106160000630DBB99DF80730C3B9D2F80031003BE7
:1061700018BF01238DF80530D2F80831003B18BF55
:1061800001238DF80630D2F80431003B18BF0123FB
:106190008DF807309DF80530002BE0D09DF80630D3
:1061A000ABB99DF8073003F0FF0293B910460B4BD3
:1061B000C3F8002504B030BC704701220B490C4BDA
:1061C00008601A6070470B4804B030BC70470A483A
:1061D000F0E70A48EEE700BF0C00F1000090035022
:1061E000000084500080FF0000148450381A84504E
:1061F000781484500600F7000100F7000200F70051
:106200002DE9F04F0024CDB00546DDE958968846CB
:106210001746214674220EA89B4600F0C7FB214674
:1062200080222CA82B9400F0C1FB8423B6F57F6F4D
:10623000CDE90A44CDE90C4405935DD805AB0DF1D9
:10624000AC0A01935946DDE9562338460296CDF84B
:1062500000A000F061F8002855D1A5420CBF4FF016
:10626000030C4FF0020C0022012307270124102108
:106270001C900EA8CDE92423CDF868808DF874C059
:106280001B971E952694FFF729F810220DF1200880
:106290000092504605990AAB06AACDF80480FFF794
:1062A000F5F80746C8B10EA874220021FFF714F8CC
:1062B00038464DB0BDE8F08F102E354628BF10256A
:1062C0000EA92A46FFF706F810210EA8FFF706F8D8
:1062D0000134761B2F44E4B213D0059B424606A935
:1062E0000EA88DF8AC40FFF7ADFD034609EB0700A3
:1062F000002BE1D01F46D6E7054F38464DB0BDE82C
:10630000F08F3746CFE7034F38464DB0BDE8F08FEA
:106310000F00F1000E00F1002DE9F041002682B0DF
:106320000A9D0196B5F57F6F3BD8EE00B6F5807FEC
:106330001F4634BF032304234D1E3F2D0C460093FC
:106340002FD870B3904617B15AB3402F29D8089A66
:106350003AB3099A116821B3E2191344994220D340
:10636000089B22460146581CFEF7B4FF0022089BFA
:1063700023445A70023407BBFF2E009615D9089BA0
:106380003502ADB21819022245EA162501A9019578
:10639000FEF7A0FF02340020099B1C6002B0BDE89C
:1063A000F0810A4802B0BDE8F081089B012218196B
:1063B0006946FEF78FFF0134EDE7089B4146181947
:1063C0003A46FEF787FF3C44D6E700BF0600008050
:1063D00008B5FBF795FABDE80840FBF731BA03466C
:1063E00058B1426802F00302012A03D0032A04D103
:1063F000026812B10020986070476FF01500704776
:106400004268034602F00302032A4FF00002816053
:1064100014BF104600685A607047002070470FB4E0
:1064200007B504A951F8040B0191FAF7B7F903B0C5
:106430005DF804EB04B07047038B13F0070305D13C
:106440000368002B0CBF002003207047022B05D1EE
:10645000438B002B14BF002004207047012B05D173
:106460000368002B0CBF00200520704700207047F8
:106470002DE9F0410D4607461946281D90461E4657
:10648000FFF7BEFF044638B1334642462946384638
:10649000A446BDE8F0416047BDE8F08110B44FF07C
:1064A0002004EFF3118284F31188BFF36F8F4161F1
:1064B00010BC0121FAF780B910B50C4640B139B1D2
:1064C000081DFFF78CFF28B9A36833F0030301D040
:1064D0006FF0150010BD38B50C46054658B151B1E6
:1064E0000B6843B14B6833B11C22002100F05EFA07
:1064F00000202C6138BD6FF01500FBE770B5044635
:106500000E46FFF7D9FF051E31DB4FF02003EFF3F6
:10651000118183F31188BFF36F8F4FF6FF75638B83
:10652000208BAB4200F007022ED0022A0ED101339D
:1065300063831546012381F31188BFF36F8FB3B1D5
:10654000002331462046FFF793FF10E0830701D078
:10655000062A0ED100233360636893B9C4E900664C
:10656000154662B90A4620460221FAF725F928465F
:1065700070BD052A0CBF6FF085056FF00405002380
:10658000D9E71E606660EBE76FF00A05F7E704469F
:1065900008B5084611461A46A047FDF76FF8FBF705
:1065A000ABFE2DE9F74F9946D37814466F2BA3F134
:1065B000410206460F4601922DD028D8582B14BF11
:1065C0000A251025AA464FF0000BDDF83080524610
:1065D0005B4630463946F9F731FF092AD3B21FD856
:1065E00030335F45DBB208BF564508F8013D01D3A3
:1065F000C84512D823789B0605D5082D16D1A37857
:1066000043F00803A370404603B0BDE8F08F03F0E9
:10661000F703702BD3E70825D4E706460F46D6E7E5
:10662000019A192A94BF37335733DAE7102DEAD18C
:10663000A37843F01003E5E72DE9F04107468846CB
:1066400015461E461446B442A4EB050002D33EB9DB
:1066500023782BB1414614F8010BB8470028F2DA31
:10666000BDE8F0817047FCF7CBB884B004AB03E918
:106670000700002383F31188BFF36F8F04B07047C6
:106680000022C0E9002282607047CBB20C2102696F
:1066900003FB0121086C00F0070070474FF0200356
:1066A000EFF3118283F31188BFF36F8F036813F048
:1066B000C00301D08B4207D101230360002082F385
:1066C0001188BFF36F8F70474FF0FF30F7E710B5B9
:1066D0004FF02003EFF3118283F31188BFF36F8F24
:1066E000036803F00704012C06D10160002082F347
:1066F0001188BFF36F8F10BD03F0C0038B4214BF2E
:106700004FF0FF306FF07700F1E74FF02003EFF329
:10671000118283F31188BFF36F8F036803F0C00306
:1067200043F00203036082F31188BFF36F8F704759
:1067300010B41C240069CBB203FB0400002110BC80
:1067400010470020FCF71CB90020FCF74BB910469D
:10675000FCF74CBC38B50C23CCB26343054600694A
:10676000403380211844FFF799FF002805DB696852
:1067700001EBC40463689847002038BD2DE9F84355
:106780000C27CDB26F430469064607F14000802113
:10679000204490469946FFF79AFF002807DB3C44C7
:1067A000C4E90E89736853F8353098470020BDE876
:1067B000F88370477047704738B505460C4651B9A5
:1067C0006FF01500BDE83840714672467346F446D6
:1067D0008EF3008C744700F065F80128F0D1204654
:1067E00000F060F80128EBD02846FBF73DF90146A0
:1067F00028B13C22204600F0AEF80020E2E76FF01E
:106800000D00DFE70020FAF777BC0021012000F03F
:1068100033B8024643B20846C1B9002B27DB01203A
:106820005B099B0003F1604303F56143D3F88012D9
:1068300002F01F02904021EA0001C3F88012D3F851
:106840008002D04000F00100C0B27047002B0DDB89
:1068500001215B099B0003F1604303F56143D3F819
:10686000800202F01F0291400143E6E700207047DA
:10687000436E83F30B88704700F0D9B80146006877
:1068800000F0D5B808B5FBF751FBBDE80840FBF7B1
:10689000D1BC40E800F313F4803FD8B208BF6FF0DA
:1068A0001500704740E800F0C0F3805070477FB596
:1068B0000A898E7A0B684D6802F01F0242EA46127E
:1068C00000938DF8082023F01F036A1E134423F061
:1068D0001F030F28039304D86946FBF7B1FD04B0EA
:1068E00070BD6FF01500FAE7034600201A5C02B98C
:1068F00070470130FAE7034600201A5C0AB188426B
:1069000000D170470130F8E710B55AB10139841849
:1069100010F8012B11F8013FA04201D09A42F7D0A4
:10692000D01A10BD1046FCE7431A934210B500EB95
:10693000020308D3024601399A420BD011F8014FE5
:1069400002F8014BF8E70A4412F8014D8A4203F8B5
:10695000014DF9D110BDF0B581EA0004A507034649
:106960000BD0013B0A4491421BD1F0BD002AFCD060
:1069700011F8014B013A03F8014B9C07F6D122F0C4
:1069800003041D1F96080F19B94205D16FF00305C6
:10699000234405FB0622E4E751F804CB45F804CF75
:1069A000F2E711F8014B03F8014FDCE7034670B53D
:1069B000C9B29C0711D141EA012422F0030644EA3E
:1069C00004451E449408B3420DD16FF0030505FB46
:1069D00004221A44934209D170BD002AFCD003F866
:1069E000011B013AE5E743F8045BECE703F8011B00
:1069F000F0E7002008B5FBF72BFCFDF70DB808B554
:106A0000FBF7FAF8FBF7A4F9BDE80840FDF704B876
:106A1000004700F065B908B50520FBF715FA20B965
:106A2000BDE808400520FBF7FFB908BD7047F8B581
:106A300005460E464FF02003EFF3118783F31188CC
:106A4000BFF36F8FFCF71AFE314604462846FFF766
:106A5000D0FF87F31188BFF36F8F2046BDE8F84061
:106A6000FBF74ABC30B50024846141EA020414F00B
:106A70000304C0E9023201610CD14461A34203D195
:106A8000C0E90000002030BD456901340D6041615E
:106A90001144F3E76FF01500F5E7F8B504460D462D
:106AA0004FF02003EFF3118683F31188BFF36F8F4C
:106AB000476977B900F0B8F858B12A68876742612A
:106AC00000F080F8314604F10800BDE8F840FCF71A
:106AD0001FBB2B6862691A602B686361A369013B65
:106AE000A36186F31188BFF36F8FF8BDEFF30580C4
:106AF000003818BF0120704708B5FAF769FBBDE8F8
:106B00000840FFF757BE03460020C3E90033C3E93E
:106B100002007047D0E9003213605A600023C0E9D8
:106B20000033704708B5FFF7F5FF437B23F00203FE
:106B300043730023836008BD034620B9EFF3058249
:106B40000AB9FBF71BB983F31188BFF36F8F704746
:106B50004FF02003EFF3118083F31188BFF36F8FA1
:106B6000FFF7EABF0368984214BF18460020704739
:106B700038B504460D46FCF711FB637B43F0020376
:106B8000637395B12B68A5609D4215D0A3B194F9AC
:106B90000E1093F90E20914208D0521A002A05DDFA
:106BA0005A68C4E9003214605C6038BD6A68934278
:106BB00002D01B68002BECD16B68C4E900531C6049
:106BC0006C60F2E710B54FF02003EFF3118483F30C
:106BD0001188BFF36F8FFCF737FC84F31188BFF384
:106BE0006F8F10BD014610B54FF02003EFF31184F5
:106BF00083F31188BFF36F8F10F80B3C13F0280F4D
:106C00000DD151F8103C18380BB1FFF78BFF11F87C
:106C10000B3C23F0140301F80B3CFCF715FC84F348
:106C20001188BFF36F8F10BD38B54FF02003EFF31D
:106C3000118583F31188BFF36F8FFFF793FF04462D
:106C400020B1FFF76FFF183000F006F885F31188C8
:106C5000BFF36F8F204638BD10B54FF02002EFF321
:106C6000118482F31188BFF36F8F03683BB1FCF787
:106C700081FD002084F31188BFF36F8F10BD6FF08A
:106C80001500F7E710B54FF02003EFF3118483F3FD
:106C90001188BFF36F8FFCF787FD84F31188BFF372
:106CA0006F8F10BD70B504460D464FF02003EFF313
:106CB000118683F31188BFF36F8FFCF775FD0128F0
:106CC00005DDA04203DB29462046FAF709FD86F3DD
:106CD0001188BFF36F8F70BD08B5FCF783FE08BD48
:106CE00008B1FAF735BA7047704770478097FF7F51
:106CF000010000002911010000000000852C0100A6
:106D000000000000FB6901000000000015130100F5
:106D1000A40000202D270100BC0000208D160100DA
:106D2000D4000020FF690100000000004927010095
:106D300000000000000000000B68010000000000DF
:106D40000B680100000000000B680100000000005B
:106D50000B680100000000000B680100692A0100B7
:106D6000116A0100000000000B6801000000000033
:106D70000B680100000000000B680100000000002B
:106D80000B680100000000000B680100000000001B
:106D90000B680100000000000B680100000000000B
:106DA0000B680100000000000B68010000000000FB
:106DB0000B680100000000000B68010000000000EB
:106DC0000B680100000000000B68010000000000DB
:106DD0000B680100000000000B68010000000000CB
:106DE0003D160100000000000B68010000000000DB
:106DF0000B680100000000000B68010000000000AB
:106E00000B680100000000000B680100000000009A
:106E10000B680100000000000B680100000000008A
:106E20000B680100000000000B680100000000007A
:106E30000B680100000000000B680100000000006A
:106E40000B680100000000000B680100000000005A
:106E50000B680100000000000B680100000000004A
:106E60000B680100000000000B680100000000003A
:106E70000B680100000000000B680100000000002A
:106E80000B680100000000000B680100000000001A
:106E90000B680100000000000B680100000000000A
:106EA0000B680100000000000B68010000000000FA
:106EB0000B680100000000000B68010000000000EA
:106EC0000B680100000000000B68010000000000DA
:106ED0000B680100000000000B68010000000000CA
:106EE0000B680100000000000B68010000000000BA
:106EF0000B680100000000000B68010000000000AA
:106F00000B680100000000000B6801000000000099
:106F10000B680100000000000B6801000000000089
:106F20000B680100000000000B6801000000000079
:106F30000B680100000000000B680100FF7FFF7F6D
:106F4000FF7FFF7FFF7FFF7FFF7FFF7FFF7FFF7F51
:106F5000FF7FFF7FFFFFFFFFFFFFFFFFFFFFFFFF41
:106F6000DEE61E284CBBCE8F025B0000DEE61E284C
:106F7000EAAC45B8025B0000DEE61E284CBBCE8FB3
:106F8000025B0000000000000000000000000000A4
:106F90000338FDD8704700004D140100556701000B
:106FA0007D670100000000008B660100C513010031
:106FB000291401004367010049670100BD12010067
:106FC00075120100000000009F74010042010000E2
:106FD000A674010005010000B07401001401000056
:106FE000B974010015010000C274010039010000EC
:106FF000CB74010009010000D67401000A010000F1
:10700000E17401000A010000EB7401000B010000B3
:10701000F57401000F01000000750100100100006F
:107020000B75010011010000167501000E01000032
:1070300020750100210100002975010022010000D6
:1070400032750100230100003B750100240100009E
:1070500044750100180100004C7501002A01000070
:10706000547501003A0100005C7501002C0100001C
:10707000647501001C0100006D7501001D01000018
:107080007675010017010000807501000401000001
:107090008F7501002601000097750100280100008E
:1070A0009F75010031010000000000000002000097
:1070B00000040000000800000010000000000000B4
:1070C00005680100911C0100491C0100011D01001F
:1070D000051C0100200000200800002018000020EE
:1070E0000000000010000020000000200000000050
:1070F0000600010002000000FC700100000000001A
:10710000FE75010006000000E0FF0F0000000020F7
:107110000676010021000000E0FF0020DD260100CE
:1071200000000000F46C01001C6D0100246D0100E2
:10713000346D0100346D0100F5FFFFFFFF8FFFFF8D
:10714000FF8FFFFFFE8FFFFFFE8FFFFFFD8FFFFF13
:10715000FC8FFFFFFC8FFFFF6D757465785F6672B3
:1071600065652063616C6C65642077697468204E86
:10717000554C4C20706172616D6574657200000041
:1071800043616E277420696E697469616C697A6500
:10719000206D757465782C20776173204E554C4CAA
:1071A0000D0A00004661696C20746F20616371757F
:1071B000697265206D757465780A00004661696CB6
:1071C00020746F20696E63726561736520504D2075
:1071D000636F756E7465720A000000004661696C29
:1071E00020746F20646563726561736520504D2063
:1071F000636F756E7465720A000000004661696C09
:1072000020746F2072656C65617365206D7574659F
:10721000780A0000436F756C64206E6F74206C6F89
:10722000636B20706F7765722073617665206D7572
:10723000746578004661696C20746F20756E6C6FA0
:10724000636B206D757465780A0000000A637478BA
:10725000206973204E554C4C0A00000001234567FD
:1072600089ABCDEFFEDCBA9876543210F0E1D2C390
:10727000D89E05C107D57C3617DD703039590EF719
:10728000310BC0FF11155868A78FF964A44FFABEDF
:1072900067E6096A85AE67BB72F36E3C3AF54FA5A7
:1072A0007F520E518C68059BABD9831F19CDE05BD3
:1072B0006374782063616E6E6F74206265204E5532
:1072C0004C4C00286E696C29004661696C6564202D
:1072D000746F207265626F6F743A207370696E6E9E
:1072E000696E6720656E646C6573736C792E2E2EE3
:1072F0000A007379735F636C6F636B00536563752A
:1073000072650909004E6F6E2D53656375726509CC
:107310000025303275202530327520307825303503
:1073200078203078253035782009002563005350C7
:107330004D3A204E5320696D61676520617420309D
:107340007825780A0053504D3A204E53204D535023
:1073500020617420307825780A0053504D3A204E31
:107360005320726573657420766563746F72206153
:107370007420307825780A0053504D3A2070726599
:107380007061726520746F206A756D7020746F2053
:107390004E6F6E2D53656375726520696D6167650B
:1073A0002E0A004E6F6E2D53656375726500466C34
:1073B00061736820726567696F6E730909446F6D48
:1073C00061696E09095065726D697373696F6E73D7
:1073D0000A004E6F6E2D7365637572652063616C74
:1073E0006C61626C6520726567696F6E2030207019
:1073F0006C6163656420696E20666C6173682072DD
:107400006567696F6E2025642077697468207369E9
:107410007A652025642E0A00436F756C64206E6FB8
:107420007420696E697469616C697A65207365633B
:10743000757265207365727669636573202865725D
:1074400072202564292E0A005352414D207265672F
:10745000696F6E0909446F6D61696E090950657243
:107460006D697373696F6E730A0050657269706835
:107470006572616C0909446F6D61696E0909537425
:10748000617475730A002530327520252D323173F1
:1074900025730009534B49500A00094F4B0A004E0F
:1074A00052465F5030004E52465F434C4F434B00B4
:1074B0004E52465F52544330004E52465F52544340
:1074C00031004E52465F4E564D43004E52465F5578
:1074D0004152544531004E52465F55415254453257
:1074E000004E52465F5457494D32004E52465F534C
:1074F00050494D33004E52465F54494D455230007D
:107500004E52465F54494D455231004E52465F54EB
:10751000494D455232004E52465F5341414443006B
:107520004E52465F50574D30004E52465F50574DB9
:1075300031004E52465F50574D32004E52465F501A
:10754000574D33004E52465F574454004E52465FEB
:10755000495043004E52465F564D43004E52465FDF
:10756000465055004E52465F45475531004E5246F3
:107570005F45475532004E52465F445050494300E4
:107580004E52465F524547554C41544F5253004E60
:1075900052465F50444D004E52465F493253004EB2
:1075A00052465F4750494F544531006D75746578B8
:1075B0005F696E69742063616C6C656420776974BF
:1075C00068204E554C4C20706172616D6574657217
:1075D00000436F756C64206E6F7420616C6C6F6318
:1075E000617465206D75746578206265666F72657B
:1075F00020696E697469616C697A696E6700464CCE
:107600004153485F30005352414D5F30004352595F
:1076100050544F43454C4C004552524F523A204330
:10762000616E6E6F742066756C66696C6C2045586F
:10763000545F41504920726571756573742E0D0A4F
:10764000005741524E494E473A204F7074696F6E51
:10765000616C204558545F415049207265717565D1
:107660007374206E6F742066756C66696C6C6564EB
:107670002E0D0A006D61696E00000000000001001F
:107680001B64010001000000EC000020010000006C
:107690000001002001000000140100200100000092
:1076A00028010020010000000090D0032C000020E1
:1076B0002C000020000000005D3A0100940D002025
:1076C00001000000B93B0100953B0100D93B0100DE
:1076D000753B0100780000203C0000207000002075
:1076E0000000000068000020980D0020010000004C
:1076F0009C0D002001000000A00D002001000000F2
:10770000A40D002058000020640000205C00002030
:10771000540000208C00002045420100514201002D
:107720005D420100AA740100AC6F0100986F010076
:107730005C020020700200204A6F01000D760100FB
:10774000000000001C710100C809002000000000BA
:10775000426F0100F2720100000000000000000012
:10776000C8020020000000003C6F0100EC00002077
:10777000EC00002000000000000000000F000000EE
:1077800000010020000100200000000000000000B7
:107790000F00000014010020140100200000000070
:1077A000000000000F000000280100202801002038
:1077B00000000000000000000F000000FFFFFFFFBE
:1077C00000000000000000000000000000000000B9
:1077D00000000000000000000000000000000000A9
:1077E0000000000000000000000000000000000099
:1077F0000000000000000000000000000000000089
:107FE0007FE97FE9FEF7E8BB7FE97FE9F9F7A2BD0A
:107FF0007FE97FE9F9F7C2BD7FE97FE9F9F760BD65
:10800000FFFFFFFFFFFFFFFFFFFFFFFFFFFFFFFF80
:10801000FFFFFFFFFFFFFFFFFFFFFFFFFFFFFFFF70
:10802000FFFFFFFFFFFFFFFFFFFFFFFFFFFFFFFF60
:10803000FFFFFFFFFFFFFFFFFFFFFFFFFFFFFFFF50
:020000040002F8
:100200008060022045D1020061F60300A5D1020002
:10021000A5D10200A5D10200A5D10200A5D10200FE
:10022000000000000000000000000000EDCE020011
:10023000A5D102000000000095CE020013F60300D5
:1002400005D1020005D1020005D1020005D102004E
:1002500005D1020005D1020005D1020005D102003E
:1002600005D1020005D1020005D1020005D102002E
:1002700005D1020005D1020005D1020005D102001E
:1002800005D1020005D1020005D1020005D102000E
:1002900005D1020005D1020005D1020005D10200FE
:1002A00005D1020005D1020005D1020005D10200EE
:1002B0001D0903002D15040005D1020005D102001F
:1002C00005D1020005D1020005D1020005D10200CE
:1002D00005D1020005D1020005D1020005D10200BE
:1002E00005D1020005D1020005D1020005D10200AE
:1002F00005D1020005D1020005D1020005D102009E
:1003000005D1020005D1020005D1020005D102008D
:1003100005D1020005D1020005D1020005D102007D
:1003200005D1020005D1020005D1020005D102006D
:1003300005D1020005D1020005D1020005D102005D
:1003400005D10200000000000000000000000000D5
:10035000000000000000000000000000000000009D
:10036000000000000000000000000000000000008D
:10037000000000000000000000000000000000007D
:10038000000000000000000000000000000000006D
:10039000000000000000000000000000000000005D
:1003A000000000000000000000000000000000004D
:1003B000000000000000000000000000000000003D
:1003C000000000000000000000000000000000002D
:1003D000000000000000000000000000000000001D
:1003E000000000000000000000000000000000000D
:1003F00000000000000000000000000000000000FD
:10040000DEE61E284CBBCE8F025B00003C000000E5
:1004100038B90200010000000002020000020200E0
:10042000FFFF02910000000000000000000000003B
:10043000000000000000000000000000FFFFFFFFC0
:1004400081F0004102E000BF83F0004330B54FEA85
:1004500041044FEA430594EA050F08BF90EA020FF2
:100460001FBF54EA000C55EA020C7FEA645C7FEA85
:10047000655C00F0E2804FEA5454D4EB5555B8BFA8
:100480006D420CDD2C4480EA020281EA030382EA19
:10049000000083EA010180EA020281EA0303362DAB
:1004A00088BF30BD11F0004F4FEA01314FF4801C7E
:1004B0004CEA113102D0404261EB410113F0004F90
:1004C0004FEA03334CEA133302D0524263EB430347
:1004D00094EA050F00F0A780A4F10104D5F1200EE5
:1004E0000DDB02FA0EFC22FA05F2801841F1000140
:1004F00003FA0EF2801843FA05F359410EE0A5F114
:1005000020050EF1200E012A03FA0EFC28BF4CF044
:10051000020C43FA05F3C01851EBE37101F00045FA
:1005200007D54FF0000EDCF1000C7EEB00006EEB07
:100530000101B1F5801F1BD3B1F5001F0CD3490891
:100540005FEA30004FEA3C0C04F101044FEA4452E8
:1005500012F5800F80F09A80BCF1004F08BF5FEA6F
:10056000500C50F1000041EB045141EA050130BD4F
:100570005FEA4C0C404141EB0101013C28BFB1F561
:10058000801FE9D291F0000F04BF01460020B1FAAC
:1005900081F308BF2033A3F10B03B3F120020CDA7F
:1005A0000C3208DD02F1140CC2F10C0201FA0CF05D
:1005B00021FA02F10CE002F11402D8BFC2F1200CC2
:1005C00001FA02F120FA0CFCDCBF41EA0C01904078
:1005D000E41AA2BF01EB0451294330BD6FEA0404C1
:1005E0001F3C1CDA0C340EDC04F11404C4F12002AC
:1005F00020FA04F001FA02F340EA030021FA04F3BE
:1006000045EA030130BDC4F10C04C4F1200220FA14
:1006100002F001FA04F340EA0300294630BD21FA52
:1006200004F0294630BD94F0000F83F4801306BF18
:1006300081F480110134013D4EE77FEA645C18BF0C
:100640007FEA655C29D094EA050F08BF90EA020FA3
:1006500005D054EA000C04BF1946104630BD91EA9B
:10066000030F1EBF0021002030BD5FEA545C05D19E
:100670004000494128BF41F0004130BD14F58004DD
:100680003CBF01F5801130BD01F0004545F0FE4151
:1006900041F470014FF0000030BD7FEA645C1ABF86
:1006A000194610467FEA655C1CBF0B46024650EABD
:1006B000013406BF52EA033591EA030F41F40021E9
:1006C00030BD00BF90F0000F04BF0021704730B56F
:1006D0004FF4806404F132044FF000054FF0000144
:1006E00050E700BF90F0000F04BF0021704730B505
:1006F0004FF4806404F1320410F0004548BF4042DA
:100700004FF000013EE700BF42004FEAE2014FEA2E
:1007100031014FEA02701FBF12F07F4393F07F4F09
:1007200081F06051704732F07F4208BF704793F00C
:100730007F4F04BF41F40021704730B54FF460741F
:1007400001F0004521F000411CE700BF50EA010222
:1007500008BF704730B54FF000050AE050EA0102CB
:1007600008BF704730B511F0004502D5404261EB3B
:1007700041014FF4806404F132045FEA915C3FF47C
:10078000D8AE4FF003025FEADC0C18BF03325FEA19
:10079000DC0C18BF033202EBDC02C2F1200300FACA
:1007A00003FC20FA02F001FA03FE40EA0E0021FAEF
:1007B00002F11444BDE600BF70B54FF0FF0C4CF4DD
:1007C000E06C1CEA11541DBF1CEA135594EA0C0F8F
:1007D00095EA0C0F00F0DEF82C4481EA030621EACA
:1007E0004C5123EA4C5350EA013518BF52EA033505
:1007F00041F4801143F4801338D0A0FB02CE4FF0B7
:100800000005E1FB02E506F00042E0FB03E54FF0E6
:100810000006E1FB03569CF0000F18BF4EF0010EDE
:10082000A4F1FF04B6F5007F64F5407404D25FEADA
:100830004E0E6D4146EB060642EAC62141EA55518D
:100840004FEAC52040EA5E504FEACE2EB4F1FD0CCF
:1008500088BFBCF5E06F1ED8BEF1004F08BF5FEA4D
:10086000500E50F1000041EB045170BD06F00046FF
:1008700046EA010140EA020081EA0301B4EB5C04AC
:10088000C2BFD4EB0C0541EA045170BD41F48011A4
:100890004FF0000E013C00F3AB8014F1360FDEBFC9
:1008A000002001F0004170BDC4F10004203C35DAA5
:1008B0000C341BDC04F11404C4F1200500FA05F328
:1008C00020FA04F001FA05F240EA020001F00042C9
:1008D00021F0004110EBD37021FA04F642EB06013F
:1008E0005EEA430E08BF20EAD37070BDC4F10C0469
:1008F000C4F1200500FA04F320FA05F001FA04F22D
:1009000040EA020001F0004110EBD37041F1000118
:100910005EEA430E08BF20EAD37070BDC4F1200523
:1009200000FA05F24EEA020E20FA04F301FA05F28B
:1009300043EA020321FA04F001F0004121FA04F233
:1009400020EA020000EBD3705EEA430E08BF20EA03
:10095000D37070BD94F0000F0FD101F0004640003D
:1009600041EB010111F4801F08BF013CF7D041EABF
:10097000060195F0000F18BF704703F000465200C3
:1009800043EB030313F4801F08BF013DF7D043EA94
:100990000603704794EA0C0F0CEA135518BF95EA4A
:1009A0000C0F0CD050EA410618BF52EA4306D1D1D1
:1009B00081EA030101F000414FF0000070BD50EAF0
:1009C000410606BF1046194652EA430619D094EA7A
:1009D0000C0F02D150EA013613D195EA0C0F05D164
:1009E00052EA03361CBF104619460AD181EA0301B8
:1009F00001F0004141F0FE4141F470014FF0000070
:100A000070BD41F0FE4141F4780170BD70B54FF00A
:100A1000FF0C4CF4E06C1CEA11541DBF1CEA13558A
:100A200094EA0C0F95EA0C0F00F0A7F8A4EB05046C
:100A300081EA030E52EA03354FEA013100F0888063
:100A40004FEA03334FF0805545EA131343EA12632C
:100A50004FEA022245EA111545EA10654FEA0026E1
:100A60000EF000419D4208BF964244F1FD0404F59A
:100A7000407402D25B084FEA3202B61A65EB0305F6
:100A80005B084FEA32024FF480104FF4002CB6EBB3
:100A9000020E75EB030E22BFB61A754640EA0C0033
:100AA0005B084FEA3202B6EB020E75EB030E22BF73
:100AB000B61A754640EA5C005B084FEA3202B6EBB4
:100AC000020E75EB030E22BFB61A754640EA9C0073
:100AD0005B084FEA3202B6EB020E75EB030E22BF43
:100AE000B61A754640EADC0055EA060E18D04FEA01
:100AF000051545EA16754FEA06164FEAC30343EAA1
:100B000052734FEAC2025FEA1C1CC0D111F4801F6D
:100B10000BD141EA00014FF000004FF0004CB6E766
:100B200011F4801F04BF01430020B4F1FD0C88BF05
:100B3000BCF5E06F3FF6AFAEB5EB030C04BFB6EB10
:100B4000020C5FEA500C50F1000041EB045170BD03
:100B50000EF0004E4EEA113114EB5C04C2BFD4EB30
:100B60000C0541EA045170BD41F480114FF0000EB4
:100B7000013C90E645EA060E8DE60CEA135594EA30
:100B80000C0F08BF95EA0C0F3FF43BAF94EA0C0F33
:100B90000AD150EA01347FF434AF95EA0C0F7FF4A8
:100BA00025AF104619462CE795EA0C0F06D152EAFC
:100BB00003353FF4FDAE1046194622E750EA4106E0
:100BC00018BF52EA43067FF4C5AE50EA41047FF4F1
:100BD0000DAF52EA43057FF4EBAE12E74FEA410254
:100BE000B2F1E04324BFB3F5001CDCF1FE5C0DD98B
:100BF00001F0004C4FEAC0024CEA5070B2F1004FD5
:100C000040EB830008BF20F00100704711F0804FD7
:100C100021D113F13872BCBF01F00040704741F49C
:100C200080114FEA5252C2F11802C2F1200C10FAA0
:100C30000CF320FA02F018BF40F001004FEAC12384
:100C40004FEAD32303FA0CFC40EA0C0023FA02F328
:100C50004FEA4303CCE77FEA625307D150EA0133FE
:100C60001EBF4FF0FE4040F44000704701F00040CE
:100C700040F0FE4040F40000704700BF4FF0FF0C12
:100C80001CEAD0521EBF1CEAD15392EA0C0F93EA21
:100C90000C0F6FD01A4480EA010C400218BF5FEAC3
:100CA00041211ED04FF0006343EA501043EA511136
:100CB000A0FB01310CF00040B1F5000F3EBF490030
:100CC00041EAD3715B0040EA010062F17F02FD2A34
:100CD0001DD8B3F1004F40EBC25008BF20F0010017
:100CE000704790F0000F0CF0004C08BF49024CEA2E
:100CF000502040EA51207F3AC2BFD2F1FF0340EAC0
:100D0000C250704740F400004FF00003013A5DDC30
:100D100012F1190FDCBF00F000407047C2F1000271
:100D2000410021FA02F1C2F1200200FA02FC5FEA5E
:100D3000310040F1000053EA4C0308BF20EADC70A8
:100D4000704792F0000F00F0004C02BF400010F41A
:100D5000000F013AF9D040EA0C0093F0000F01F0C7
:100D6000004C02BF490011F4000F013BF9D041EAE9
:100D70000C018FE70CEAD15392EA0C0F18BF93EAEB
:100D80000C0F0AD030F0004C18BF31F0004CD8D115
:100D900080EA010000F00040704790F0000F17BF9C
:100DA00090F0004F084691F0000F91F0004F14D0E2
:100DB00092EA0C0F01D142020FD193EA0C0F03D13A
:100DC0004B0218BF084608D180EA010000F000403D
:100DD00040F0FE4040F40000704740F0FE4040F418
:100DE000400070474FF0FF0C1CEAD0521EBF1CEAB7
:100DF000D15392EA0C0F93EA0C0F69D0A2EB0302D5
:100E000080EA010C49024FEA402037D04FF080536E
:100E100043EA111143EA10130CF000408B4238BF33
:100E20005B0042F17D024FF4000C8B4224BF5B1A41
:100E300040EA0C00B3EB510F24BFA3EB510340EA8F
:100E40005C00B3EB910F24BFA3EB910340EA9C003D
:100E5000B3EBD10F24BFA3EBD10340EADC001B01AD
:100E600018BF5FEA1C1CE0D1FD2A3FF650AF8B4251
:100E700040EBC25008BF20F0010070470CF0004C5E
:100E80004CEA50207F32C2BFD2F1FF0340EAC25089
:100E9000704740F400004FF00003013A37E792F04A
:100EA000000F00F0004C02BF400010F4000F013AA8
:100EB000F9D040EA0C0093F0000F01F0004C02BFA3
:100EC000490011F4000F013BF9D041EA0C0195E70C
:100ED0000CEAD15392EA0C0F08D142027FF47DAFA5
:100EE00093EA0C0F7FF470AF084676E793EA0C0F95
:100EF00004D14B023FF44CAF08466EE730F0004C93
:100F000018BF31F0004CCAD130F000427FF45CAF22
:100F100031F000437FF43CAF5FE700BF42000ED2E8
:100F2000B2F1FE4F0BD34FF09E03B3EB126209D424
:100F30004FEA002343F0004323FA02F070474FF0DA
:100F40000000704712F1610F01D1420202D14FF04F
:100F5000FF3070474FF00000704700BF53B94AB9E7
:100F6000002908BF00281CBF4FF0FF314FF0FF30B1
:100F700000F084B9ADF1080C6DE904CE00F006F87C
:100F8000DDF804E0DDE9022304B070472DE9F04FFD
:100F9000099E0D4604468A46002B40F085808A4211
:100FA000174644D9B2FA82F24AB1C2F1200105FAD9
:100FB00002F39740944020FA01F141EA030A4FEA14
:100FC00017484FEA144C1FFA87F9BAFBF8FE08FBE2
:100FD0001EA30EFB09F14CEA0343994207D9FB1803
:100FE0000EF1FF3002D2994200F230818646591A42
:100FF000A3B2B1FBF8F008FB101100FB09F943EABA
:101000000144A14507D93C1900F1FF3302D2A145A3
:1010100000F219811846A4EB090440EA0E400021B1
:101020001EB1D4400023C6E90043BDE8F08F02B9E9
:10103000FFDEB2FA82F2002A51D1CB1B4FEA174EE3
:101040001FFA87F80121250CB3FBFEFC0EFB1C30B8
:1010500008FB0CF945EA0045A9450BD97D190CF1AF
:10106000FF332CBF01200020A94502D9002800F041
:10107000F1809C46A5EB0905A3B2B5FBFEF00EFB83
:10108000105508FB00F843EA0544A04507D93C1970
:1010900000F1FF3302D2A04500F2D2801846A4EB43
:1010A000080440EA0C40BBE78B4208D9002E00F050
:1010B000BE800021C6E900050846BDE8F08FB3FAFE
:1010C00083F100294DD1AB42C0F0B480824240F29E
:1010D000B1800846002EA8D0C6E9004AA5E7C2F1B3
:1010E0002000974001FA02F34FEA174EC14024FA5C
:1010F00000F51FFA87F894401D43B1FBFEF02B0C5E
:101100000EFB101100FB08FC43EA01439C450ED97D
:10111000FB1800F1FF312CBF4FF001094FF000091F
:101120009C4503D9B9F1000F00F098800846A3EB65
:101130000C03ADB2B3FBFEF10EFB113301FB08FC57
:1011400045EA0345AC4507D97D1901F1FF3302D2C9
:10115000AC4500F28A801946A5EB0C0341EA004138
:1011600071E7C1F120048B4002FA01F705FA01FC96
:10117000E24020FA04F8E54000FA01FE134348EA91
:101180000C024FEA13484FEA124C1FFA83F9B5FBE1
:10119000F8FA08FB1A550AFB09F04CEA054C6045C1
:1011A0000ED913EB0C0C0AF1FF352CBF4FF0010BDD
:1011B0004FF0000B604502D9BBF1000F51D0AA4699
:1011C000ACEB000C92B2BCFBF8F008FB10CC00FBBF
:1011D00009F942EA0C4CE14507D913EB0C0C00F17C
:1011E000FF3201D2E14543D8104640EA0A40ACEB59
:1011F000090CA0FB0789CC4545464A4602D306D1D7
:10120000C64504D20138B8EB070569EB030296B373
:10121000BEEB05036CEB020C23FA01F20CFA04F4AA
:101220002CFA01F300211443C6E90043FDE63146E0
:101230003046FAE6841A65EB030301209A4649E733
:1012400002383C442BE702383C44E4E6AEF1020E9F
:101250003B44CCE6ACF1020C3D440BE702383B4486
:1012600065E7AAF1020A9C44AAE702393D4473E704
:1012700002389C44B9E73146D7E600BF704700BF4B
:101280004FF0FF3C06E000BF4FF0010C02E000BF52
:101290004FF0010C4DF804CD4FEA410C7FEA6C5C35
:1012A0004FEA430C18BF7FEA6C5C1BD001B050EAD8
:1012B000410C0CBF52EA430C91EA030F02BF90EAC3
:1012C000020F0020704710F1000F91EA030F58BF82
:1012D000994208BF90422CBFD8176FEAE37040F0E4
:1012E000010070474FEA410C7FEA6C5C02D150EA82
:1012F000013C07D14FEA430C7FEA6C5CD6D152EA3D
:10130000033CD3D05DF8040B704700BF8446104601
:1013100062468C461946634600E000BF01B5FFF700
:10132000B7FF002848BF10F1000F01BD4DF808EDD0
:10133000FFF7F4FF0CBF012000205DF808FB00BFA1
:101340004DF808EDFFF7EAFF34BF012000205DF8FB
:1013500008FB00BF4DF808EDFFF7E0FF94BF012048
:1013600000205DF808FB00BF4DF808EDFFF7CEFF49
:1013700094BF012000205DF808FB00BF4DF808ED88
:10138000FFF7C4FF34BF012000205DF808FB00BF59
:101390004FEA410C7FEA6C5C02D150EA013C0AD171
:1013A0004FEA430C7FEA6C5C02D152EA033C02D163
:1013B0004FF0000070474FF0010070474FEA4102C4
:1013C00012F5001215D211D56FF47873B3EB625297
:1013D00012D94FEAC12343F0004343EA505311F0BE
:1013E000004F23FA02F018BF404270474FF0000050
:1013F000704750EA013005D111F0004008BF6FF08E
:10140000004070474FF00000704700BF10F8012BFC
:1014100011F8013B012A28BF9A42F7D0D01A704731
:10142000034613F8012B002AFBD1181A0138704724
:101430002DE9F04F164699B01F46446A0546DDF87F
:101440009480CDE9046774B910201BF0BDFA024600
:10145000686220B9A84BEA21A8481AF02BF9C0E924
:1014600001440460C4606B6A196851B15A68012371
:10147000284693404A608B601BF0EEFA6B6A0022AC
:101480001A603B1EB7BF23F00043002301220593DF
:10149000A8BFC8F80030DDF81490994BB8BFC8F861
:1014A000002033EA090319D142F20F73249A136022
:1014B000C9F31303334300F07E85269B53B9914B48
:1014C00022E0914B08930833269A1360089819B0CC
:1014D000BDE8F08F8B4B08930333F5E7DDE9043467
:1014E0000022CDE90C34DDE90C010023FFF71EFFDB
:1014F000804658B10123249A1360269B002B00F0EC
:10150000578582481860431E0893DFE716ABC9F37E
:101510000A542846019317AB0093DDE90C231BF016
:101520001BFD8246002C7CD00D9BA4F2FF34CDF82D
:101530004C80C3F31303DDE90C0143F07F5141F408
:1015400040110022724BFEF77FFF65A3D3E9002311
:10155000FFF732F964A3D3E90023FEF777FF0646CD
:101560000F462046FFF7BEF861A3D3E90023FFF73B
:1015700023F902460B4630463946FEF767FF06461A
:101580000F46FFF71BFF00228146002330463946F5
:10159000FFF7D6FE48B14846FFF7A4F832463B466F
:1015A000FFF7C4FE08B909F1FF39B9F1160F56D893
:1015B000584B03EBC903DDE90C01D3E90023FFF726
:1015C000BFFE00284DD009F1FF3900230F93169B71
:1015D0001C1B631E099349BFC4F10103002306933A
:1015E000002354BF06930993B9F1000F3BDB099B1D
:1015F000CDF838904B44099300230A93229B092B82
:1016000000F28C80052BC5BF043B002401242293EB
:10161000229B023B032B00F28D80DFE803F02E506B
:101620004E5CDDE916431C4404F23243202BC6BF56
:10163000C3F1400304F21240C3F1200304F1FF346C
:10164000C5BF09FA03F326FA00F006FA03F01843BF
:10165000FFF738F80123A1F1F871139371E7012323
:10166000B4E70F90B3E7069BA3EB09030693C9F118
:1016700000030A9300230E93C0E700230B93239BE0
:10168000002B5ADC4FF0010B5B46CDF808B0CDF8CB
:101690008CB00022686A4260042202F1140641689C
:1016A0009E4250D928461BF097F9089000284ED149
:1016B000194B02464FF4D571CEE60123DEE7002335
:1016C0000B93239B09EB030B0BF10103012B0293FB
:1016D000B8BF0123DDE70123F2E700BFAFF30080CD
:1016E00061436F63A787D23FB3C8608B288AC63F28
:1016F000FB799F501344D33F5EB2040075B20400DF
:101700000000F07F5AB2040051B204008A6A04005B
:101710000000F83F50500400F1B2040001240023FF
:101720000B9422934FF0FF3B00221223CDF808B018
:101730002392AEE701230B93F4E7DDF88CB05B4610
:10174000CDF808B0A5E7013152004160A5E76B6A0A
:10175000089A1A60029B0E2B00F2A880002C00F061
:10176000A580B9F1000F34DD09F00F03994A19F48F
:10177000807F02EBC303D3E90034CDE910344FEA94
:10178000291416D0944B04F00F040327D3E908233F
:10179000DDE90C01FFF73AF9CDE904018E4E54B9A9
:1017A000DDE91023DDE90401FFF730F9CDE904019B
:1017B00029E00227F2E7E10708D50137DDE910014A
:1017C000D6E90023FEF7F8FFCDE9100164100836D2
:1017D000E5E700F0A580C9F100047E4B7E4E0227AC
:1017E00004F00F02241103EBC203DDE90C01D3E97D
:1017F0000023FEF7E1FF0023CDE90401002C40F0B7
:101800008480002BD2D10F9B002B00F08B80002214
:10181000DDE90434CDE91034DDE910016F4BFFF749
:101820008FFD00287ED0029B002B7BD0BBF1000FE8
:1018300038DD09F1FF3801375C460022684BDDE9ED
:101840001001FEF7B9FFCDE904013846FEF74AFF63
:10185000DDE90423FEF7B0FF0022624BFEF7F6FD40
:10186000A1F15076CDE910011196002C5DD1002236
:101870005D4BDDE90401FEF7E7FD02460B46CDE9CD
:101880000423109A3346FFF779FD002840F09C822C
:10189000109A06F10043DDE90401FFF751FD00282D
:1018A00040F09082DDE90C34CDE90434179B002B25
:1018B000C0F25281B9F10E0F00F34E81454B03EB9C
:1018C000C903D3E90034CDE90634239B002B80F211
:1018D000DA80029B002B00F3D68040F07282002257
:1018E000414BDDE90601FEF767FFDDE90423FFF761
:1018F0003BFD029C2646002840F04882089F312389
:1019000009F1010907F8013B44E2E20705D5013777
:10191000D6E90023FEF750FF0123641008366DE777
:10192000022770E7C846029C8FE70899294B21449B
:1019300003EBC40312910B99DDE9106753E902230D
:10194000002955D000202949FFF760F83B46324670
:10195000FEF77AFD089FCDE91001DDE90401FFF7EC
:101960002DFD0446FEF7BEFE02460B463034DDE98F
:101970000401FEF769FD02460B4607F8014BCDE96D
:101980000423DDE91023FFF7DBFC002873D10020DE
:101990001249DDE90423FEF757FDDDE91023FFF7C7
:1019A000CFFC002840F0B580129B9F423FF47AAFF5
:1019B00000220B4BDDE91001FEF7FEFE0022084B72
:1019C000CDE91001DDE90401FEF7F6FECDE90401E1
:1019D000C3E700BF50500400285004000000F03F4F
:1019E0000000244000001C40000014400000E03FC4
:1019F00030463946FEF7E0FE129B089C1493CDE971
:101A00001001DDE90401FFF7D9FC1590FEF76AFE2D
:101A100002460B46DDE90401FEF716FD159B06465E
:101A20000F463033002204F8013B129B9C4224D124
:101A3000B14BDDE91001FEF709FD02460B463046C9
:101A40003946FFF79BFC002862D10020AA49DDE956
:101A50001023FEF7F9FC02460B4630463946FFF7E5
:101A60006FFC00283FF41EAF149F7B1E149317F8E1
:101A7000013C302BF8D0C1463AE0A04BFEF79CFE6B
:101A8000CDE90401BDE7089FDDE90623DDE9040196
:101A9000FEF7BCFFFFF792FC0446FEF723FE04F1BD
:101AA0003006DDE90623FEF787FE0B460246DDE938
:101AB0000401FEF7C9FC07F8016B089E029BBE1BE0
:101AC000B3423AD102460B46FEF7C0FC02460B4633
:101AD000CDE90223DDE90623FFF750FC58BBDDE921
:101AE0000623DDE90201FFF721FC08B1E10722D45A
:101AF000284651461AF0B0FF002309F101003B705F
:101B0000249B1860269B002B3FF4E0AC1F60DDE4B3
:101B100027463B461F4613F8012D392A07D1089A5C
:101B20009A42F7D13022089908F101080A701A7810
:101B300001321A709FE7C846EBE700226F4BFEF7B1
:101B40003BFE02460B46CDE9042300220023FFF7AB
:101B5000EDFB002898D0CBE70B9A002A00F0D0804C
:101B6000229A012A00F3AE80139A002A00F0A68080
:101B700003F233430A9C069F069A012128461A4421
:101B80000692099A1A4409921AF0D2FF0646002FCB
:101B90000CDD099B002B09DDBB42069AA8BF3B4622
:101BA000D21AFF1A0692099AD31A09930A9BF3B123
:101BB0000B9B002B00F0A880002C10DD3146224644
:101BC00028461BF071F852460146064628461AF090
:101BD000C5FF804651462846C2461AF03DFF0A9B83
:101BE0001A1B04D0514628461BF05EF8824601219C
:101BF00028461AF09DFF0E9B0446002B40F386807A
:101C00001A46014628461BF04FF8229B0446012B3A
:101C10007FDD4FF00008236904EB8303186922F08D
:101C20002CFEC0F12000099B184410F01F0000F0AA
:101C30009280C0F12003042B40F38A80C0F11C0085
:101C4000069B074403440693099B03440993069BA0
:101C5000002B05DD51461A4628461BF07FF88246C8
:101C6000099B002B05DD21461A4628461BF076F815
:101C700004460F9B002B70D02146504622F04BFEAD
:101C800000286ADA002351460A2228461AF006FF85
:101C90000B9B09F1FF398246002B00F093813146FE
:101CA00000230A2228461AF0F9FEBBF1000F06466F
:101CB00000F39380229B022B57DC8EE0169BC3F12E
:101CC000360357E7029B5C1E0A9BA342B7BF0A9BE1
:101CD0001C1B0A94E21ABFBF0E9B00249B180E9394
:101CE000029B002BBBBF069B029A069F9F1AACBFAC
:101CF000029B002340E700BF0000E03F00002440BB
:101D00000A9C069F0B9E42E70A9A6BE7229B012BD7
:101D100019DC049BBBB9059BC3F313039BB9059B5B
:101D200023F000431B0D1B0583B1069B4FF00108F8
:101D300001330693099B013309930E9B002B7FF41B
:101D40006AAF01206FE74FF00008F6E79846F4E726
:101D50003FF47DAF18461C3072E7029B002B36DC47
:101D6000229B022B33DDDDF808B0BBF1000F0DD153
:101D700021465B46052228461AF090FE014604469D
:101D8000504622F0C8FD00283FF7B8AD239B089FBE
:101D90006FEA03094FF00008214628461AF05CFE5E
:101DA000002E3FF4A5AEB8F1000F05D0B04503D02A
:101DB000414628461AF050FE314628461AF04CFE9D
:101DC00096E600242646E1E7C146264696E50B9BAB
:101DD000DDF808B0002B00F0FC80002F05DD314657
:101DE0003A4628461AF0BAFF0646B8F1000F5CD012
:101DF000716828461AF0F0FD074628B97F4B024665
:101E000040F2EA21FFF728BB326906F10C010C30E1
:101E10000232920022F0E5F90122394628461AF0F2
:101E20009DFF089BB046064601330293089B5B4426
:101E30000A93049B03F001030993029B2146504639
:101E400003F1FF3B22F014FC034641460490504648
:101E500030330B9322F05FFD324606902146284630
:101E60001AF0E8FFC26807460B9B02BB01465046CA
:101E700022F051FD0B9B024639462846CDE90B3234
:101E80001AF0EAFD229B0C9A029F43EA0201099B89
:101E90000B430B9B0DD1392B27D0069A002A01DD6D
:101EA000049B31338BF8003076E73046B9E70122E6
:101EB000E2E70699002904DB2298014309980143CF
:101EC00020D1002AEEDD51460122284602931AF065
:101ED00045FF2146824622F01EFD0028029B02DCBF
:101EE000E0D1DA07DED5392BDAD139238BF800308F
:101EF0003B461F46013B17F8012C392A50D00132CE
:101F00001A7049E7002A03DD392BEED00133C9E707
:101F1000029A0A9902F8013C8A422AD051460023CB
:101F20000A2228461AF0BAFDB04582464FF0000357
:101F30004FF00A024146284607D11AF0AFFD80460D
:101F40000646029B0133029377E71AF0A7FD31465C
:101F5000804600230A2228461AF0A0FD0646F0E734
:101F6000BBF1000F089A4FF00008CCBF5F46012775
:101F7000174451460122284602931AF0EFFE2146EB
:101F8000824622F0C8FC0028B2DC02D1029BDB07AB
:101F9000AED43B461F4613F8012D302AFAD0FBE69B
:101FA000089A9A42A5D1312309F101091370F3E689
:101FB000134BFFF7A9BA269B002B7FF482AA114B83
:101FC000FFF7A2BABBF1000F03DC229B022B3FF705
:101FD000CCAE089F2146504622F04AFB089A00F1F9
:101FE000300307F8013BBA1A9345B9DD5146002387
:101FF0000A2228461AF052FD8246EBE7F1B20400AD
:10200000896A040051B204000149024821F062BD0E
:1020100038710120984C0120F8B51F4B1F4C204E01
:10202000E41AE4081F4DA40131781F4844F003026C
:102030001CF076F8286883684FF400529F690621E7
:102040000023B84728688368DB6913B10022174969
:102050009847286802698168136823F04003136079
:102060000B684FF4807206219847337853B101F022
:10207000FBF8014670B10E4844F00102BDE8F8409B
:102080001CF04EB801F056F8014618B1094844F06A
:102090000102F3E7F8BD00BF584E0400604E040093
:1020A000C4C50120547101209859040048710120D1
:1020B000B1590400CC590400054A064B0146D21A16
:1020C000D2089201044842F001021CF029B800BF76
:1020D000604E0400584E0400E759040038B5044629
:1020E0002D4817F0C5FE2D4D286058B92C4B2D49B1
:1020F0002D48C91AC908890141F00101BDE83840DD
:102100001CF001B802698168136823F04003136072
:102110000B684FF4887206219847014658B1214A4E
:102120001F4B2248D21AD208920142F00102BDE8A8
:1021300038401BF0F5BF1E491E4B28684B604023FA
:102140008B608368DB6963B101229847014658B10F
:10215000144A134B1848D21AD208920142F00102D5
:10216000E5E76FF08501F3E72868836806219D693C
:102170004FF480424FF40033A847014640B1094A6A
:10218000074B0E48D21AD208920142F00102CEE764
:102190000B4B1C7038BD00BF0B5A0400547101205A
:1021A000584E0400604E0400125A0400245A0400E1
:1021B00048710120092002003C5A04005A5A0400C8
:1021C000C4C501200C22094BC3F81822D3F81822E9
:1021D00042F44032C3F818224FF040230122C3F8E2
:1021E0000025BFF34F8F20BFFDE700BF00258440CF
:1021F00010B50EF06DFB2E4B044698421ADC023BE4
:1022000098423FDC002851D0A0F18863013B012BAC
:1022100042D8284A284B0146D21AD20892012748B0
:1022200042F001021BF07CFF0122254B1A70254B66
:102230001C6014E0244B98422ED11F4B1D492348AB
:10224000C91AC908890141F003011BF05CFF05228E
:102250001F4B1A7000231A4A13701A4A136000F0B9
:1022600023FA154B13491B48C91AC908890141F0C3
:1022700002011BF048FF08F003FFBDE810400120F9
:1022800008F048BC0B4A0C4B0146D21AD208920106
:10229000114842F00102C5E7064A074B2146D21A0F
:1022A000D20892010D4842F00102BBE710BD00BF09
:1022B00004004004604E0400584E04007B5A0400A1
:1022C000C6C501205871012001005005A75A04001D
:1022D000C5C501202A5B0400CE5A0400FB5A040045
:1022E00037B5214B214C2248E41AE408A40144F0FC
:1022F00003011BF008FF00F097F9014638B11D48B3
:1023000044F0010203B0BDE830401BF009BF1A4B96
:102310001D78012D09D0FFF76BFF00F0A5FF0146E6
:1023200098B1164844F00102ECE71DF0EEF91449AB
:102330000B78002BF1D0134A134B10B115701860B5
:10234000EBE7052510700D70F9E700900E234FF4B0
:1023500000620E490E4818F0C9FA0E490E4803B043
:10236000BDE8304021F0ADBB584E0400604E040083
:10237000375B0400485B0400C7C50120B159040065
:10238000C5C50120C6C5012058710120C00F02201B
:10239000984C01201920020038710120F8B505463B
:1023A00008460E46FFF73CF804462846FFF738F883
:1023B000844217D100230C4FA34201DB0120F8BD5A
:1023C000E95CCA5D02F00302022AF25C08BF203910
:1023D000B85C00F00300022808BF203A914201D106
:1023E0000133E9E70020EAE712B10400F8B5064638
:1023F00008460F46FFF714F804463046FFF710F87A
:10240000844223D800251348A5420DDB3046FFF750
:1024100007F80234A0421BD9705D00F0FD00A0F166
:102420003D0358425841F8BD725D135C03F003034D
:10243000022B7B5D08BF203AC15C01F00301022939
:1024400008BF203B9A4201D10135DDE70020EAE7D1
:102450000120E8E712B104002DE9F8430D4690464B
:102460000746A8B1A2B1B3EB410F4FEA41060FDB1B
:102470000024DFF82490A54202DC3046BDE8F88352
:102480003A5D08EB4400494619F0F8FD0134F2E7E3
:102490006FF01506F1E700BF479B0400F0B5A1B04F
:1024A00006460023802269460F480FF021FB0746AD
:1024B00010B1002021B0F0BD68460C4922F08EF822
:1024C00004460028F5D001342046084922F086F859
:1024D0000028EED0051B2A462146304621F081FE19
:1024E00001207755E6E700BF6C5B04002A73040007
:1024F000F8B50C463849074615461E46FEF786FFD6
:1025000078B9012C02D06FF01500F8BD224633498E
:102510003046A847002802DC6FF00100F5E70020F4
:10252000F3E738462E49FEF771FF20B9012CEAD1B6
:1025300022462C49ECE738462B49FEF767FF20B9C5
:10254000012CE0D122462949E2E738462849FEF726
:102550005DFF20B9042CD6D122462649D8E738465B
:102560002549FEF753FF20B9012CCCD1224623493F
:10257000CEE738462249FEF749FF20B9042CC2D1E4
:1025800022462049C4E738461F49FEF73FFF20B9DD
:10259000012CB8D122461D49BAE738461C49FEF73E
:1025A00035FF20B9012CAED122461A49B0E7384692
:1025B0001949FEF72BFF20B9012CA4D1012217499C
:1025C000A6E738461649FEF721FF0028A4D1012CC2
:1025D00099D1224613499BE7CB5B0400C7C5012074
:1025E000F75B0400C5C50120255C0400C6C50120B9
:1025F000555C040058710120815C0400C8C50120AD
:10260000955C04005C710120A75C040060710120EE
:10261000B75C040061710120CA5C04006271012092
:10262000DD5C04006371012010B509F0FDFC044677
:1026300060B1164A164B0146D21AD20892011548CB
:1026400042F001021BF06CFD204610BD124809F05B
:10265000D3FB044648B10D4A0D4B0146D21AD208AD
:1026600092010E4842F00102ECE70D4809F08EFBA2
:1026700004460028E8D0054A054B0146D21AD20884
:102680009201084842F00102DCE700BF484F040015
:10269000584E0400775B0400C84501208F5B04009E
:1026A000AB5B0400AF5B040010B501222349244852
:1026B00009F032FB044660B1224A234B0146D21A8C
:1026C000D2089201214842F001021BF029FD204668
:1026D00010BD01221E491F4809F01EFB044648B1E7
:1026E000184A194B0146D21AD20892011A4842F0F0
:1026F0000102EAE701221949194809F00DFB0446D5
:1027000048B1104A104B0146D21AD208920115481E
:1027100042F00102D9E704221349144809F0FCFAF7
:1027200004460028D3D0074A074B0146D21AD208E4
:1027300092010F4842F00102C7E700BFC7C5012060
:10274000C75B0400484F0400584E0400D55B0400EA
:10275000C5C50120F35B0400025C0400C6C501206E
:10276000215C0400315C040058710120515C0400BC
:102770005F5C04000023044A1370044A1370044A87
:102780001370044A13607047C7C50120C5C50120F6
:10279000C6C501205871012008B50122124913480D
:1027A00009F0BAFAF0B904221149124809F0B4FA52
:1027B000C0B901221049114809F0AEFA90B90122BE
:1027C0000F49104809F0A8FA60B901220E490F48D4
:1027D00009F0A2FA30B9BDE8084001220C490D48C1
:1027E00009F09ABA08BD00BFC8C501207D5C04008D
:1027F0005C710120915C040060710120A35C040005
:1028000061710120B35C040062710120C65C0400A8
:1028100063710120D95C04000D4B10B50D4C0E48BE
:10282000E41AE408A40144F003011BF06CFC0B4B18
:10283000D3E900239A4204D0BDE81040084818F0BC
:102840004FB844F002010748BDE810401BF05BBCE4
:10285000584E0400704E0400F75C040080710120A3
:10286000A07101200A5D0400F8B507460E464FF03E
:10287000FF324FF0FF331E4817F022FF304621F0A1
:1028800076FC1C4D0446286080B91B4B1B491C4834
:10289000C91AC908890141F002011BF034FC14482F
:1028A00017F0E8FE6FF00B042046F8BD32463946BB
:1028B00021F097FC134B1868836821465F68324605
:1028C0004FF0FF33B84704460028EDD00A4B0B4ABF
:1028D0000146D21AD208920142F002020A481BF0C5
:1028E0001FFC286821F03CFC014817F0C3FEDBE721
:1028F0005C4C0120B4710120584E0400704E04005D
:102900001C5D0400B07101202A5D0400104B10B55D
:10291000186883684FF48072DC680E490123A04771
:10292000044680B10C4B0D4A0146D21AD2089201DE
:102930000B4842F001021BF0F3FB0D210948FFF7A1
:1029400093FF204610BD084B1870084B1880F8E71D
:10295000B071012090DC0120584E0400704E04003C
:102960003D5D0400505D0400C9D5012074C50120FF
:1029700008B5FFF7CBFF0022014B1A7008BD00BF5E
:102980008FDC012038B54FF40062134913481BF067
:1029900056FB054688B1124B124C0146E41AE40876
:1029A000A401114844F003021BF0BAFB0F4B1B6853
:1029B0005BB12A460020084998470D4C23781BB18B
:1029C000FFF7A4FF0023237038BD0A4844F002013A
:1029D0001BF099FBF1E700BFC9CD012080710120F8
:1029E000584E0400704E04005E5D04009C7101208E
:1029F000CBD501206A5D04002DE9F04F0B780C4621
:102A000085B0062B73D8DFE813F00700110025000E
:102A10005201AB01C201AF01B34B186821F0A0FB1A
:102A2000B24805B0BDE8F04F17F024BEAE4B1868B1
:102A300021F096FBAD4817F01DFEAD4BAD49AE48F9
:102A4000C91AC908890141F0030105B0BDE8F04F7A
:102A50001BF059BBA94BAA4E93F800B0BBF1000F75
:102A600063D1A44FA24BB6F80080FF1AA54DDFF842
:102A7000E892FF083388E2681344434504D832885B
:102A8000E3681344338032E0636813F808202B684E
:102A9000082A01D07F2A05D10BB1013B2B6008F138
:102AA0000108E7E799F80010DFF8B0A211BB0A2A85
:102AB00020D1FBB1581E1AF800C0BCF10D0F19D17E
:102AC00028604FF0000B904B18681AF058FD2B68E7
:102AD0008E4A8F480AF803B0138017F001FF8D4B20
:102AE00089F800B01B78C5F800B0002BD7D005B02E
:102AF000BDE8F08F0AF803200133B3F5805F2B6047
:102B00000CD3B901844841F001011BF0FCFA012209
:102B10002B68013B2B607F4B1A70D2E7222ABED173
:102B200081F0010189F80010B9E7BBF1010F40F015
:102B3000B3804A68B6F8008078489044CF68FEF7C2
:102B40006FFC81461AF020FD754D2A68AA46831A4B
:102B500002936B68C5E9000161EB03030393DDE9B0
:102B60000223B2F57A7F73F1000338DA6D4D2B78CA
:102B70009BB16D4821F084F9002368494A466B48AF
:102B80002B701BF0F2F95B49594B6948C91AC90807
:102B9000890141F003011BF0B6FA664D2B8813B191
:102BA000654821F06DF9DFF884913A464146484680
:102BB0001BF0DBF98742024636D04D494D4B5F484A
:102BC0005B1ADB089B01394643F001031BF0BCFA9A
:102BD0004D4B186805B0BDE8F04F1AF0D0BC4F451A
:102BE000DBD13A4640464D4921F09FFC0028D4D124
:102BF0004C4A82F800B0002200234B48CDE9002364
:102C00004FF40042002318F043FC394B39494C483B
:102C1000C91AC908890141F003011BF074FA1AF0BE
:102C2000B3FCC5E900012AE7D9F80030D9F8101043
:102C30001944D9F80430C91AFF290ADC2C4B2D4A53
:102C40004048D21AD208920142F002021BF068FA00
:102C5000BEE72988E1B14FF4004040F2E7384FF079
:102C60000009E1FB00894FF47A720023404649468F
:102C7000FEF774F902460B4600200021CDE9000161
:102C80002D4818F005FC1AF07FFCCAE90001F6E6B1
:102C90002D4817F025FEF6E7154B16492B48C91AA3
:102CA000C908890141F002011BF02DFAE7E6002274
:102CB000134B27491A80144B096818684FF4807227
:102CC00083681B699847014600283FF410AF084B02
:102CD000084A2048D21AD208920142F0020205B0F6
:102CE000BDE8F04F1BF01CBAB47101205C4C012010
:102CF000584E0400704E0400835D04008EDC0120F9
:102D000078C5012064710120B071012074C50120D3
:102D100070710120C9D501208E5D04009E5D040004
:102D2000384D0120CAD50120604A01208071012060
:102D3000A25D040076C50120F0490120CE5D0400AB
:102D4000B95D0400EA5D0400A0710120005E04008A
:102D5000E04501200B5E0400CDD50120C9C501204E
:102D60004A68184B1A60C2E6174B184A0979D21AFA
:102D7000D2089201164842F002021BF0D1F92379E1
:102D8000002B3FF4B4AE0122124B1A70AFE6124B87
:102D9000104D1B78012B04BF104A13702B78002BA9
:102DA0003FF4A5AE0E4C2678002E7FF4A0AE002393
:102DB0004FF480420B4817F0FDFD01232E70237065
:102DC00095E600BFE0450120584E0400704E040017
:102DD0001F5E0400CCD501208EDC0120CBD5012064
:102DE0008FDC0120404D012030B5504B8DB01B7859
:102DF0003BB109214E48FFF737FDFFF787FD0DB0C6
:102E000030BD4C4B1B88012B2CD94B4A4B4B1178B6
:102E1000C85C00F00300022808BF2039412921D1F5
:102E20005178585C00F00300022808BF203954296B
:102E300018D1927832B3252A03D002F0F702232A60
:102E400010D13F480446024610F8011B5D5C6D0737
:102E5000F9D1A24206D0A9B13D290ED03F2901D116
:102E600053787BB1374B38493848C91AC9088901AA
:102E700041F001011BF047F9BBE753783F2B01D12B
:102E80009378EEE72C4800F0F5FC10B906213048A5
:102E9000B1E710F16E0FB2D00230AAD126494FF43B
:102EA000805208460DF10F030EF022FE041E0DDACB
:102EB000244B254A2146D21AD2089201254842F0D5
:102EC00001021BF02DF901238DF80F301A48FEF78F
:102ED000A7FA50B102212048FFF7C6FC1648FEF7BA
:102EE0009FFA014614481AF05DFB9DF80F30032B42
:102EF00083D801A252F823F08D2E0200F32D020098
:102F0000092F0200272F0200144B009420220021D9
:102F100004A821F0C3FA04A8FEF782FA014604A827
:102F20001AF040FB69E70E4B0094EFE7C9D501208A
:102F30002F5E040074C50120C9C5012012B1040030
